:020000040800F2
:1000000000000220A9550008E11E0008E31E0008B8
:10001000E51E0008E71E0008E91E000800000000B9
:10002000000000000000000000000000EB1E0008BF
:10003000ED1E000800000000EF1E0008F11E000881
:10004000F9550008F9550008F9550008F955000858
:10005000F9550008F9550008F9550008F955000848
:10006000F9550008F9550008F9550008F955000838
:10007000F9550008F9550008F9550008F955000828
:10008000F9550008F9550008F9550008F955000818
:10009000F9550008F9550008F9550008F955000808
:1000A000F91E0008F9550008F9550008F95500082F
:1000B000F9550008F9550008F9550008F9550008E8
:1000C000F9550008F9550008F9550008F9550008D8
:1000D000F9550008F9550008F9550008F9550008C8
:1000E000F9550008F9550008F9550008F9550008B8
:1000F000F9550008F9550008F9550008F9550008A8
:10010000F9550008F9550008091F0008F9550008BD
:10011000F9550008F9550008F9550008F955000887
:10012000191F0008F9550008F9550008F95500088D
:10013000F95500080000000000000000F955000813
:10014000F9550008F9550008F9550008F955000857
:10015000F9550008F9550008F9550008F955000847
:10016000F9550008F9550008F9550008F955000837
:10017000F9550008F95500080000000000000000D3
:08018000F9550008F9550008CB
:1001900010B5054C237833B9044B13B10448AFF3C1
:1001A00000800123237010BDDC020020000000004D
:1001B0006880020808B5034B1BB103490348AFF33D
:1001C000008008BD00000000E002002068800208F6
:1001D00001F0FF01102A2BDB10F0070F08D010F8F8
:1001E000013B013A8B422DD010F0070F42B3F6D1FC
:1001F000F0B441EA012141EA014122F007047FF015
:1002000000070023F0E80256083C85EA010586EA6B
:10021000010685FA47F5A3FA87F586FA47F6A5FAA7
:1002200087F68EB9EED1F0BC01F0FF0102F00702B3
:1002300032B110F8013B013A83EA010313B1F8D15E
:100240000020704701387047002D06BF354603383F
:10025000073815F0010F07D1013015F4807F02BF78
:10026000013015F4C03F0130F0BC0138704700BFC9
:1002700010F8012B11F8013B012A28BF9A42F7D050
:10028000D01A7047034613F8012B002AFBD1181A25
:100290000138704781F0004102E000BF83F0004365
:1002A00030B54FEA41044FEA430594EA050F08BF11
:1002B00090EA020F1FBF54EA000C55EA020C7FEAD5
:1002C000645C7FEA655C00F0E2804FEA5454D4EB52
:1002D0005555B8BF6D420CDD2C4480EA020281EA1C
:1002E000030382EA000083EA010180EA020281EA54
:1002F0000303362D88BF30BD11F0004F4FEA0131A6
:100300004FF4801C4CEA113102D0404261EB4101B4
:1003100013F0004F4FEA03334CEA133302D052423A
:1003200063EB430394EA050F00F0A780A4F10104F6
:10033000D5F1200E0DDB02FA0EFC22FA05F2801830
:1003400041F1000103FA0EF2801843FA05F3594116
:100350000EE0A5F120050EF1200E012A03FA0EFC95
:1003600028BF4CF0020C43FA05F3C01851EBE371BF
:1003700001F0004507D54FF0000EDCF1000C7EEBDC
:1003800000006EEB0101B1F5801F1BD3B1F5001F1A
:100390000CD349085FEA30004FEA3C0C04F1010439
:1003A0004FEA445212F5800F80F09A80BCF1004F62
:1003B00008BF5FEA500C50F1000041EB045141EAE4
:1003C000050130BD5FEA4C0C404141EB0101013CAD
:1003D00028BFB1F5801FE9D291F0000F04BF01469C
:1003E0000020B1FA81F308BF2033A3F10B03B3F16E
:1003F00020020CDA0C3208DD02F1140CC2F10C02FE
:1004000001FA0CF021FA02F10CE002F11402D8BF5B
:10041000C2F1200C01FA02F120FA0CFCDCBF41EA27
:100420000C019040E41AA2BF01EB0451294330BDF6
:100430006FEA04041F3C1CDA0C340EDC04F11404D3
:10044000C4F1200220FA04F001FA02F340EA0300AA
:1004500021FA04F345EA030130BDC4F10C04C4F1F0
:10046000200220FA02F001FA04F340EA03002946D0
:1004700030BD21FA04F0294630BD94F0000F83F41A
:10048000801306BF81F480110134013D4EE77FEAFD
:10049000645C18BF7FEA655C29D094EA050F08BF49
:1004A00090EA020F05D054EA000C04BF194610462A
:1004B00030BD91EA030F1EBF0021002030BD5FEA6E
:1004C000545C05D14000494128BF41F0004130BD96
:1004D00014F580043CBF01F5801130BD01F00045EA
:1004E00045F0FE4141F470014FF0000030BD7FEA5D
:1004F000645C1ABF194610467FEA655C1CBF0B4658
:10050000024650EA013406BF52EA033591EA030F6E
:1005100041F4002130BD00BF90F0000F04BF002166
:10052000704730B54FF4806404F132044FF0000599
:100530004FF0000150E700BF90F0000F04BF002112
:10054000704730B54FF4806404F1320410F0004578
:1005500048BF40424FF000013EE700BF42004FEA73
:10056000E2014FEA31014FEA02701FBF12F07F43F0
:1005700093F07F4F81F06051704732F07F4208BFA7
:10058000704793F07F4F04BF41F40021704730B5AE
:100590004FF4607401F0004521F000411CE700BFFA
:1005A00050EA010208BF704730B54FF000050AE07D
:1005B00050EA010208BF704730B511F0004502D57E
:1005C000404261EB41014FF4806404F132045FEA80
:1005D000915C3FF4D8AE4FF003025FEADC0C18BF29
:1005E00003325FEADC0C18BF033202EBDC02C2F11B
:1005F000200300FA03FC20FA02F001FA03FE40EAAD
:100600000E0021FA02F11444BDE600BF70B54FF0B0
:10061000FF0C4CF4E06C1CEA11541DBF1CEA13558E
:1006200094EA0C0F95EA0C0F00F0DEF82C4481EAF6
:10063000030621EA4C5123EA4C5350EA013518BF16
:1006400052EA033541F4801143F4801338D0A0FB03
:1006500002CE4FF00005E1FB02E506F00042E0FBB0
:1006600003E54FF00006E1FB03569CF0000F18BFB6
:100670004EF0010EA4F1FF04B6F5007F64F540745E
:1006800004D25FEA4E0E6D4146EB060642EAC621F1
:1006900041EA55514FEAC52040EA5E504FEACE2E5E
:1006A000B4F1FD0C88BFBCF5E06F1ED8BEF1004F61
:1006B00008BF5FEA500E50F1000041EB045170BDDD
:1006C00006F0004646EA010140EA020081EA030121
:1006D000B4EB5C04C2BFD4EB0C0541EA045170BD1D
:1006E00041F480114FF0000E013C00F3AB8014F197
:1006F000360FDEBF002001F0004170BDC4F10004E0
:10070000203C35DA0C341BDC04F11404C4F1200560
:1007100000FA05F320FA04F001FA05F240EA0200BB
:1007200001F0004221F0004110EBD37021FA04F6F1
:1007300042EB06015EEA430E08BF20EAD37070BDAB
:10074000C4F10C04C4F1200500FA04F320FA05F00A
:1007500001FA04F240EA020001F0004110EBD3700C
:1007600041F100015EEA430E08BF20EAD37070BD7C
:10077000C4F1200500FA05F24EEA020E20FA04F355
:1007800001FA05F243EA020321FA04F001F0004104
:1007900021FA04F220EA020000EBD3705EEA430E75
:1007A00008BF20EAD37070BD94F0000F0FD101F0A4
:1007B0000046400041EB010111F4801F08BF013CDD
:1007C000F7D041EA060195F0000F18BF704703F01B
:1007D0000046520043EB030313F4801F08BF013DA2
:1007E000F7D043EA0603704794EA0C0F0CEA13555E
:1007F00018BF95EA0C0F0CD050EA410618BF52EA18
:100800004306D1D181EA030101F000414FF000001D
:1008100070BD50EA410606BF1046194652EA43062B
:1008200019D094EA0C0F02D150EA013613D195EA9F
:100830000C0F05D152EA03361CBF104619460AD1E7
:1008400081EA030101F0004141F0FE4141F47001F1
:100850004FF0000070BD41F0FE4141F4780170BDE1
:1008600070B54FF0FF0C4CF4E06C1CEA11541DBF46
:100870001CEA135594EA0C0F95EA0C0F00F0A7F848
:10088000A4EB050481EA030E52EA03354FEA013175
:1008900000F088804FEA03334FF0805545EA131388
:1008A00043EA12634FEA022245EA111545EA106550
:1008B0004FEA00260EF000419D4208BF964244F1E7
:1008C000FD0404F5407402D25B084FEA3202B61A06
:1008D00065EB03055B084FEA32024FF480104FF4DA
:1008E000002CB6EB020E75EB030E22BFB61A75464E
:1008F00040EA0C005B084FEA3202B6EB020E75EBE1
:10090000030E22BFB61A754640EA5C005B084FEA48
:100910003202B6EB020E75EB030E22BFB61A754615
:1009200040EA9C005B084FEA3202B6EB020E75EB20
:10093000030E22BFB61A754640EADC0055EA060EE1
:1009400018D04FEA051545EA16754FEA06164FEA24
:10095000C30343EA52734FEAC2025FEA1C1CC0D1D0
:1009600011F4801F0BD141EA00014FF000004FF05D
:10097000004CB6E711F4801F04BF01430020B4F11E
:10098000FD0C88BFBCF5E06F3FF6AFAEB5EB030CD6
:1009900004BFB6EB020C5FEA500C50F1000041EBD3
:1009A000045170BD0EF0004E4EEA113114EB5C04A0
:1009B000C2BFD4EB0C0541EA045170BD41F4801173
:1009C0004FF0000E013C90E645EA060E8DE60CEA7B
:1009D000135594EA0C0F08BF95EA0C0F3FF43BAF98
:1009E00094EA0C0F0AD150EA01347FF434AF95EA4F
:1009F0000C0F7FF425AF104619462CE795EA0C0F33
:100A000006D152EA03353FF4FDAE1046194622E7FF
:100A100050EA410618BF52EA43067FF4C5AE50EAD9
:100A200041047FF40DAF52EA43057FF4EBAE12E7C9
:100A30004FF0FF3C06E000BF4FF0010C02E000BFAA
:100A40004FF0010C4DF804CD4FEA410C7FEA6C5C8D
:100A50004FEA430C18BF7FEA6C5C1BD001B050EA30
:100A6000410C0CBF52EA430C91EA030F02BF90EA1B
:100A7000020F0020704710F1000F91EA030F58BFDA
:100A8000994208BF90422CBFD8176FEAE37040F03C
:100A9000010070474FEA410C7FEA6C5C02D150EADA
:100AA000013C07D14FEA430C7FEA6C5CD6D152EA95
:100AB000033CD3D05DF8040B704700BF844610465A
:100AC00062468C461946634600E000BF01B5FFF759
:100AD000B7FF002848BF10F1000F01BD4DF808ED29
:100AE000FFF7F4FF0CBF012000205DF808FB00BFFA
:100AF0004DF808EDFFF7EAFF34BF012000205DF854
:100B000008FB00BF4DF808EDFFF7E0FF94BF0120A0
:100B100000205DF808FB00BF4DF808EDFFF7CEFFA1
:100B200094BF012000205DF808FB00BF4DF808EDE0
:100B3000FFF7C4FF34BF012000205DF808FB00BFB1
:100B40004FEA410C7FEA6C5C02D150EA013C0AD1C9
:100B50004FEA430C7FEA6C5C02D152EA033C02D1BB
:100B60004FF0000070474FF0010070474FEA41021C
:100B700012F5001215D211D56FF47873B3EB6252EF
:100B800012D94FEAC12343F0004343EA505311F016
:100B9000004F23FA02F018BF404270474FF00000A8
:100BA000704750EA013005D111F0004008BF6FF0E6
:100BB000004070474FF00000704700BF4A0011D25C
:100BC00012F5001211D20DD56FF47873B3EB6252A7
:100BD0000ED44FEAC12343F0004343EA505323FAB3
:100BE00002F070474FF00000704750EA013002D128
:100BF0004FF0FF3070474FF0000070474FEA41025E
:100C0000B2F1E04324BFB3F5001CDCF1FE5C0DD96A
:100C100001F0004C4FEAC0024CEA5070B2F1004FB4
:100C200040EB830008BF20F00100704711F0804FB7
:100C300021D113F13872BCBF01F00040704741F47C
:100C400080114FEA5252C2F11802C2F1200C10FA80
:100C50000CF320FA02F018BF40F001004FEAC12364
:100C60004FEAD32303FA0CFC40EA0C0023FA02F308
:100C70004FEA4303CCE77FEA625307D150EA0133DE
:100C80001EBF4FF0FE4040F44000704701F00040AE
:100C900040F0FE4040F40000704700BF53B94AB92D
:100CA000002908BF00281CBF4FF0FF314FF0FF3074
:100CB00001F014B9ADF1080C6DE904CE00F03CF878
:100CC000DDF804E0DDE9022304B0704738B5002206
:100CD000002304460D46FFF70BFF28B9204629469E
:100CE000BDE8384000F00AB8204605F1004100F0A8
:100CF00005F8404261EB410138BD00BFD0B50C4B57
:100D0000002206460F46FFF781FCFFF757FF044617
:100D1000FFF702FC074B0022FFF778FC02460B4668
:100D200030463946FFF7BAFAFFF748FF2146D0BDF3
:100D30000000F03D0000F0412DE9F047089D044619
:100D40008E46002B4DD18A42944669D9B2FA82F27E
:100D500052B101FA02F3C2F1200120FA01F10CFABA
:100D600002FC41EA030E94404FEA1C48210CBEFBF2
:100D7000F8F61FFA8CF708FB16E341EA034306FB7B
:100D800007F199420AD91CEB030306F1FF3080F00A
:100D90001F81994240F21C81023E63445B1AA4B257
:100DA000B3FBF8F008FB103344EA034400FB07F7F9
:100DB000A7420AD91CEB040400F1FF3380F00A813A
:100DC000A74240F207816444023840EA0640E41B2F
:100DD00000261DB1D4400023C5E900433146BDE8DB
:100DE000F0878B4209D9002D00F0EF800026C5E97D
:100DF000000130463146BDE8F087B3FA83F6002E95
:100E00004AD18B4202D3824200F2F980841A61EB0C
:100E1000030301209E46002DE0D0C5E9004EDDE72A
:100E200002B9FFDEB2FA82F2002A40F09280A1EB12
:100E30000C014FEA1C471FFA8CFE0126200CB1FB67
:100E4000F7F307FB131140EA01410EFB03F0884260
:100E500008D91CEB010103F1FF3802D2884200F2ED
:100E6000CB804346091AA4B2B1FBF7F007FB10117F
:100E700044EA01440EFB00FEA64508D91CEB04041D
:100E800000F1FF3102D2A64500F2BB800846A4EB78
:100E90000E0440EA03409CE7C6F12007B34022FA63
:100EA00007FC4CEA030C20FA07F401FA06F31C4392
:100EB000F9404FEA1C4900FA06F3B1FBF9F8200C9F
:100EC0001FFA8CFE09FB181140EA014108FB0EF0E5
:100ED000884202FA06F20BD91CEB010108F1FF3A35
:100EE00080F08880884240F28580A8F10208614441
:100EF000091AA4B2B1FBF9F009FB101144EA01414F
:100F000000FB0EFE8E4508D91CEB010100F1FF34F9
:100F10006CD28E456AD90238614440EA0840A0FB91
:100F20000294A1EB0E01A142C846A64656D353D067
:100F30005DB1B3EB080261EB0E0101FA07F722FA8B
:100F400006F3F1401F43C5E9007100263146BDE8B4
:100F5000F087C2F12003D8400CFA02FC21FA03F317
:100F6000914001434FEA1C471FFA8CFEB3FBF7F098
:100F700007FB10360B0C43EA064300FB0EF69E42BD
:100F800004FA02F408D91CEB030300F1FF382FD256
:100F90009E422DD9023863449B1B89B2B3FBF7F6FE
:100FA00007FB163341EA034106FB0EF38B4208D9D7
:100FB0001CEB010106F1FF3816D28B4214D9023E18
:100FC0006144C91A46EA004638E72E46284605E736
:100FD0000646E3E61846F8E64B45A9D2B9EB020807
:100FE00064EB0C0E0138A3E74646EAE7204694E797
:100FF0004046D1E7D0467BE7023B614432E73046CA
:1010000009E76444023842E703685A004CBF43F0E2
:10101000004323F000431844704700BF2DE9F84314
:1010200029B34F1E044615463E464FF0000808EB14
:10103000060101EBD171491004EBC1094846FFF7E5
:10104000E3FF0346C80008308F42204409D0AB427A
:1010500009D8FFF7D9FF0138A8420AD201F10108E7
:10106000E5E7AB4205D9884501D04E1EDFE74FF0DA
:1010700000094846BDE8F883012807D0022807D0B8
:10108000044B00280CBF18460020704702487047E8
:1010900002487047511700085517000859170008F3
:1010A00030B5234B83B004468D1E3BB301A92846BF
:1010B000AFF30080E8B101992A46FFF7AFFF014680
:1010C000B8B1FFF7A1FF4B68A064012B2CD0002B17
:1010D00001F1040024DBFFF797FF0023C4E91303A9
:1010E0000368002B11DBFFF78FFF2061002003B0A6
:1010F00030BD00230920236103B030BD0D4B0E49E4
:10110000C91AC91018460191D6E7C3F30360FFF767
:10111000B3FF0028206114BF0020092003B030BDB8
:101120000123C4E91303DBE7002323610520DEE785
:10113000000000006CCA0208E4CB02080368DA076A
:1011400010B5044606D49B0700F1480009D500F00D
:101150005BFC2368590709D51A070ED5DB0613D5A2
:1011600010BD00F049FC23685907F5D404F1D00004
:1011700000F052FC23681A07F0D404F5A87000F0C0
:1011800053FC2368DB06EBD404F5E870BDE810409F
:1011900000F08EBC092070470346006800B1184477
:1011A000704700BF704700BF70B504460E46316CF3
:1011B0002046FFF775FF054688B9326C62612369E6
:1011C00032462146012098470828F0D0072806D14A
:1011D0002846316CFFF7E6FF301D00F001FC1EF0E1
:1011E00097F800BF2DE9F0470D1DD0F80C80D0F81E
:1011F0001890074614460FCDADF5727D0DF10C0C1D
:10120000ACE80F000FCDACE80F000FCDACE80F003D
:1012100095E80F0002AE4FF0000E8CE80F00C6F804
:1012200000E020E0336C7B614FF4F07231467AA825
:101230001EF0D8FE3B697AAA394650469847889BEB
:1012400073642146CDE9006905463B463A460120D4
:10125000C0470446E0B94FF4F0727AA930461EF058
:10126000C1FE082D1AD1316C3846FFF719FF093439
:101270005FFA84FA05460028D4D0B36B73643A460B
:10128000CDE900693B464AF010010120C04700B19A
:10129000092528460DF5727DBDE8F087072DF7D1A9
:1012A0002046316CFFF77EFF03A800F099FB00BFDA
:1012B000406C7047F0B5CB6B0B6401F1040C0E462B
:1012C0000546BCE80F00F9B001AC0FC4BCE80F0044
:1012D0000FC4BCE80F000FC49CE80F004FF0FF37AD
:1012E00084E80F00009706E02B696A462946984774
:1012F0000828044608D110992846FFF7D1FE002897
:10130000F2D0092079B0F0BD6846FFF717FF062C30
:10131000F7D131462846FFF747FF00BFC160D96BC0
:1013200082611964002219465CE700BF70B5C66887
:1013300043690B64AEB903690A4604460D4601468B
:1013400002209847072805D008280FD129462046B3
:10135000FFF72AFF3046296CFFF724FF281D00F015
:101360003FFB0122FFF73EFF1DF0D2FF1DF0D0FF33
:10137000C2681AB1CA6B0A64002233E79AE700BF59
:10138000704700BF836801460BB1012018477047C2
:10139000012912D009D873B90F2A0CD800EB8202A8
:1013A00018465368009A136070470339012994BFA7
:1013B000012002207047022070470846704700BF96
:1013C00000B585B00A46002303A900911946FFF72E
:1013D000DFFF039805B05DF804FB00BF012912D0C0
:1013E00009D873B90F2A0CD800EB8200009A126852
:1013F0004260184670470339012994BF012002203A
:101400007047022070470846704700BF10B584B08F
:10141000002303AC039200940A461946FFF7DEFF4F
:1014200004B010BD70B5D36B136402F1040C054613
:101430000C46BCE80F00ADF50E7D0DF15C0EAEE87C
:101440000F00BCE80F00AEE80F00BCE80F00AEE8EC
:101450000F009CE80F004FF0FF368EE80F00169645
:1014600010E0FFF7D3FF214616A8A847034616AAA7
:101470006946082083B9049B9847052806460CD086
:10148000092809D026996846FFF70AFE03466A46EE
:101490000C2116A8002BE4D0092616A8FFF74EFE53
:1014A00030460DF50E7D70BD2DE9F04FCC6C89B046
:1014B0001E4654F8043B06940D46174600F00308F8
:1014C000002E79D01A0C1B0405938DF81D200223E1
:1014D000D2B204EB82048DF81C302B6DB8F1020FF0
:1014E00008BFAC6B13F001030CD005A9384600F01F
:1014F00079FB18B9082009B0BDE8F08F092009B0C0
:10150000BDE8F08FD4F800A0BAF1000FEDD0019340
:1015100000F008030293022E4AD0B4F800A0B4F8F9
:1015200002900434AB6C29F0010B0F2138469B4428
:10153000FFF746FF834539D82AF001039B448345D2
:1015400094BF002001204FEA490303F002030AF090
:10155000010A43EA0A03012B49D0022B32D0002BA7
:10156000CCD1B8F1000F02D0002840F0CD80043477
:10157000D4F800A0BAF1000FCDD105A9384600F08B
:1015800031FB0028BAD1019B002BB3D00F21384684
:10159000FFF716FF0E2102463846FFF737FF3846A1
:1015A0006A4A0F21FFF732FF0720A8E70020CAE7A9
:1015B000D4F804900834B5E71B0205930323ADF873
:1015C0001C308AE7236823F0004BB8F1000F45D1A7
:1015D00028B1029A002A5CD0BBF1000F74D0002B16
:1015E00000DA04340BF1010B04EB8B04C0E7B8F113
:1015F000000F19D1B0B163682268991C4FEAD2720A
:101600003FF47CAF05F158010133049100F0908064
:10161000201DFFF7C1FD04AB0146284604F08CF8FD
:1016200000285BD10834A3E70D213846D5F8209077
:10163000FFF7C6FE8145F5D1AB6A9C42F2D1204648
:10164000FFF7E2FC0F2102463846FFF7DFFE38467F
:101650002A460021FFF7DAFE072050E70D21384621
:10166000D5F82090FFF7ACFE814501D02368B6E79E
:10167000AB6A9C42FAD104230022C5E90B23E3188C
:10168000C5F828B06B632368002B59DB0123019355
:10169000A8E705F15803CDF80C8004F1040AB04620
:1016A00091461E460EE050460496FFF775FD002257
:1016B000014604AB284609F101090AF1040A04F0C5
:1016C0003BF8E0B9D945EED10D213846FFF778FE59
:1016D000049BAC62C5E90803062010E781460D2192
:1016E0003846FFF76DFEB9F1020F286225D12B466F
:1016F000049A43F82C2F6B62AC620620FFE6464644
:101700002368DDF80C806AE72046FFF77DFC04348F
:101710000246AC632846144604F06CF800283FF4F7
:10172000EDAE384622460F21FFF770FE0720E6E6B1
:101730000D213846FFF744FE2862049B6B62DBE70D
:101740000BF1010004EB80007AE700BF19E101080A
:101750000023A9E60123A7E60223A5E62DE9F0432D
:101760000646C3B015461C46042900F2BF80DFE8D8
:1017700001F09E57BD2D0300002C40F0B780102AC9
:1017800000F2B4800368D80600F1F98020AF384633
:1017900000F098F9B46B394600234FF0010C0CFAB5
:1017A00003F22A42204603F1010303D050F8042B30
:1017B0000A600446042B01F10401F0D13846B463F9
:1017C00000F076F9002043B0BDE8F083032C40F030
:1017D0008D8094B204EB1243102B4FEA124500F2B5
:1017E000858003681F0700F1D28020AF384600F0E3
:1017F0003DF9B26B07EBC50154B10B46D01A01EBB2
:10180000C401E4001D5843F8045B8B42FAD1224422
:101810003846B26300F008F9002043B0BDE8F08319
:10182000012C4FEA124895B25CD0052C5ED108EB32
:101830000509B9F1200F59D8B8F10F0F79D9A94688
:10184000002D40F08A80B36B6DB320AF4FF00009DC
:1018500007EBC807043F03EBC50553F8041B47F823
:10186000041FAB42F9D1B9F1000F0FD06F464146CA
:10187000102938BF102107EBC101843903EBC905DA
:1018800053F8040B41F8040FAB42F9D1012C00F0DE
:101890008680B8F10F0FB56347D9B9F1000F02D0B8
:1018A000684600F0B9F8002043B0BDE8F083ECB919
:1018B000806B23461FFA82FC0124371D04FA03F2D1
:1018C00012EA0C0F014604D051F8042B47F82320EC
:1018D00008460133102BF1D115F40055E3D1B06364
:1018E000284604E008EB0503102B03D9022043B07F
:1018F000BDE8F083B8F10F0FF8D83368DA0706D5E2
:10190000304623F0030340F8483B00F079F820AF5D
:10191000384600F075F8B36B002D97D11D4604359D
:10192000B563384600F068F8BDE720A800F06CF811
:10193000B3E7B9F1100F40D9A9F110093368D907FD
:1019400008D523F00103304643F0020340F8483B3A
:1019500000F05EF8B9F1000F32D033685A0720D496
:10196000B8F10F0F25D96F463846C8F1100500F0C1
:1019700057F8002DB36B7FF77AAF20AF68E723F0FD
:101980001003336006F5E87000F09CF8FEE623F0E3
:101990000803036000F5A87000F068F825E720AFA1
:1019A000BDE7304623F0040340F8D03B00F038F8A0
:1019B000D6E720A800F02CF8D5E74FF00009BDE7E6
:1019C000B8F10F0F3FF63FAF20AF384600F020F8D8
:1019D000B36B002D7FF43AAF384600F015F862E79C
:1019E00000F1340191E838009C46A6464CF8045DAD
:1019F00090E8FF0FE54600BD90EC210B704700BF5B
:101A000080EC210B704700BF90EC200B704700BFAB
:101A100080EC200B704700BFD0EC200B704700BF5C
:101A2000C0EC200B704700BFF0EC0201F0EC02119B
:101A3000F0EC0221F0EC0231F0EC0241F0EC02514A
:101A4000F0EC0261F0EC0271F0EC0281F0EC02913A
:101A5000F0EC02A1F0EC02B1F0EC02C1F0EC02D12A
:101A6000F0EC02E1F0EC02F1704700BFE0EC0201A3
:101A7000E0EC0211E0EC0221E0EC0231E0EC02418A
:101A8000E0EC0251E0EC0261E0EC0271E0EC02817A
:101A9000E0EC0291E0EC02A1E0EC02B1E0EC02C16A
:101AA000E0EC02D1E0EC02E1E0EC02F1704700BFB3
:101AB000B0FC0181B0FC0191B0FC01A1B0FC01B10E
:101AC000704700BFA0FC0181A0FC0191A0FC01A116
:101AD000A0FC01B1704700BFEC4600B52DE90050F5
:101AE0002DE9FF1F4FF000032DE90C0001A9FFF7BE
:101AF000E1FBDDF840E012B0704700BFEC4600B5F6
:101B00002DE900502DE9FF1F4FF000032DE90C00D7
:101B100001A9FFF70BFCDDF840E012B0704700BFF1
:101B2000EC4600B52DE900502DE9FF1F4FF00003F2
:101B30002DE90C0001A9FFF71BFCDDF840E012B015
:101B4000704700BFEC4600B52DE900502DE9FF1F9E
:101B50004FF000032DE90C0001ABFFF7DFFBDDF8D0
:101B600040E012B0704700BFEC4600B52DE90050D0
:101B70002DE9FF1F4FF000032DE90C0001AAFFF72C
:101B800051FCDDF840E012B0704700BF027A034616
:101B90007AB9427AA2B14168013A10B44272086837
:101BA00003220C1D1A7202025C60000E10BC1A6047
:101BB00070470068013A1A7202021A60000E7047FC
:101BC000B020704700B585B0002303AA00921946E3
:101BD0000C22FFF7DDFB039805B05DF804FB00BFA6
:101BE000F0E700BF2DE9F043054685B00E464FF003
:101BF00000083046FFF7CAFFB028044600F0BA805C
:101C0000070620D500F0F003802B4DD0902B36D066
:101C1000A02B60D0B02B74D0C02B00F08B8000F0D4
:101C2000F803D02B0BD100F007020132052342F458
:101C3000002201212846FFF791FD0028D9D0092074
:101C400005B0BDE8F0838300DBB21F1D0DF10C0968
:101C500000231946CDF800900D222846FFF798FB87
:101C6000039BCDF8009060064CBFDF1BFF180023DC
:101C70000D22194628460397FFF7B0FBB9E700F09D
:101C80000D030D2BDBD003AF002300F00F0219462C
:101C900000972846FFF77CFB002300970D2219468A
:101CA0002846FFF79BFBA4E73046FFF76FFF2402AF
:101CB0002043B0F5004FC2D004010023A2B2194660
:101CC0002846FFF74BFD0028B9D114F4004F18BF88
:101CD0004FF001088DE7C24302F007034FF47F6223
:101CE0001A41010702F47F624FF0000348BF42F43B
:101CF000804219462846FFF731FD00283FF479AFAE
:101D00009DE7B1283BD0B22800F09380B32841D0A2
:101D100000F0FC03B42B92D000F007020132012343
:101D200042F4002219462846FFF718FD00283FF428
:101D300060AF84E7C6284AD0C72854D000F0F80323
:101D4000C02B63D0C82868D0C9287FF478AF30464C
:101D5000FFF71CFF020300F00F0002F470220130B5
:101D60000243012105232846FFF7F8FC00283FF431
:101D700040AF64E7B8F1000F18D0002060E73046AC
:101D8000FFF704FF024600283FF459AF10F0F003BC
:101D9000C8D054E73046FFF7F9FE020300F00F0306
:101DA000013302F470221A430123BBE703AC43461C
:101DB0000E22414600942846FFF7EAFA0094434673
:101DC0000F2241462846FFF709FB404638E73046D8
:101DD000FFF7DCFE020300F00F03013302F4702270
:101DE0001A4303239EE73046FFF7D0FE0246002841
:101DF0003FF425AF10F0F0037FF421AF0421284613
:101E0000FFF7ACFC00283FF4F4AE18E700F00F0237
:101E10000132032342F4202284E73046FFF7B6FE66
:101E200000F0F00200F00F031032013343EA0232F7
:101E300097E700230DF10C090D221946CDF800900B
:101E40002846FFF7A5FA3046FFF7A0FE02064FF03E
:101E500002040CD5039B00F07F00A04018440390BF
:101E60003046FFF793FE030604F10704F2D4039B08
:101E7000CDF8009000F07F02A24003F501731A44F0
:101E80000023039219460D222846FFF7A7FAB0E671
:101E900010B5C26C536884B04FF0030C08321C02BA
:101EA00008461B0E01A9019402928DF80CC08DF812
:101EB0000D30FFF797FE04B010BD00BF08B5FFF767
:101EC0008FFE806C08BD00BF08B5FFF789FEC06CAF
:101ED000C379023300EB830008BD00BF704700BF29
:101EE000FEE7FEE7FEE7FEE7FEE770477047704754
:101EF00008B501F055FA08BD08B5024801F09EFB8F
:101F000008BD00BF0404002008B5024801F096FB9C
:101F100008BD00BF2405002008B5024801F0A6F85E
:101F200008BD00BF4C03002082B0002100910B4B84
:101F30005A6C42F480425A645A6C02F48042009215
:101F4000009A01911A6C42F080521A641B6C03F0E3
:101F500080530193019B02B0704700BF00380240DC
:101F600070B588B0002303930493059306930793F9
:101F7000026803F1804303F590339A4201D008B020
:101F800070BD04460025009503F58C335A6C42F46D
:101F900080725A645A6C02F480720092009A019521
:101FA0001A6B42F004021A631A6B02F004020192E7
:101FB000019A02951A6B42F001021A631B6B03F03F
:101FC00001030293029B012303930326049603A9B2
:101FD000144800F079FE0F2303930496059503A996
:101FE000114800F071FE1148114B03604560856097
:101FF000C5604FF4806303614FF4006343614FF4A5
:10200000005383614FF48073C3610562456200F041
:10201000C7FF18B9054BA3639C63B0E702F034FE19
:10202000F8E700BF00080240000002404C03002017
:102030001064024000B589B0002303930493059314
:10204000069307930268154B9A4202D009B05DF8D7
:1020500004FB0021019103F5FE331A6C42F40042A7
:102060001A641A6C02F400420192019A02911A6BEE
:1020700042F004021A631B6B03F004030293029BF9
:102080004FF4E053039302230493032306930623A0
:10209000079303A9024800F017FED7E7003C004071
:1020A0000008024000B585B00368284A93420BD06F
:1020B000B3F1804F1CD0264A934226D0254A934242
:1020C00030D005B05DF804FB00210091224B5A6C22
:1020D00042F001025A645B6C03F001030093009B21
:1020E0000A46182001F0C2F8182001F0F7F8E8E7D6
:1020F00000230193184B1A6C42F001021A641B6C06
:1021000003F001030193019BDBE700230293124BD1
:102110001A6C42F002021A641B6C03F00203029371
:10212000029BCEE7002103910B4B1A6C42F0080290
:102130001A641B6C03F008030393039B0A463220C6
:1021400001F094F8322001F0C9F8BAE7000001402C
:1021500000040040000C00400038024000B589B087
:102160000023039304930593069307930268134B8C
:102170009A4202D009B05DF804FB0021019103F5F9
:102180000C331A6C42F004021A641A6C02F0040256
:102190000192019A02911A6B42F002021A631B6BC0
:1021A00003F002030293029BC023039302230493D0
:1021B000079303A9024800F087FDDBE70008004011
:1021C0000004024000B589B00023039304930593F3
:1021D00006930793026803F1804303F582339A4222
:1021E00002D009B05DF804FB0021019103F59A3398
:1021F0005A6C42F002025A645A6C02F002020192D6
:10220000019A02911A6B42F004021A631B6B03F0ED
:1022100004030293029BC02303930223049303232A
:10222000079303A9014800F04FFDDAE700080240D8
:1022300070B588B000230393049305930693079326
:102240000368B3F1804F04D0234A93422ED008B0E4
:1022500070BD0024009403F50E331A6B42F00102A6
:102260001A631A6B02F001020092009A01941A6B31
:1022700042F002021A631B6B03F002030193019BFD
:1022800020230393022604960125079503A91348EA
:1022900000F01AFD4FF4006303930496059406942E
:1022A000079503A90E4800F00FFDD0E70023029325
:1022B0000C4B1A6B42F002021A631B6B03F0020311
:1022C0000293029B3023039302230493079303A9F1
:1022D000034800F0F9FCBAE70004004000000240A7
:1022E000000402400038024000B589B00023039387
:1022F0000493059306930793026803F1804303F563
:1023000088339A4202D009B05DF804FB00210191A4
:1023100003F594335A6C42F010025A645A6C02F07E
:1023200010020192019A02911A6B42F001021A63A3
:102330001B6B03F001030293029B4FF4C0630393F2
:1023400002230493032306930723079303A9024858
:1023500000F0BAFCD7E700BF000002404A4B5A68C1
:1023600022F440325A605A6841680A435A6002684F
:10237000536823F48073536002685368016943EA29
:10238000012353600268536823F04073536002686E
:10239000536881680B4353600268936823F40063B9
:1023A000936002689368C1680B439360826A374BFD
:1023B0009A4257D00268936823F070639360026872
:1023C0009368816A0B4393600268936823F04053DB
:1023D000936002689368C16A0B43936002689368D4
:1023E00023F00203936002689368017E43EA41038D
:1023F000936090F82030002B3FD00268536843F47C
:10240000006353600268536823F4604353600168BB
:102410004B68426A013A43EA42334B600268D36A2E
:1024200023F47003D3620168CB6AC269013A43EABC
:102430000253CB620268936823F4007393600268CE
:10244000936890F8301043EA4123936002689368E0
:1024500023F48063936002689368416943EA8123AF
:10246000936070470268936823F07063936002681A
:10247000936823F040539360B0E70268536823F4F5
:1024800000635360CAE700BF002301400100000F52
:1024900038B310B50446036C43B1236C13F0100F2E
:1024A0000BD00120002384F83C3010BDFFF758FD0D
:1024B0000023636484F83C30EFE7236C23F48853F3
:1024C00023F0020343F0020323642046FFF746FF94
:1024D00000206064236C23F0030343F001032364B2
:1024E000E0E701207047000030B482B00023019380
:1024F00090F83C30012B00F0BB80012380F83C3089
:102500000B68092B41D90468E2689BB203EB4303D3
:102510001E3B4FF0070C0CFA03F322EA0303E360BF
:102520000468E2680B8803EB43031E3B8D6805FAE1
:1025300003F31343E3604B68062B3DD80468626BDA
:1025400003EB8303053B4FF01F0C0CFA03F322EA65
:10255000030363630468626B4B6803EB8303053B0F
:10256000B1F800C00CFA03F3134363630268414BF4
:102570009A4251D002683F4B9A4256D0002380F8CD
:102580003C30184602B030BC7047046822699BB2E8
:1025900003EB43034FF0070C0CFA03F322EA0303A7
:1025A0002361046822690B8803EB43038D6805FAF5
:1025B00003F313432361BEE70C2B16D805682A6B7F
:1025C00003EB8303233B1F2404FA03F322EA0303F0
:1025D0002B6305682A6B4B6803EB8303233B0C8852
:1025E00004FA03F313432B63C0E70568EA6A03EBBD
:1025F0008303413B1F2404FA03F322EA0303EB6243
:102600000568EA6A4B6803EB8303413B0C8804FAD4
:1026100003F31343EB62A9E70B68122BAAD1164A06
:10262000536843F480035360A4E70B68103B012B0D
:10263000A4D8114A536843F4000353600B68102B6D
:102640009CD10E4B1B6802F1467202F52E3202F24B
:102650008332A2FB03239B0C03EB83035B000193F8
:1026600002E0019B013B0193019B002BF9D185E71F
:10267000022087E700200140002301400C000020D9
:10268000002800F0E08170B582B00446036813F0C2
:10269000010F3BD09F4B9B6803F00C03042B2CD005
:1026A0009C4B9B6803F00C03082B21D06368B3F5A7
:1026B000803F4FD0B3F5A02F52D0964B1A6822F42A
:1026C00080321A601A6822F480221A606368002B34
:1026D00050D000F071FE05468E4B1B6813F4003F8E
:1026E00014D100F069FE401B6428F5D90320B1E144
:1026F000884B5B6813F4800FD8D0864B1B6813F4AB
:10270000003F03D06368002B00F09F81236813F023
:10271000020F54D07F4B9B6813F00C0F3ED07D4BC3
:102720009B6803F00C03082B33D0E368002B68D0C0
:10273000794B01221A6000F03FFE0546754B1B687D
:1027400013F0020F54D100F037FE401B0228F5D9D8
:1027500003207FE16F4A136843F480331360B5E7C9
:102760006C4B1A6842F480221A601A6842F4803274
:102770001A60ABE700F020FE0546664B1B6813F4B9
:10278000003FC3D000F018FE401B6428F5D9032099
:1027900060E1604B5B6813F4800FC6D15D4B1B6832
:1027A00013F0020F03D0E368012B40F05081594A27
:1027B000136823F0F803216943EAC1031360236817
:1027C00013F0080F42D063696BB3534B0122C3F877
:1027D000802E00F0F1FD05464E4B5B6F13F0020FAB
:1027E00034D100F0E9FD401B0228F5D9032031E186
:1027F000484A136823F0F803216943EAC1031360D0
:10280000DDE7454B00221A6000F0D6FD0546414B3E
:102810001B6813F0020FD2D000F0CEFD401B02283F
:10282000F5D9032016E13C4B0022C3F8802E00F0BE
:10283000C3FD0546374B5B6F13F0020F06D000F067
:10284000BBFD401B0228F5D9032003E1236813F0E8
:10285000040F77D02F4B1B6C13F0805F33D1002314
:1028600001932C4B1A6C42F080521A641B6C03F0DB
:1028700080530193019B0125284B1B6813F4807F33
:1028800023D0A368012B34D0052B38D0214B1A6FED
:1028900022F001021A671A6F22F004021A67A36875
:1028A000002B3DD000F088FD06461A4B1B6F13F03D
:1028B000020F46D100F080FD801B41F28833984220
:1028C000F3D90320C6E00025D6E7144A136843F481
:1028D0008073136000F070FD0646104B1B6813F404
:1028E000807FCED100F068FD801B0228F5D903203F
:1028F000B0E0084A136F43F001031367CFE7054BBD
:102900001A6F42F004021A671A6F42F001021A6746
:10291000C5E700BF00380240000047420070004099
:1029200000F04AFD0646524B1B6F13F0020F08D011
:1029300000F042FD801B41F288339842F3D9032016
:1029400088E0EDB9A369002B00F08380484A9268C3
:1029500002F00C02082A51D0022B17D0454B00225E
:102960001A6600F029FD0446414B1B6813F0007FF6
:1029700042D000F021FD001B0228F5D9032069E0B8
:102980003B4A136C23F080531364DBE7394B00227E
:102990001A6600F011FD0546354B1B6813F0007FE9
:1029A00006D000F009FD401B0228F5D9032051E0B4
:1029B000E369226A1343626A43EA8213A26A5208F5
:1029C000013A43EA0243E26A43EA0263284A536057
:1029D000284B01221A6600F0EFFC0446244B1B68CA
:1029E00013F0007F06D100F0E7FC001B0228F5D9A8
:1029F00003202FE000202DE000202BE0012B2BD026
:102A00001B4B5B6803F48001E269914226D103F01D
:102A10003F02216A8A4223D1616A47F6C0721A4096
:102A2000B2EB811F1ED103F44031A26A5208013A71
:102A3000B1EB024F18D103F07063E26AB3EB026F9F
:102A400014D1002006E001207047012002E001209F
:102A500000E0002002B070BD0120FBE70120F9E793
:102A60000120F7E70120F5E70120F3E70120F1E776
:102A7000003802400000474208B5254B9B6803F030
:102A80000C03042B3FD0082B3FD1214B5A6802F096
:102A90003F025B6813F4800F12D01D4B5968C1F3DD
:102AA00088111C480023A1FB0001FEF7F7F8184B22
:102AB0005B68C3F3014301335B00B0FBF3F025E037
:102AC000134B5968C1F3881C4FEA4C11B1EB0C0051
:102AD0006EEB0E0E4FEA8E1343EA90638101091AE2
:102AE00063EB0E03DB0043EA5173C90011EB0C0CDE
:102AF00043F10003990200234FEA8C2041EA9C51E4
:102B0000FEF7CCF8D3E7034800E0034808BD00BF58
:102B10000038024040787D010024F400002800F0D5
:102B20009B8070B50D4604464F4B1B6803F00703AE
:102B30008B4208D2CBB24C4A1370136803F00703E0
:102B40008B4240F08B80236813F0020F17D013F0F4
:102B5000040F04D0454A936843F4E053936023681C
:102B600013F0080F04D0414A936843F46043936024
:102B70003E4A936823F0F003A1680B4393602368F7
:102B800013F0010F32D06368012B21D09A1E012A65
:102B900025D9364A126812F0020F61D033498A688B
:102BA00022F0030213438B6000F006FC06462F4B15
:102BB0009B6803F00C036268B3EB820F16D000F041
:102BC000FBFB801B41F288339842F0D9032042E09E
:102BD000264A126812F4003FE0D101203BE0234A6C
:102BE000126812F0007FD9D1012034E01E4B1B681F
:102BF00003F00703AB4207D9EAB21B4B1A701B68FC
:102C000003F00703AB422DD1236813F0040F06D065
:102C1000164A936823F4E053E1680B4393602368FA
:102C200013F0080F07D0114A936823F46043216919
:102C300043EAC1039360FFF71FFF0C4B9B68C3F38C
:102C400003130B4AD35CD8400A4B18600A4B186830
:102C500000F066FB002070BD012070470120FAE7FC
:102C60000120F8E70120F6E7003C0240003802406E
:102C7000948002080C00002008000020014B186816
:102C8000704700BF0C00002008B5FFF7F7FF044BAA
:102C90009B68C3F38223034AD35CD84008BD00BFBE
:102CA00000380240A480020808B5FFF7E7FF044B94
:102CB0009B68C3F34233034AD35CD84008BD00BFCE
:102CC00000380240A480020800230F2B00F2E480A9
:102CD00070B582B060E085685E000324B44025EAE8
:102CE0000405CC68B4402C438460456825EA02059D
:102CF0004C68C4F300129A402A4342605AE0DC0850
:102D0000083450F8246003F0070295000F22AA400F
:102D100026EA020E0A69AA4042EA0E0240F824207E
:102D20005CE0072200E0002202FA0EF22A4302349D
:102D30005A4D45F824205A4A94686FEA0C0224EA56
:102D40000C054E6816F4801F01D04CEA0405544C63
:102D5000A560E46802EA04054E6816F4001F01D07D
:102D60004CEA04054E4CE560646802EA04054E68CE
:102D700016F4003F01D04CEA0405494C6560246814
:102D800022404D6815F4803F01D04CEA0402444CC7
:102D9000226001330F2B7DD801229A400C6804EA8F
:102DA000020C32EA0404F4D14C6804F00304013C40
:102DB000012C90D94A6802F00302032A09D0C468A2
:102DC0005D000322AA4024EA02048A68AA40224342
:102DD000C2604A6802F00302022A90D004684FEAF7
:102DE000430E032202FA0EF224EA02044A6802F0B9
:102DF000030202FA0EF2224302604A6812F4403FD4
:102E0000C7D000220192274A546C44F48044546491
:102E1000526C02F480420192019A9C08A51C1F4A40
:102E200052F8255003F003024FEA820E0F2202FAF5
:102E30000EF225EA02051C4A90423FF474AF02F5F7
:102E4000806290421AD002F58062904218D002F55A
:102E50008062904216D002F58062904214D002F552
:102E60008062904212D002F58062904210D002F54A
:102E7000806290423FF455AF082255E7012253E7A4
:102E8000022251E703224FE704224DE705224BE7D8
:102E9000062249E702B070BD704700BF003801400C
:102EA000003C014000380240000002400AB181614C
:102EB0007047090481617047436901EA030221EA0E
:102EC000030141EA024181617047000010B40368C8
:102ED000D9B210390C4AA2FB014212090B4CA25C78
:102EE000C2655F2909D923F47F7323F003030433F8
:102EF0008365806D5DF8044B704723F47F7323F086
:102F000003038365F5E700BFABAAAAAA8C80020879
:102F1000836A826992B9012B0AD0022B02D00BB1CD
:102F200000207047C36A13F0807F28D100207047CB
:102F3000C36AB3F1C07F24D000207047B2F5005FB0
:102F400009D0022B25D9032B25D1C36A13F0807F2A
:102F500023D100207047032B03D8DFE803F01404CB
:102F6000140A00207047C36A13F0807F0DD100203F
:102F70007047C36AB3F1C07F09D0002070470120B9
:102F800070470120704701207047012070470120E1
:102F900070470120704700207047012070470000F3
:102FA00070B5044600F008FA002C5BD005460223F9
:102FB00084F83530002384F834302268136823F015
:102FC0000103136023681A6812F0010F0AD000F0A1
:102FD000F3F9431B052BF5D920236365032084F8FF
:102FE000350070BD1A68204810406168A2680A4325
:102FF000E1680A4321690A4361690A43A1690A43F6
:10300000E1690A43216A0A430243616A04291ED026
:103010001A602668756925F00705636A1D43042B4D
:1030200007D1A36A1D43E36A1BB12046FFF770FF77
:1030300090B975612046FFF749FFE26D3F23934049
:10304000836000206065012384F83530C9E7E16AB8
:10305000206B01430A43DBE740236365012084F8CA
:103060003500BEE70120BCE73F8010F0F0B583B02B
:10307000044600230193724B1D68724BA3FB053578
:10308000AD0A876D3E68C26D08239340334210D06D
:1030900003681A6812F0040F0BD01A6822F00402B9
:1030A0001A60C26D08239340BB60436D43F0010377
:1030B0004365E26D01239340334209D0226852698F
:1030C00012F0800F04D0BB60636D43F002036365B0
:1030D000E26D04239340334209D02268126812F053
:1030E000020F04D0BB60636D43F004036365E26DBF
:1030F00010239340334224D02268126812F0080F44
:103100001FD0BB6023681A6812F4802F0DD01B6893
:1031100013F4002F04D1236C9BB12046984710E094
:10312000A36C73B1204698470BE01A6812F4807FB5
:1031300003D11A6822F008021A60236C0BB12046F2
:103140009847E26D20239340334255D0226812689D
:1031500012F0100F50D0BB6094F83530DBB2052B65
:103160000ED023681A6812F4802F33D01B6813F432
:10317000002F2AD1636C002B3ED0204698473BE0BD
:103180002268136823F0160313602268536923F042
:1031900080035361236CA3B12268136823F00803F2
:1031A0001360E26D3F239340BB60012384F8353008
:1031B000002384F83430236D002B3FD020469847FD
:1031C0003CE0A36C002BE7D1EBE7E36BA3B1204617
:1031D000984711E01A6812F4807F09D11A6822F02A
:1031E00010021A60012384F83530002384F834304B
:1031F000E36B0BB120469847636DFBB1636D13F031
:10320000010F17D0052384F835302268136823F0A6
:1032100001031360019B01330193AB4204D823687F
:103220001B6813F0010FF5D1012384F8353000231A
:1032300084F83430E36C0BB12046984703B0F0BDFE
:103240000C000020B5814E1B074AD36823F4E063CD
:103250001B041B0C000200F4E060034343F0BF6357
:1032600043F40033D360704700ED00E000B5194B24
:10327000DB68C3F30223C3F1070CBCF1040F28BFC2
:103280004FF0040C03F1040EBEF1060F18D9033BF6
:103290004FF0FF3E0EFA0CFC21EA0C0199400EFAA9
:1032A00003F322EA0303194300280BDB0901C9B227
:1032B00000F1604000F5614080F800135DF804FB08
:1032C0000023E5E700F00F000901C9B2024B1954D1
:1032D000F4E700BF00ED00E014ED00E0002807DB9C
:1032E00000F01F02400901239340024A42F82030B7
:1032F000704700BF00E100E00138B0F1807F0BD2E1
:103300004FF0E0235861054AF02182F82310002095
:10331000986107221A6170470120704700ED00E0B4
:1033200010B504460E4B18784FF47A73B3FBF0F3E4
:103330000C4A1068B0FBF3F0FFF7DEFF68B90F2C02
:1033400001D901200AE0002221464FF0FF30FFF7AB
:103350008DFF054B1C60002000E0012010BD00BF68
:10336000040000200C0000200800002008B50B4BD2
:103370001A6842F400721A601A6842F480621A6095
:103380001A6842F480721A600320FFF75DFF0F2075
:10339000FFF7C6FFFEF7C8FD002008BD003C024055
:1033A000034A1168034B1B780B441360704700BF3E
:1033B000F802002004000020014B1868704700BF8D
:1033C000F802002038B50446FFF7F6FF0546B4F1D1
:1033D000FF3F02D0044B1B781C44FFF7EDFF401B5E
:1033E000A042FAD338BD00BF0400002000285AD004
:1033F00010B50446436A33B94368B3F5827F05D0FC
:103400000023C36102E00023036143610023A36240
:1034100094F85130002B40D0022384F851302268B8
:10342000136823F040031360636803F48273A26897
:1034300002F404421343E26802F400621343226977
:1034400002F002021343626902F001021343A2690F
:1034500002F400721343E26902F038021343226A55
:1034600002F080021343A26A02F40052216813435F
:103470000B60638B03F00403626A02F010022168A0
:1034800013434B602268D36923F40063D3610020A7
:103490006065012384F8513010BD84F85030204617
:1034A000FEF7C8FDB8E701207047000030B4036A9A
:1034B000026A22F0010202624268846924F0730405
:1034C0000D682C4323F0020C8B6843EA0C03104D6B
:1034D000A84203D005F58065A84205D123F0080372
:1034E000CD682B4323F00403094DA84203D005F512
:1034F0008065A84205D122F440724D692A438D6946
:103500002A43426084614A684263036230BC704768
:103510000000014030B4036A026A22F48072026241
:103520004268C46924F0730C0C6844EA0C0523F467
:1035300000738C6843EA0423114CA04203D004F5C5
:103540008064A04206D123F40063CC6843EA0423DC
:1035500023F480630A4CA04203D004F58064A042A7
:1035600007D122F440524C6942EA04128C6942EAC3
:1035700004124260C5614A68C263036230BC70478E
:103580000000014030B4036A026A22F480520262F1
:103590004468C26922F4E6420D6842EA052223F437
:1035A00000538D6843EA0533094DA84203D005F561
:1035B0008065A84204D124F480444D6944EA85140E
:1035C0004460C2614A680264036230BC704700BF55
:1035D0000000014010B4036A046A24F0010404628C
:1035E000846924F0F00C4CEA021223F00A030B4326
:1035F000826103625DF8044B704710B4036A046A89
:1036000024F010040462846924F4704C4CEA023201
:1036100023F0A00343EA0113826103625DF8044BC7
:103620007047836823F070030B4343F00703836004
:1036300070477047704770477047704770B50446D1
:103640000368DE681D6915F0020F10D016F0020F36
:103650000DD06FF002021A610123037703689B69A2
:1036600013F0030F5ED0FFF7E6FF0023237715F07A
:10367000040F12D016F0040F0FD023686FF004026D
:103680001A610223237723689B6913F4407F4FD08C
:103690002046FFF7D0FF0023237715F0080F12D044
:1036A00016F0080F0FD023686FF008021A61042388
:1036B00023772368DB6913F0030F40D02046FFF720
:1036C000BAFF0023237715F0100F12D016F0100F59
:1036D0000FD023686FF010021A6108232377236844
:1036E000DB6913F4407F31D02046FFF7A4FF0023AD
:1036F000237715F0010F02D016F0010F2DD115F030
:10370000800F02D016F0800F2FD115F0400F02D09D
:1037100016F0400F31D115F0200F02D016F0200F17
:1037200033D170BDFFF786FF2046FFF785FF9CE78A
:103730002046FFF77FFF2046FFF77EFFABE72046DE
:10374000FFF778FF2046FFF777FFBAE72046FFF73D
:1037500071FF2046FFF770FFC9E723686FF0010291
:103760001A61204601F03AFDC9E723686FF0800234
:103770001A61204600F006FCC7E723686FF040029C
:103780001A612046FFF759FFC5E723686FF0200252
:103790001A61204600F0F5FBC3E700000368344AD5
:1037A000904212D0B0F1804F0FD0A2F57C429042EF
:1037B0000BD002F58062904207D002F58062904201
:1037C00003D002F57842904203D123F070034A6897
:1037D0001343274A90422AD0B0F1804F27D0A2F558
:1037E0007C42904223D002F5806290421FD002F5C5
:1037F000806290421BD002F57842904217D002F5C9
:103800007052904213D002F5806290420FD002F5C0
:10381000806290420BD0A2F59832904207D002F518
:103820008062904203D002F58062904203D123F47B
:103830004073CA68134323F080034A69134303604B
:103840008B68C3620B688362094B984203D003F50F
:103850008063984201D10B690363012343610369CB
:1038600013F0010F03D0036923F0010303617047D4
:103870000000014040B310B5044690F83D30F3B16C
:10388000022384F83D30214651F8040BFFF786FFF0
:10389000012384F8463084F83E3084F83F3084F8C1
:1038A000403084F8413084F8423084F8433084F862
:1038B000443084F8453084F83D30002010BD80F855
:1038C0003C30FEF7EFFBDBE70120704740B310B55B
:1038D000044690F83D30F3B1022384F83D30214690
:1038E00051F8040BFFF75AFF012384F8463084F89F
:1038F0003E3084F83F3084F8403084F8413084F81A
:10390000423084F8433084F8443084F8453084F8F9
:103910003D30002010BD80F83C30FEF71FFCDBE797
:103920000120704740B310B5044690F83D30F3B124
:10393000022384F83D30214651F8040BFFF72EFF97
:10394000012384F8463084F83E3084F83F3084F810
:10395000403084F8413084F8423084F8433084F8B1
:10396000443084F8453084F83D30002010BD80F8A4
:103970003C30FFF75EFEDBE701207047002856D0A1
:10398000F8B50D46044690F83D30002B4AD002238E
:1039900084F83D302268936823F4804323F00703C2
:1039A0009360214651F8040BFFF7F8FE21688A68FE
:1039B0008B690E6A2868104323F4407C2CF0030CBA
:1039C000AA68AB6942EA032343EA0C0323F47C436D
:1039D00023F0FC03EA69EF6847EA022C4CEA030C87
:1039E0002A6A13032A6943EA021343EA0C0326F006
:1039F000AA066A686D6942EA051232438860216846
:103A00008B6123681A62012384F8463084F83E30C3
:103A100084F83F3084F8423084F8433084F83D30F5
:103A20000020F8BD80F83C30FEF7CCFBAFE701206A
:103A30007047000030B4036A026A22F0100202628A
:103A40004468826922F4E6420D6842EA052223F0C6
:103A500020038D6843EA0513114DA84203D005F5F4
:103A60008065A84206D123F08003CD6843EA0513A0
:103A700023F040030A4DA84203D005F58065A84213
:103A800007D124F440644D6944EA85048D6944EA11
:103A90008504446082614A688263036230BC704777
:103AA0000000014090F83C30012B28D010B50446AE
:103AB000012380F83C300C2A1CD8DFE802F0071BF9
:103AC0001B1B0C1B1B1B111B1B1B16000068FFF78D
:103AD000EDFC00200FE00068FFF7ACFF00200AE0DB
:103AE0000068FFF717FD002005E00068FFF74AFDBA
:103AF000002000E00120002384F83C3010BD0220AB
:103B0000704738B590F83C30012B66D004460D461E
:103B1000012380F83C300C2A5AD8DFE802F007591C
:103B200059591B5959593059595944000068FFF7E0
:103B3000BDFC2268936943F008039361226893698E
:103B400023F0040393612268936929690B4393610D
:103B500000203EE00068FFF76DFF2268936943F4A0
:103B6000006393612268936923F480639361226800
:103B70009369296943EA01239361002029E00068E1
:103B8000FFF7C8FC2268D36943F00803D3612268B9
:103B9000D36923F00403D3612268D36929690B43F5
:103BA000D361002015E00068FFF7ECFC2268D369C0
:103BB00043F40063D3612268D36923F48063D36143
:103BC0002268D369296943EA0123D361002000E018
:103BD0000120002384F83C3038BD0220FCE710B4FB
:103BE000846824F47F4C42EA03220A4342EA0C022E
:103BF00082605DF8044B704790F83C30012B78D020
:103C000010B50446012380F83C30022380F83D3093
:103C10000268936823F47F4323F0770393600B6873
:103C2000602B4CD029D8402B54D00CD9502B22D10A
:103C3000CA6849680068FFF7CDFC50212068FFF78B
:103C4000F0FC002005E0202B0DD009D9302B0AD044
:103C50000120012384F83D30002384F83C3010BD5E
:103C60000BB1102B05D119462068FFF7DAFC0020B4
:103C7000EFE70120EDE70120EBE7B3F5805F34D0FB
:103C8000B3F5005F0CD1CB684A6889680068FFF71C
:103C9000A6FF2268936843F4804393600020D8E72E
:103CA000702B24D1CB684A6889680068FFF797FFBA
:103CB0002268936843F0770393600020C9E7CA68DD
:103CC00049680068FFF799FC60212068FFF7A9FCAC
:103CD0000020BEE7CA6849680068FFF77BFC402106
:103CE0002068FFF79EFC0020B3E70020B1E7012029
:103CF000AFE70220704701F01F01012303FA01FC26
:103D0000036A23EA0C030362036A02FA01F10B431C
:103D10000362704710B504460846002942D194F862
:103D20003E30DBB2013B18BF0123002B6ED10028CF
:103D300051D1022384F83E30012201462068FFF76A
:103D4000DAFF2368334A934203D002F5806293423C
:103D500003D15A6C42F400425A6423682D4A9342BC
:103D600049D0B3F1804F46D0A2F57C42934242D075
:103D700002F5806293423ED002F5806293423AD0CF
:103D800002F57842934236D002F57052934232D017
:103D9000A2F5943293422ED01A6842F001021A60C2
:103DA000002032E0042908D008290DD094F84130D1
:103DB000DBB2013B18BF0123B7E794F83F30DBB219
:103DC000013B18BF0123B0E794F84030DBB2013B60
:103DD00018BF0123A9E7042805D0082807D002232B
:103DE00084F84130A8E7022384F83F30A4E7022397
:103DF00084F84030A0E79A6802F00702062A07D04C
:103E00001A6842F001021A60002010BD0120FCE790
:103E10000020FAE70000014038B504460D460022B4
:103E20000068FFF768FF23681D4A934218D002F527
:103E30008062934214D02368196A41F21112114230
:103E400008D1196A40F24442114203D11A6822F0A3
:103E500001021A609DB9012384F83E30002038BD6C
:103E6000196A41F211121142E5D1196A40F2444235
:103E70001142E0D15A6C22F400425A64DBE7042D6F
:103E800005D0082D07D0012384F84130E6E701234F
:103E900084F83F30E2E7012384F84030DEE700BFDA
:103EA0000000014090F83C30012B3DD010B40123BC
:103EB00080F83C30022380F83D3003685A689C68E3
:103EC00022F0700C0A6842EA0C025A600368174A32
:103ED00093421AD0B3F1804F17D0A2F57C4293429F
:103EE00013D002F5806293420FD002F580629342B4
:103EF0000BD002F57842934207D002F570529342FC
:103F000003D0A2F59432934204D124F080044A688D
:103F100014439C60012380F83D30002380F83C303E
:103F200018465DF8044B70470220704700000140BE
:103F300090F83C30012B22D0012380F83C30CB6834
:103F400023F440738A68134323F480634A6813435D
:103F500023F400630A68134323F480530A6913436C
:103F600023F400534A69134323F48043CA6913437B
:103F700002685364002380F83C30184670470220E2
:103F8000704770477047026802F10C0353E8003F26
:103F900023F490730C3242E800310029F3D1026817
:103FA00002F1140353E8003F23F00103143242E806
:103FB00000310029F3D1036B012B05D0202380F8B9
:103FC0004230002303637047026802F10C0353E898
:103FD000003F23F010030C3242E800310029F3D1F6
:103FE000ECE7000038B504460268136923F4405337
:103FF000C1680B4313618368026913434269134329
:10400000C2691A430168CB6823F4164323F00C03FA
:104010001343CB600268536923F4407381690B43F7
:1040200053610368314A934206D002F5806293429D
:1040300002D0FEF729FE01E0FEF736FEE369B3F594
:10404000004F29D00021031849411B1841F10001FC
:10405000C90041EA5371DB00181863684FEA830214
:104060004FEA937341F10001FCF718FE204DA5FBC8
:1040700000325109642303FB11031B013233A5FBFA
:1040800003235B0903F0F00202EB011203F00F03BC
:10409000216813448B6038BD0023021843EB0301F1
:1040A000121841F10001C90041EA5271D200101802
:1040B00041F10001626892185B41FCF7EFFD0C4D85
:1040C000A5FB00325109642303FB1103DB003233EB
:1040D000A5FB03235B095A0002F4F87202EB0112FC
:1040E00003F00703216813448B60D4E700100140FC
:1040F0001F85EB512DE9F04383B005460E46174668
:104100009946DDF828802C68246836EA04030CBF41
:104110004FF0010C4FF0000CBC4528D1B8F1FF3F27
:10412000F1D0FFF749F9A0EB0900404523D8B8F1D9
:10413000000F22D02B68DA6812F0040FE3D0802E33
:10414000E1D0402EDFD01A6812F0080FDBD0002437
:1041500001941A6801925B680193019B2846FFF75E
:1041600012FF08236B6485F84040012000E0002026
:1041700003B0BDE8F0830320FAE70320F8E760B35B
:1041800010B5044690F8413013B3242384F841302D
:104190002268D36823F40053D3602046FFF722FF40
:1041A0002268136923F4904313612268536923F052
:1041B0002A0353612268D36843F40053D36000207C
:1041C0006064202384F8413084F84230606310BD7D
:1041D00080F84030FEF788F8D7E7012070472DE9D6
:1041E000F04182B01E4690F84130DBB2202B56D110
:1041F00004460D469046002955D00AB901204FE0EB
:1042000000234364212380F84130FFF7D5F80746A7
:10421000A4F82480A4F82680A368B3F5805F02D0B8
:104220004FF0000814E023692BB34FF000080FE0B3
:10423000202384F84130032032E038F8023B226822
:10424000C3F308035360E28C92B2013A92B2E28463
:10425000E38C9BB293B100963B460022802120461E
:10426000FFF748FF0028E3D1002DE6D015F8012B19
:1042700023685A60E7E7A8460025E9E700963B4631
:10428000002240212046FFF735FF18B9202384F88B
:10429000413005E0202384F84130032000E0022073
:1042A00002B0BDE8F0810120FAE70000034AD2F82D
:1042B000883043F47003C2F88830704700ED00E0A6
:1042C00010B503460C4A0D490D48006840B10C4832
:1042D00000680344521A934206D8094A136010BD7D
:1042E0000748084C0460F2E71BF072F80C230360E7
:1042F0004FF0FF30F3E700BF000002200004000091
:10430000FC020020B81C00200120704708B51BF0FB
:104310005FF8162303604FF0FF3008BD08B54FF07B
:10432000FF31FFF7F3FFFEE770B50C461646002598
:1043300006E0AFF30080214601F8010B01350C4681
:10434000B542F6DB304670BD70B50C46164600250A
:1043500004E014F8010B00F0B7FB0135B542F8DBBF
:10436000304670BD4FF0FF3070474FF400534B6044
:1043700000207047012070470020704700B595B0BD
:104380003022002108A81BF055FE0023039304935C
:1043900005930693079301931F4A116C41F08051D6
:1043A0001164126C02F080520192019A02931B4A2E
:1043B000116841F480411160126802F48042029257
:1043C000029A0222089201210B9110210C910E9267
:1043D0000F9308231093A82311931292042313938D
:1043E00008A8FEF74DF988B90F230393022304931D
:1043F000002305934FF4A05306930793052103A8C8
:10440000FEF78CFB28B915B05DF804FB00F03CFC0E
:10441000EAE700F039FCF6E700380240007000409F
:1044200000B585B0002300930193029303932D48B8
:104430002D4A02604360836001220261037680F8A6
:104440002030C36202F170628262C3600522C261E1
:1044500080F830304361FEF71BF800282FD101238C
:1044600000930193029369461E48FEF73DF848BB4E
:10447000032300930223019369461A48FEF734F898
:1044800018BB002300930323019369461548FEF7E8
:104490002BF8E8B9022300930423019369461148DD
:1044A000FEF722F8B8B90A23009305230193694661
:1044B0000C48FEF719F888B905B05DF804FB00F068
:1044C000E3FBCCE700F0E0FBD2E700F0DDFBD8E750
:1044D00000F0DAFBDEE700F0D7FBE4E700F0D4FB06
:1044E000EAE700BF040300200020014008B50E48A1
:1044F0000E4B03604FF48273436000238360C360FC
:10450000036143614FF4007282612022C261036241
:10451000436283620A23C362FEF768FF00B908BDE5
:1045200000F0B2FBFBE700BFAC030020003C004002
:1045300010B596B00024129413941494159410940A
:10454000119409940A940B940C940D940E940F9466
:104550002022214601A81BF06DFD2B482B4B036048
:1045600053234360846040F2E733C36004614461D5
:104570008461FFF77FF9002833D14FF48053129301
:1045800012A92148FFF738FB00282DD11E48FFF75C
:104590009DF900282BD100231093119310A91A48DC
:1045A000FFF780FC30BB002209920A920B920C921A
:1045B0000D920E920F9209A91348FFF773FAE0B912
:1045C0000023019302930393049305934FF4005245
:1045D0000692089301A90C48FFF7AAFC80B916B00F
:1045E00010BD00F051FBC8E700F04EFBCEE700F035
:1045F0004BFBD0E700F048FBD5E700F045FBDFE7D9
:1046000000F042FBEBE700BF040400200000014083
:1046100000B58FB000230A930B930C930D9308936E
:1046200009930193029303930493059306930793CD
:1046300025484FF0804202604360836040F2E732D9
:10464000C26003618361FFF715F950BB4FF48053DB
:104650000A930AA91C48FFF7CFFA28BB1A48FFF7AC
:1046600061F920BB00230893099308A91648FFF7B6
:1046700019FCF8B96023019300220292039205927B
:1046800001A91148FFF73DFAB8B90C2201A90E485B
:10469000FFF737FAA0B90C48FDF7CAFD0FB05DF877
:1046A00004FB00F0F1FAD1E700F0EEFAD6E700F0F3
:1046B000EBFAD7E700F0E8FADCE700F0E5FAE4E728
:1046C00000F0E2FAE7E700BF4C04002000B58FB02D
:1046D00000230A930B930C930D9308930993019372
:1046E0000293039304930593069307932548264A60
:1046F000026053224260836040F2E732C26003618D
:104700008361FFF7B7F858BB4FF480530A930AA9A7
:104710001C48FFF771FA30BB1A48FFF703F928BBB2
:1047200000230893099308A91648FFF7BBFB00BBB9
:1047300060230193002202920392059201A911487D
:10474000FFF7DFF9C0B904220DEB02010D48FFF7B6
:10475000D8F9A0B90B48FDF76BFD0FB05DF804FB6D
:1047600000F092FAD0E700F08FFAD5E700F08CFA6B
:10477000D6E700F089FADBE700F086FAE3E700F01D
:1047800083FAE7E7940400200004004000B593B0EA
:10479000242200210DEB02001BF04CFC00230793A8
:1047A0000893009301930293039304930593069354
:1047B0001F48204A0260436083604EF65F22C26059
:1047C00003618361FFF782F830BB03230993002361
:1047D0000A9301220B920C930D930E930F92109358
:1047E000119309A91248FFF7C9F8C0B9002307932C
:1047F000089307A90E48FFF755FB98B900230093CB
:10480000019302930493082269460948FFF74AF985
:1048100058B913B05DF804FB00F036FAD5E700F0A4
:1048200033FAE3E700F030FAE8E700F02DFAF0E7BA
:10483000DC0400200008004000B587B0002302938C
:10484000039304930593009301931548154A02605E
:1048500053224260836040F2E732C26003618361A9
:10486000FFF708F890B94FF48053029302A90C485F
:10487000FFF7C2F968B9002300930193694608481D
:10488000FFF710FB40B907B05DF804FB00F0FCF93E
:10489000E9E700F0F9F9EEE700F0F6F9F3E700BF19
:1048A00024050020000C004000B58DB0242200211A
:1048B00003A81BF0BFFB0023019302931248134A85
:1048C0000260436083604EF65F22C2600361436111
:1048D00083610323039301230593099303A9FFF73E
:1048E0004DF850B900230193029301A90648FFF740
:1048F000D9FA28B90DB05DF804FB00F0C5F9F1E76D
:1049000000F0C2F9F6E700BF6C050020000401408A
:1049100008B50A480A4B03604FF4E13343600023B3
:104920008360C36003610C2242618361C361FFF74E
:1049300026FC00B908BD00F0A7F9FBE7B40500208C
:104940000010014000B583B000210191094B1A6BA2
:1049500042F480021A631B6B03F480030193019BF2
:104960000A463820FEF782FC3820FEF7B7FC03B079
:104970005DF804FB003802402DE9F0478AB00024BE
:10498000059406940794089409940094484B1A6B74
:1049900042F004021A631A6B02F004020092009AB9
:1049A00001941A6B42F080021A631A6B02F08002C3
:1049B0000192019A02941A6B42F001021A631A6B77
:1049C00002F001020292029A03941A6B42F0020270
:1049D0001A631A6B02F002020392039A04941A6B90
:1049E00042F008021A631B6B03F008030493049B54
:1049F000304E22464FF440413046FEF757FADFF87A
:104A0000BCA0224603215046FEF750FADFF8B090D2
:104A1000224649F640014846FEF748FADFF8A480EE
:104A200022464BF203414046FEF740FA224F22460F
:104A300004213846FEF73AFA4FF440430593012526
:104A400006950794089405A93046FEF73DF903231F
:104A5000059306950794089405A95046FEF734F986
:104A60003E2305930694079405A93046FEF72CF9DA
:104A700049F64003059306950794089405A948460E
:104A8000FEF722F94BF20343059306950794089429
:104A900005A94046FEF718F90423059306950794E7
:104AA000089405A93846FEF70FF90AB0BDE8F0876B
:104AB0000038024000080240000C0240001C024086
:104AC000000002400004024000B583B08DF80700EA
:104AD00001231A460DF107010248FFF780FB03B0DE
:104AE0005DF804FBB4050020012800D070474FF6A4
:104AF000FF739942FAD110B5044C204601F03AFAFE
:104B0000034A0449204600F078FD10BDFC05002052
:104B100000000020DD61000870B50446806A10B115
:104B200003681B6A98470023A362666AA6B19EB118
:104B300076B106F11C0501E000232B60AE4207D0E0
:104B400055F8040D0028F7D0082100F0CFFDF3E759
:104B50001C21304600F0CAFD00236362256A5DB166
:104B600055B1A86810B1202100F0C0FD0023AB6052
:104B70000C21284600F0BAFD00232362E06910B141
:104B8000042100F0B3FD0023E361A06910B10C2102
:104B900000F0ACFD0023A361606910B1202100F09A
:104BA000A5FD00236361206910B1042100F09EFD82
:104BB00000232361E06810B1082100F097FD002375
:104BC000E360A06810B1182100F090FD0023A360FD
:104BD000606810B1012100F089FD00236360206846
:104BE00010B11C2100F082FD00232360204670BD1F
:104BF00010B58CB0FEF7BAFBFFF7C0FBFFF7BCFEA9
:104C0000FFF7A0FEFFF70CFCFFF770FCFFF790FC2E
:104C1000FFF7FEFCFFF75AFDFFF7B8FDFFF70CFEAC
:104C2000FFF742FEFFF774FE12481CF013F8124C17
:104C30001249204612F044FD12F08FFC1049204624
:104C400012F03EFD0F4912F03BFD4FF47A70FEF773
:104C5000B9FB2C22002101A81BF0ECF901A800F0FF
:104C600041F801A800F0A6F9FEE701A8FFF754FFFC
:104C700000F03EFDAC800208DC080020B480020891
:104C8000C0800208D080020872B6FEE708B54FF671
:104C9000FF710120FFF728FF08BD0000012800D0A8
:104CA00070474FF6FF739942FAD110B5044C204675
:104CB00001F060F9034A0449204600F09EFC10BD53
:104CC0000006002000000020DD61000810B5044649
:104CD000006810B1082100F009FD00232360204680
:104CE00010BD000030B597B0082001F05CF8044614
:104CF0004FF48052A74900F01FFA0EE00623C3F1DB
:104D0000060308AA02EB830408AB9C4200F025814D
:104D1000043C2046FFF7DAFFF6E7002308930894E7
:104D2000082001F040F804464FF40052994900F081
:104D300003FA07E00523E2E70821204600F0D6FC4D
:104D40000623DCE7002309930994082001F02BF8DF
:104D500004464FF400428F4900F0EEF907E00423C7
:104D6000CDE70821204600F0C1FC0523C7E700235A
:104D70000A930A94082001F016F804464022864956
:104D800000F0DAF905E00821204600F0AFFC04232A
:104D9000B5E700230B930B94082001F004F80446B8
:104DA0004FF480527C4900F0C7F907E00223A6E7E0
:104DB0000821204600F09AFC0323A0E700230C936F
:104DC0000C94082000F0EFFF04464FF40062724993
:104DD00000F0B2F907E0012391E70821204600F036
:104DE00085FC02238BE700230D930D94082000F02F
:104DF000DAFF04464FF40042674900F09DF907E0EE
:104E000000237CE70821204600F070FC012376E7B0
:104E100000230E930E9408AA06230FA9002B0DDB86
:104E2000106841F8040B002042F8040B013BF5E741
:104E30000821204600F05AFC002360E70FA901A8D2
:104E400000F0E8FA16AC01E0002323600FAB9C42AF
:104E500007D054F8040D0028F6D0082100F046FCD5
:104E6000F2E7012419E06420FEF7ACFA0DE008AC8B
:104E700001AB9C4200F0878054F8040D10B108216A
:104E800000F034FC00232360F2E7294601A800F07B
:104E900003FB01E008ACEBE70134072C05DCE5B2CD
:104EA000294601A800F0C8FADDE701240FE008ACAC
:104EB000DEE76420FEF786FA01E008ACD8E7294671
:104EC00001A800F019FB01E008ACD1E70134082C7F
:104ED00005DCE5B2294601A800F00EFBE9E70FACBE
:104EE00001E00023236008AB9C4207D054F8040D76
:104EF0000028F6D0082100F0F9FBF2E708AC01E049
:104F00000023236001AB9C4207D054F8040D002815
:104F1000F6D0082100F0EAFBF2E708AC01E000233C
:104F2000236001AB9C4207D054F8040D0028F6D052
:104F3000082100F0DBFBF2E70FAC01E00023236067
:104F400008AB9C4223D054F8040D0028F6D0082169
:104F500000F0CCFBF2E70323D1E600F0C9FB16AC6E
:104F60000FAB9C4204D0043C2046FFF7AFFEF7E7AE
:104F70000FAC08AB9C4208D0043C2046FFF7A6FECD
:104F8000F7E708AC74E70FACF3E700F0B1FB17B03C
:104F900030BD00BF000402400000024010B50446CE
:104FA000006810B1202100F0A1FB002323602046FF
:104FB00010BD000010B586B0202000F0F4FE0446BD
:104FC00004222B4900F030F9002304930494059443
:104FD000049305A901A800F0D1F905E0202120469D
:104FE00000F084FB00F084FB059810B1202100F054
:104FF0007DFB002305939FED1F0A4FF42F7101A83D
:1050000000F0C1F94FF47A70FEF7DCF901A800F066
:10501000D0F94FF4FA70FEF7D5F99FED160A4FF468
:105020007A72114601A800F0C9F9049810B1202144
:1050300000F05CFB00230493039810B1202100F0E2
:1050400055FB00230393049810B1202100F04EFB80
:105050000023049306B010BD05A8FFF79FFF04A826
:10506000FFF79CFF00F044FB03A8FFF797FFF6E76C
:10507000940400200000A04208B54FF6FF71012003
:10508000FFF70CFE08BD0000012800D070474FF666
:10509000FF739942FAD110B5044C204600F06AFF24
:1050A000034A0449204600F0A8FA10BD0406002077
:1050B00000000020DD61000808B54FF6FF710120F7
:1050C000FFF7E2FF08BD0000012800D070474FF64F
:1050D000FF739942FAD110B5044C204600F04AFF04
:1050E000034A0449204600F088FA10BD0806002053
:1050F00000000020DD61000808B54FF6FF710120B7
:10510000FFF7E2FF08BD0000012800D070474FF60E
:10511000FF739942FAD110B5044C204600F02AFFE3
:10512000034A0449204600F068FA10BD0C0600202E
:1051300000000020DD61000801608280704708B532
:10514000012281880068FDF7B1FE08BD08B5002284
:1051500081880068FDF7AAFE08BD08B5818800684F
:10516000FDF7AAFE08BD08B54FF6FF710120FFF755
:10517000CBFF08BD012800D070474FF6FF7399425E
:10518000FAD110B5044C204600F0F4FE034A04495D
:10519000204600F032FA10BD20060020000000205A
:1051A000DD6100080146002300E00133032B08D82D
:1051B000054A52F823000028F7D002688A42F4D149
:1051C00000E00020704700BF1006002008B502482C
:1051D0001BF040FD08BD00BFD480020808B5FFF7F2
:1051E000E1FF08B1FFF7F2FF08BD08B54FF6FF7108
:1051F0000120FFF7BFFF08BD012800D070474FF620
:10520000FF739942FAD110B5044C204600F0B2FE6B
:10521000034A0449204600F0F0F910BD240600209E
:1052200000000020DD61000810B504460023C360C3
:1052300000202061636121606260CB68A360FDF79C
:1052400023FD4000A06123685B68E361204610BD38
:1052500008B541680068FEF75DFD08BD9FED1C7A4A
:10526000C0EE077AC0ED047AF5EEC07AF1EE10FADE
:1052700006DBB7EE007AF4EEC77AF1EE10FA06D943
:1052800043688BB903681B68C2685A6370478368B8
:10529000013307EE103AB8EE477A67EE277AFCEE54
:1052A000E77AC0ED037AEBE7042B06D0082B09D090
:1052B00003681B68C2681A64704703681B68C26889
:1052C0009A63704703681B68C268DA63704700BF5F
:1052D0000000C84241618369C26902FB0111B3FB4E
:1052E000F1F3013B836002681268D3620268D36005
:1052F000704708B541680068FEF78EFD08BD08B527
:105300004FF6FF710120FFF777FF08BD012800D09D
:1053100070474FF6FF739942FAD110B5044C2046FE
:1053200000F028FE034A0449204600F066F910BD4B
:105330002806002000000020DD61000808B54FF6B7
:10534000FF710120FFF7E2FF08BD0000012800D037
:1053500070474FF6FF739942FAD110B5044C2046BE
:1053600000F008FE034A0449204600F046F910BD4B
:105370002C06002000000020DD6100080B6883601F
:1053800000230B60704738B52DED028B04460D46A7
:10539000B0EE408A8068FFF75BFF2946A068FFF700
:1053A00099FFB0EE480AA068FFF758FFBDEC028BEA
:1053B00038BD08B58068FFF79CFF08BD38B50446C6
:1053C0001546FFF7E0FF2846FDF7FCFF2046FFF7F4
:1053D000F0FF38BD08B54FF6FF710120FFF7B6FFAB
:1053E00008BD0000012800D070474FF6FF739942B6
:1053F000FAD110B5044C204600F0BCFD034A044924
:10540000204600F0FAF810BD300600200000002011
:10541000DD61000802460623002B0CDB10B40C688B
:1054200042F8044B002441F8044B013B002BF6DA10
:105430005DF8044B7047704738B5044601390729B9
:1054400008D8DFE801F004080C1014181C200068CC
:10545000FFF775FE38BD4068FFF771FEFAE7806818
:10546000FFF76DFEF6E7C068FFF769FEF2E7006937
:10547000FFF765FEEEE74069FFF761FEEAE7806946
:10548000FFF75DFEE6E70025062DE3DC54F8250076
:10549000FFF755FE0135F7E738B50446013907290E
:1054A00008D8DFE801F004080C1014181C2000686C
:1054B000FFF74CFE38BD4068FFF748FEFAE780680A
:1054C000FFF744FEF6E7C068FFF740FEF2E7006929
:1054D000FFF73CFEEEE74069FFF738FEEAE7806938
:1054E000FFF734FEE6E70025062DE3DC54F825003F
:1054F000FFF72CFE0135F7E738B5044601390729D7
:1055000008D8DFE801F004080C1014181C2000680B
:10551000FFF723FE38BD4068FFF71FFEFAE78068FB
:10552000FFF71BFEF6E7C068FFF717FEF2E700691A
:10553000FFF713FEEEE74069FFF70FFEEAE7806929
:10554000FFF70BFEE6E70025062DE3DC54F8250007
:10555000FFF703FE0135F7E708B54FF6FF710120AD
:10556000FFF740FF08BD0000012800D070474FF64C
:10557000FF739942FAD110B5044C204600F0FAFCB2
:10558000034A0449204600F038F810BD34060020D4
:1055900000000020DD61000808B54FF6FF71012012
:1055A000FFF7E2FF08BD0000DFF834D0FEF77EFE13
:1055B0000C480D490D4A002302E0D458C45004336E
:1055C000C4188C42F9D30A4A0A4C002301E0136044
:1055D0000432A242FBD31AF057FBFFF709FB7047D6
:1055E0000000022000000020DC0200202CCC020879
:1055F000DC020020B81C0020FEE70B4601461846DE
:1056000019F0D8BE7FB500241023CDE90234036819
:1056100015469E6912686B46CDE90044B0479DF877
:10562000043003F00603062B03BF009B2B60012010
:10563000204604B070BD0098904214BF012006209F
:105640007047000010B5034B0360044600F03FFCB8
:10565000204610BD1881020810B50446FFF7F2FF7E
:105660002046082100F042F8204610BD2DE9F04107
:105670001F46DDE90834DDF81880984506461546D2
:1056800007D1079900F026FC18B165710020BDE82C
:10569000F0813946304600F01DFC0028F6D0012389
:1056A000C4F800802571A371F0E738B515461C4693
:1056B00000F010FC20B10823E3600623256023716D
:1056C00038BD73B505460C4601921E4600F002FC3B
:1056D00050B9032E08D82368019A5B6929462046F1
:1056E00002B0BDE87040184702B070BD18F088BC29
:1056F0001EB400F09CF81EBCFCF700FA0378472BA0
:1057000017D143784E2B14D18378552B11D1C37800
:10571000432B0ED10379432B0BD143792B2B08D18B
:1057200083792B2B05D1C07901288CBF0020012063
:1057300070470020704700002DE9F3411D460378B3
:10574000472B0E460246C17913D143784E2B10D118
:105750008378552B0DD1C378432B0AD10379462B7F
:1057600007D143794F2B04D18379522B01D10029E2
:1057700031D01046FFF7C2FF80F00100C4B2002311
:105780000020019053BB5CBB01290ABF52F8203CAA
:10579000A2F12003783B012908BF52F8202C1C6895
:1057A00018BF58320192236820469B689847C8B1B9
:1057B000019B1B6801930227336801AAD3F810806C
:1057C000214601233046C04770B1019B2B6038460B
:1057D00002B0BDE8F08101230C46D1E7034CE2E7BB
:1057E000034CE0E70127E7E70746F0E73C810208C2
:1057F0004481020810B5044600F032F80246204603
:10580000A4F12001FFF77AFF60B154F8043C0133A2
:10581000012B44F8043C03D1936844F8083C9160A0
:10582000012010BD9368002BF9D000F0A5FA10B547
:1058300000F016F8826801460AB900F09DFA02F1FC
:1058400020042046FFF75AFF40B1D369013BD361E2
:1058500013B9906988609361204610BD8860FBE7AA
:10586000004870473806002030B500231A4610F86B
:10587000015B05F07F04944023432C0602F10702EC
:10588000F5D40B6030BD30B500231A4610F8014B3B
:1058900004F07F0595402B43250602F10702F5D45D
:1058A0001F2A06D8640642BF4FF0FF3404FA02F202
:1058B00013430B6030BD50282DE9F341064688465E
:1058C00015461F4608D1033222F0030050F8044B5E
:1058D0003C6002B0BDE8F08100F00F030C2B2ED825
:1058E000DFE803F025071D25292D2D2D2D18212555
:1058F000290001A92846FFF7B7FF019C002CE7D03B
:1059000006F07003102B08BFA8464444330648BF76
:105910002468DDE701A92846FFF7B5FFEDE7284633
:1059200030F8024BEAE7284630F9024BE6E7284612
:1059300050F8044BE2E7284650F8084BDEE719F030
:10594000E7FC08B50346FF2B084610D003F07002B1
:10595000302A12D007D8202A0BD002D813F0600FBB
:1059600005D019F0D5FC402A0BD0502AF9D10020DF
:1059700008BDBDE8084022F074BBBDE8084022F035
:105980006DBBBDE80840FCF799BA13B50C4601465B
:105990002046CDE90032FFF7D4FFDDE900320146B1
:1059A000204602B0BDE81040FFF785BF73B50C4636
:1059B0001546064628B3FCF781FA034620462B60BD
:1059C00010F8011BFF291ED002462B1D3046FFF7A1
:1059D000DCFF10F8013B2B75FF2B16D010232B7525
:1059E00001A9FFF741FF019B0344EB6010F8013B65
:1059F0006B7501A9FFF738FF019B03442B6102B0CF
:105A000070BD0346DAE76B60E3E70023EDE71FB5FF
:105A100003AB009300230A461946FBF7B9FC039831
:105A200005B05DF804FB00002DE9F04F91B00023B4
:105A3000059300F00303012B06460C4617460ED0D3
:105A4000022B03D0002B3BD101073BD53946204622
:105A5000FCF71EFA90B3092011B0BDE8F08F0207E1
:105A600006D40D6A38460D21FFF7D1FF85422BD0B1
:105A70000220002306F008060DF1280A0643CDF89F
:105A800000A00C22194638460A94FBF7A7FC062E04
:105A90001CD1D4F83080D4E90A59B8F1000F0CBFFA
:105AA0004FF0010B4FF0030B16F0080600F00781D2
:105AB000BBF1010F40F0FF8000F05EF90820CBE75A
:105AC00019F026FC0120D4E70620D2E73846FCF77F
:105AD000FBF981460028B9D0524601463846FFF707
:105AE00065FF394605469DF83C00FFF72AFF0F2168
:105AF0000C903846FFF78BFF20F0010808F1FF38C3
:105B00000E9BAB4240F2BF802A469DF83D1006AB8B
:105B10000020FFF73AFF9DF83D10024607AB00203A
:105B2000FFF733FF08AB02469DF83D100020FFF75A
:105B30002CFF09A9FFF798FE0A9B069A13444345D8
:105B4000054601D90E9DDBE7079A13444345D7D993
:105B5000DDF82080B8F1000F01D00B9B9844099D1F
:105B600015B10E98013D0544B8F1000F3FF46EAF3A
:105B7000002D00F0F28016F00803029334D0472382
:105B800023704E2363705523A3704323E370462391
:105B900023714F2363715223A3710023E3714FF0EC
:105BA000000B07A92846FFF76EFE08A90390FFF730
:105BB0006AFE0799002963D03ADD9DF83C00FF2872
:105BC00032D000F00703042B3FF67AAF01A252F85F
:105BD00023F000BF2D5C0008C15A0008FB5B0008E1
:105BE0002D5C0008255C0008E379012B0CBF54F8FC
:105BF000203C04F158030593D1E702250D9A09AB27
:105C000005FB11220C99FFF756FE099931B15CB3DF
:105C100005AB00222046FFF78FFD28B3079D4FF00C
:105C2000030B34E00825E9E70025E7E70425E5E76D
:105C3000C1F17F5101F57F110D9B01F57F513F317E
:105C400003EB8105BCB1029AAAB9059B0993043DF7
:105C500055F8041F0029E1D009AB00222944204651
:105C6000FFF76AFD0028F3D0089D002D71D0039B3B
:105C70002B441D4695E753F82130002BF4D1CDE796
:105C80004FF0010BF0E70025A8464FF0010BF3079A
:105C90007FF50AAFBBF1020F3FF4D8AE0D213846B5
:105CA000059EFFF7B4FEC4E90A59C4E90806C4F822
:105CB00030800620D0E6002D22DA00F06FF8BBF12C
:105CC000010F02D1204618F018FA002D18DA5246BA
:105CD00049463846FFF76AFE9DF83C003946FFF713
:105CE00030FE0D9A0C90EB4302EB830353F8262011
:105CF0000AB10136FAE70422C4E90A60C4E90C23B8
:105D0000002309AE1A461946009638460994FBF757
:105D100065FB002319460122009638460995FBF7DA
:105D20005DFB0F213846FFF772FE00F0010040EAEC
:105D300008000023099000960F2219463846FBF709
:105D40004DFBBBF1020F02D12046FFF753FD0720A8
:105D500082E6BBF1000F3FF479AE4FF0020B96E7FD
:105D600008B5804719F0D4FA024B1868BFF35B8F6F
:105D7000704700BF1C00002008B5FFF7F5FFFFF7D4
:105D8000EFFF08B58047FFF7F7FF0000024B1868E8
:105D9000BFF35B8F704700BF1400002008B5FFF70A
:105DA000F5FFFFF7EEFF012838BF012010B50446CC
:105DB00020461AF0BDF830B918F01AFA08B919F0EF
:105DC000A7FA8047F4E710BD08B5FFF7D5FF00003C
:105DD00010B5034B03600446FFF734FC204610BDAA
:105DE000CC81020810B50446FFF7F2FF20460C21D3
:105DF000FFF77CFC204610BDF7B5089F974205468B
:105E00000E4614460AD0A86802680897156A3146FB
:105E10002246AC4603B0BDE8F04060471946019306
:105E200000F058F8019B0028EDD0062003B0F0BD2B
:105E30002DE9F14F0D461946DDE90A4BDDE90CA6C7
:105E400081461746984600F045F890B1002D346021
:105E5000377109DB61198A450CBF06210121B17137
:105E6000002001B0BDE8F08F0235F9D10123B371F4
:105E7000F6E7544506D15946484600F02BF808B1DC
:105E80007771EDE7D9F808000368CDE90CA6CDE9F4
:105E90000A4BDC693A4643462946A44601B0BDE8B0
:105EA000F04F60472DE9F04107460C4615461E4667
:105EB000FFF7FBFB48B9B86803689F692A46334679
:105EC0002146BC46BDE8F0416047BDE8F08170471F
:105ED00000207047814208B50ED0406803782A2B15
:105EE0000CD049680B782A2B08BF0131FAF7C0F9AA
:105EF000B0FA80F0400908BD0120FCE70020FAE775
:105F000037B5051D0446284601910BF061FD0023BD
:105F1000C4E91D33C4E92033C4E9223384F87C305A
:105F2000054B0199236028461433636003B0BDE834
:105F300030400BF036BD00BF98A7020837B5051DED
:105F40000446284601910BF043FD0023C4E91F33AA
:105F5000C4E921336367A4F87830054B01992360C5
:105F600028461433636003B0BDE830400BF0CFBC6B
:105F700068A702082DE9F04FDFF844922DED028B5F
:105F8000D9F80040631C08EE100A83B0C9F800304D
:105F9000002C40F0ED80DFF82CB2794B794F7A4E2F
:105FA000DFF824A201221A70DBF80030774A9D68DE
:105FB000BC61C7E90024C7E90244C7E9044407F10A
:105FC0001C0000F0A7FEDBF80010704A3D624FF0A5
:105FD000FF384D68C7F800A0C7F82480C6E9002440
:105FE000C6E90244C6E90444B46106F11C0000F0AD
:105FF00091FEC6E90858DBF80010654D634ACB688E
:10600000C6F800A0C5E90024C5E90244C5E9044476
:10601000AC6105F11C00019300F07CFE019BC5F80A
:1060200000A0DFF8A8A1C5E9083839465046FFF7B7
:1060300085FF584A10460BF0CBFC564A564942F8A9
:10604000081CA2F108071431B9603146534E146799
:10605000C2E91E44C2E92044A2F8744042F8044C4C
:1060600010460BF054FC29463046FFF767FF2946DF
:106070004B48FFF763FF3269DBF80030C7F878A0C0
:1060800042F40052474F3261474A9D68C6F874A0F7
:10609000C7E90024C7E90244C7E90444BC6107F129
:1060A0001C0000F037FE414EDBF800103E4ADFF8DE
:1060B00020A1C7F800A0C7E9085806F11C004D68E8
:1060C000B461C6E90024C6E90244C6E9044400F00C
:1060D00021FEDBF80010344AD1F80CB0C6F800A05D
:1060E000C6E90858324DC5E90024C5E90244C5E9AE
:1060F0000444AC6105F11C0000F00CFEC5E908B8D1
:10610000DFF8D0B0DFF8D080C5F800A03946584697
:10611000FFF7F6FE40460BF05BFC264B88F8784014
:10612000A8F10807C8E91C44C8E91F44C8E921448C
:1061300048F8083C48F8044C14331F4CBB60314607
:1061400040460BF02EFC29462046FFF7D9FE1B489F
:106150002946FFF7D5FE2369C8F870B043F4005311
:106160002361D9F80030C4F874B00133C9F80030A5
:1061700018EE100A03B0BDEC028BBDE8F08F00BF33
:1061800018000020940600204406002080A8020881
:106190006C0600203C0700202CA10208C407002048
:1061A000500800200C070020C0A80208BC060020F0
:1061B000E40600205CA10208FC0900208C0A0020F3
:1061C000B01B0020A4000020689F0208DC0800200B
:1061D000A89F02081C0B0020700900200D4A1368BC
:1061E000591E022B10B50446116011D10A4811F056
:1061F00043F90A4811F040F9094811F03DF90948FE
:1062000011F0D0F9084811F0CDF9084811F0CAF999
:10621000204610BDB01B0020DC080020C407002071
:10622000500800201C0B0020FC0900208C0A0020D4
:1062300070474268511E012A416002D103685B68C1
:1062400018477047044A0B681268036093421EBFE8
:106250001A6801321A607047B00B00200160704765
:1062600002490348002218F0FFBA00BF0582020865
:10627000B80B002010B5034C23680BB9FFF7F0FFF3
:10628000206810BDB80B0020004870470582020846
:1062900038B5436804465BB10025D4E90132AA420F
:1062A00006D953F8250008B1FFF7C3FF0135F4E71D
:1062B000606808B117F0A6FEE3685BB10025D4E979
:1062C0000223AA4206D953F8250008B1FFF7B1FF0F
:1062D0000135F4E7E06808B117F094FE23691BB9B3
:1062E000206958B9204638BD00252369585908B19E
:1062F00017F088FE0435182DF7D1F1E717F082FE6C
:10630000F0E703685A1E012B10B50446026006D15F
:10631000FFF7BEFF2046BDE8104017F071BE10BD6C
:10632000054B10B51B6804460068984201D0FFF782
:10633000E8FF204610BD00BFB00B00200A4A38B568
:106340000B680D4611688B4218BF1A680446006836
:106350001CBF01321A60814201D0FFF7D2FF2B68C7
:106360002360204638BD00BFB00B0020036823B96E
:10637000034A1368013313600360006801387047F3
:10638000B40B00202DE9F84F044616460846002AB3
:1063900000F0AD80FFF7EAFFA368013B9842054695
:1063A00041D900F104086FF06043984534BF4FEACB
:1063B00088074FF0FF373846D4F804A017F020FFC5
:1063C0008346A0680023984269D1C0F104022A44A0
:1063D0009200804538BF002200210BEB800019F0AD
:1063E00029FE3846D4F80C9017F00AFF0746A0683B
:1063F000002398425AD1C0F104022A4492008045F9
:1064000038BF0022002107EB800019F013FEC4E919
:1064100001B8E760BAF1000F4FD1B9F1000F02D017
:10642000484617F0EFFD7368D4F8049001337360A9
:1064300059F825300BB32F490868D0B1FFF796FF04
:1064400085423ED14868D4F804A0FFF78FFF5AF880
:10645000203007466BB14968304608F037F843688A
:106460000133804643605AF82700FFF7E2FE4AF8FE
:10647000278059F82500FFF7DCFE49F82560002544
:106480002E46A368AB4232D9E36853F8250020B109
:10649000FFF7CFFEE36843F825600135F1E7626856
:1064A00052F823204BF8232001338CE7E26852F89E
:1064B000232047F8232001339BE7504617F0A2FD25
:1064C000ABE74868FFF752FF85420ED10868D4F861
:1064D00004A0FFF74BFF5AF820300746002BC8D026
:1064E0000968304602F0FCFEB9E70831A4E7BDE8D0
:1064F000F88F00BF248202082DE9F041214F3B783C
:10650000BFF35B8FDB0706460C46154606D43846BC
:1065100017F05EFE10B1384617F066FE1A4908689B
:10652000F0B1FFF723FFA84248680DD1FFF71EFF27
:106530000346F16851F82520AAB104B32368204628
:106540005B68BDE8F0411847FFF710FFA84205D18E
:106550000868FFF70BFF2B460546EAE70831DEE740
:106560004FF0FF33E5E76268501C6060581C18BFAD
:10657000023241F825401CBF626041F82340BDE86B
:10658000F08100BFAC0B00202482020810B5084C3B
:106590002378BFF35B8FDB0708D4204617F018FE83
:1065A00020B12046BDE8104017F01EBE10BD00BF50
:1065B000C00B00202DE9F04F30238360C24B0160F7
:1065C00087B00646C0220021184619F033FDBF4BA4
:1065D0007060C0221846002119F02CFDBC4CBD4D46
:1065E000F06014220021201D19F024FD3461256083
:1065F000FFF74AFEB84C03882B8000220123114686
:10660000204604F067FB22463046B449B44CDFF81C
:10661000C4A3DFF8C4B3B34DDFF8C093DFF8C08381
:10662000FFF7B0FEB04A0121104618F08DF9304650
:10663000AD4AAE49FFF7A6FEAD4AAE4B1360012747
:106640000023C2E90233C2E90533C2E907331374F8
:10665000938482F8643057601146A74A67602260CD
:10666000A1602046194600F00FFF22463046A3499C
:10667000A34CFFF787FEA34AA34957601160304639
:10668000A249FFF77FFEA24AA24957601160304637
:10669000A149FFF777FEA14A67602260FFF7EAFD94
:1066A0002246A0609E499F4C3046FFF76BFE9E4AF3
:1066B000CAF8002000239D4A676019462260C4F88A
:1066C00008A01A462046CAE90233CAE90533CAE9D6
:1066D0000733CAE90933CAE90B33AAF810308AF83C
:1066E0001230CAF834308AF84330CAF8047000F027
:1066F0006FFB224630468E498E4CFFF743FE8E4A92
:10670000CBF8002000238D4A676019462260C4F848
:1067100008B01A462046CBE90233CBE90533CBE972
:106720000733CBE90933CBE90B33ABF810308BF8E7
:106730001230CBF834308BF84330CBF8047000F0D3
:1067400003FB224630467E497E4CFFF71BFE7E4A05
:106750007E495760116030467D49FFF713FE7D4A40
:106760007D495760116030467C49FFF70BFE0023DE
:106770007B4A6F60C5E90233C5E90433C5E90633D6
:10678000C5E90833C5E90A33C5E90C33C5E90E3359
:10679000C5E91033C5E91233C5E91433C5E9163329
:1067A000C5E91833C5E91A33C5E91C33C5E91E33F9
:1067B0002A602946C5E920333A46C5E92233C5E9AE
:1067C0002433C5E92633C5E92833C5E92A33C5E9A9
:1067D0002C33C5E92E33C5F8C03085F8C4302046C7
:1067E0000BF08AFD224630465E495F4CFFF7CAFD3A
:1067F0005E4A5F495760116030465E49FFF7C2FD4F
:106800005D4A5E495760116030465D49FFF7BAFD49
:106810005C4A3946104605F015F83046594A5A493F
:10682000FFF7B0FD594A3946104604F03FFA3046AA
:10683000564A5749FFF7A6FD564A3946104618F002
:1068400093F83046534A5449FFF79CFD534B544A42
:106850001A601A465F600023C2E90233C2E90533B9
:10686000C2E9073313745362936282F824311146EC
:106870004C4A67602260A1602046194600F06CFE19
:10688000224630464849494CFFF77CFD484A494971
:106890005760116030464849FFF774FD474A484940
:1068A0005760116030464749FFF76CFD464A676004
:1068B0002260FFF7DFFC2246A0604449444C30468A
:1068C000FFF760FD8EE000BF6819002078180020F7
:1068D00060180020501100205C110020281B0020AF
:1068E000E40B0020580E002038190020781C0020EE
:1068F000C80C00202C830208809102085C1B002039
:1069000050190020281A00201CA20208FC1B00209D
:10691000381A002058A20208F81B002064910208CF
:10692000501B0020880C0020C4820208D891020865
:106930006C1B0020940C0020B4820208A491020871
:10694000681B00204C0C00202C0C00202892020810
:10695000641B00203C0C002040920208601B0020B9
:1069600088A20208F41B0020F00B0020FC0B002082
:1069700058920208581B00200C0C002088A3020823
:10698000F01B0020C40B0020541B00207C130020AF
:106990002C1B0020441900207C1C0020300D0020FE
:1069A0003C830208589C02089C1B00205C190020B4
:1069B000301A002014AA02085C1C0020401A002093
:1069C00050AA0208581C00203C9C0208901B002082
:1069D000A00C0020E80F00202C10002070100020D8
:1069E000E01000208F4AC9F8002000238E4A67601B
:1069F00019462260C4F808901A462046C9E90233B5
:106A0000C9E90533C9E90733C9E90933C9E90B33D2
:106A1000C9E90D3389F81030C9F83C3089F86C3079
:106A2000C9F8047000F094FA224630467F49804C41
:106A3000FFF7A8FC7F4AC8F8002000237E4A676061
:106A400019462260C4F808801A462046C8E9023375
:106A5000C8E90533C8E90733C8E90933C8E90B3386
:106A6000C8E90D3388F81030C8F83C3088F86C302D
:106A7000C8F8047000F024FA224630466F49704C82
:106A8000FFF780FC6F4A70495760116030466F49CC
:106A9000FFF778FC6E4A6F495760116030466E49C7
:106AA000FFF770FC00236D4A6760C4E90233C4E954
:106AB0000433C4E90633C4E90833C4E90A33C4E93A
:106AC0000C33C4E90E33C4E91033C4E91233C4E90A
:106AD0001433C4E91633C4E91833C4E91A33C4E9DA
:106AE0001C33C4E91E332260C4E92033C4E92233D5
:106AF000C4E92433C4E92633C4E92833C4E92A337A
:106B0000C4E92C33C4E92E33C4F8C03084F8C4304F
:106B1000534B3A462146184611F066FF504B5149F7
:106B20001A463046FFF72EFC4F4A504B5760136011
:106B300030464F49FFF726FC4E4A4F4B13605760D3
:106B400030464E49FFF71EFC4D4A3946104608F0C4
:106B5000B1FD30464A4A4B49FFF714FC4A4A4B4BB9
:106B60005760136030464A49FFF70CFC494A4A4BCC
:106B70005760136030464949FFF704FC484A494BC7
:106B80005760136030464849FFF7FCFB474A484BC3
:106B90005760136030464749FFF7F4FB4649474BBF
:106BA000CDF808B0CDE9031930466946CDE9003A81
:106BB000CDF8148001F0ECFA4148F768FFF7D6FBF6
:106BC0003E4B47F820303F48F768FFF7CFFB47F8C8
:106BD00020A03D48F768FFF7C9FB47F820B03B48C5
:106BE000F768FFF7C3FB47F820503948F568FFF70F
:106BF000BDFB314945F820100C48F568FFF7B6FB9E
:106C000045F820900D48F568FFF7B0FB45F8208067
:106C10001448F568FFF7AAFB45F82040304607B056
:106C2000BDE8F08FE4820208B09C0208AC1B002093
:106C3000AC0C0020D48202087C9C0208A81B002017
:106C4000200F0020340C0020009D0208A41B00200F
:106C5000440C0020189D0208A01B002080AA0208F6
:106C6000600C0020541C0020040C0020309D020801
:106C7000981B0020140C002080AB0208501C002040
:106C8000D40B0020941B00201C0C00207C860208E2
:106C9000541A0020240C0020248602084C1A0020DC
:106CA000B80C002050860208501A0020C00C0020AA
:106CB000F8850208481A0020300D0020C80C00207A
:106CC0005C1B00206C1B0020681B0020F41B0020B4
:106CD0009C1B002010B5074C02212046FFF76AFCE0
:106CE000054B06481C60064B21461C60BDE8104061
:106CF000FFF7B4BA740C0020B00B00205C18002021
:106D0000BC0B0020024B1B680BB9FFF7E3BF7047B9
:106D1000B00B002038B5002303600446084DFFF790
:106D2000F1FF084A2B6812682360934206D0FFF7F0
:106D30002DFC2B6823601A6801321A60204638BD8A
:106D4000BC0B0020B00B002038B584680546ACB9F8
:106D50004420FFF728F81A4B0482C0E90034C0E948
:106D60000244C0E90544C0E90744C0E90944C0E958
:106D70000B448474446380F84340A860AB681149B5
:106D80002E225A74AB682C229A74AA680023C2E996
:106D90000513C2E90713C2E9091391600A49D360D8
:106DA00008681063D362AA685063084A1068AA682A
:106DB000C15C1A4401330B2B82F83810F7D138BD6F
:106DC000B482020894C4020820B2020828000020FD
:106DD00038B584680546ACB94420FEF7E4FF1A4B89
:106DE0000482C0E90034C0E90244C0E90544C0E9B6
:106DF0000744C0E90944C0E90B448474446380F843
:106E00004340A860AB6811492E225A74AB682C220B
:106E10009A74AA680023C2E90513C2E90713C2E9FC
:106E2000091391600A49D36008681063D362AA68A5
:106E30005063084A1068AA68C15C1A4401330B2BDE
:106E400082F83810F7D138BDC482020894C4020811
:106E500020B2020828000020064B10B5044603604B
:106E6000806810B103685B6898472046FFF7E0F937
:106E7000204610BDA491020810B50446FFF7ECFFB0
:106E8000204617F0BDF8204610BD0000064B10B597
:106E900004460360806810B103685B689847204629
:106EA000FFF7C6F9204610BDD891020810B5044678
:106EB000FFF7ECFF204617F0A3F8204610BD0000B6
:106EC00038B584680546B4B97020FEF76CFFC0E998
:106ED0000244C0E90544C0E90744C0E90944C0E9E7
:106EE0000B44C0E90D44154B446003600474C46353
:106EF00080F86C40A860AB682E212C22C3E90512F3
:106F00000F49104A9A600022C3E90712C3E9091227
:106F1000C3E90B12DA605A630B4A10689863AB68D6
:106F2000D8630A4BAA681B684032591E0A3311F80D
:106F3000010F42F8040B9942F9D138BDD4820208FE
:106F40009CC8020894C4020820B20208280000204D
:106F500038B584680546B4B97020FEF724FFC0E94F
:106F60000244C0E90544C0E90744C0E90944C0E956
:106F70000B44C0E90D44154B446003600474C463C2
:106F800080F86C40A860AB682E212C22C3E9051262
:106F90000F49104A9A600022C3E90712C3E9091297
:106FA000C3E90B12DA605A630B4A10689863AB6846
:106FB000D8630A4BAA681B684032591E0A3311F87D
:106FC000010F42F8040B9942F9D138BDE48202085E
:106FD0009CC8020894C4020820B2020828000020BD
:106FE000064B10B504460360806810B103685B6807
:106FF00098472046FFF71CF9204610BD7C9C0208EC
:1070000010B50446FFF7ECFF204616F0F9FF2046C6
:1070100010BD0000064B10B504460360806810B137
:1070200003685B6898472046FFF702F9204610BDC9
:10703000B09C020810B50446FFF7ECFF204616F09E
:10704000DFFF204610BD00000D4B10B5036090F827
:10705000433004467BB1806808B116F0D3FF606905
:1070600008B116F0CFFFE06908B116F0CBFF606AF7
:1070700008B116F0C7FF2046FFF7DAF8204610BD2A
:10708000B482020810B50446FFF7DEFF204616F072
:10709000B7FF204610BD00000D4B10B5036090F8FF
:1070A000433004467BB1806808B116F0ABFF6069DD
:1070B00008B116F0A7FFE06908B116F0A3FF606AF7
:1070C00008B116F09FFF2046FFF7B2F8204610BD2A
:1070D000C482020810B50446FFF7DEFF204616F012
:1070E0008FFF204610BD00000D4B10B5036090F8D7
:1070F0006C3004467BB1806808B116F083FFE0690C
:1071000008B116F07FFF606A08B116F07BFFE06AF5
:1071100008B116F077FF2046FFF78AF8204610BD29
:10712000D482020810B50446FFF7DEFF204616F0B1
:1071300067FF204610BD00000D4B10B5036090F8AE
:107140006C3004467BB1806808B116F05BFFE069E3
:1071500008B116F057FF606A08B116F053FFE06AF5
:1071600008B116F04FFF2046FFF762F8204610BD29
:10717000E482020810B50446FFF7DEFF204616F051
:107180003FFF204610BD000038B584680546ACB905
:107190004420FEF708FE1A4B0482C0E90034C0E91F
:1071A0000244C0E90544C0E90744C0E90944C0E914
:1071B0000B448474446380F84340A860AB68114971
:1071C0002E225A74AB682C229A74AA680023C2E952
:1071D0000513C2E90713C2E9091391600A49D36094
:1071E00008681063D362AA685063084A1068AA68E6
:1071F000C15C1A4401330B2B82F83810F7D138BD2B
:10720000B482020894C4020820B2020828000020B8
:1072100038B584680546ACB94420FEF7C4FD1A4B66
:107220000482C0E90034C0E90244C0E90544C0E971
:107230000744C0E90944C0E90B448474446380F8FE
:107240004340A860AB6811492E225A74AB682C22C7
:107250009A74AA680023C2E90513C2E90713C2E9B8
:10726000091391600A49D36008681063D362AA6861
:107270005063084A1068AA68C15C1A4401330B2B9A
:1072800082F83810F7D138BDC482020894C40208CD
:1072900020B2020828000020064B10B50446036007
:1072A000806810B103685B6898472046FEF7C0FF0E
:1072B000204610BDA8A2020810B50446FFF7ECFF57
:1072C000204616F09DFE204610BD0000064B10B56E
:1072D00004460360806810B103685B6898472046E5
:1072E000FEF7A6FF204610BDDCA2020810B504463A
:1072F000FFF7ECFF204616F083FE204610BD00008D
:1073000038B584680546B4B97020FEF74CFDC0E975
:107310000244C0E90544C0E90744C0E90944C0E9A2
:107320000B44C0E90D44154B446003600474C4630E
:1073300080F86C40A860AB682E212C22C3E90512AE
:107340000F49104A9A600022C3E90712C3E90912E3
:10735000C3E90B12DA605A630B4A10689863AB6892
:10736000D8630A4BAA681B684032591E0A3311F8C9
:10737000010F42F8040B9942F9D138BDD4820208BA
:107380009CC8020894C4020820B202082800002009
:1073900038B584680546B4B97020FEF704FDC0E92D
:1073A0000244C0E90544C0E90744C0E90944C0E912
:1073B0000B44C0E90D44154B446003600474C4637E
:1073C00080F86C40A860AB682E212C22C3E905121E
:1073D0000F49104A9A600022C3E90712C3E9091253
:1073E000C3E90B12DA605A630B4A10689863AB6802
:1073F000D8630A4BAA681B684032591E0A3311F839
:10740000010F42F8040B9942F9D138BDE482020819
:107410009CC8020894C4020820B202082800002078
:10742000064B10B504460360806810B103685B68C2
:1074300098472046FEF7FCFE204610BDA0AA020891
:1074400010B50446FFF7ECFF204616F0D9FD2046A4
:1074500010BD0000064B10B504460360806810B1F3
:1074600003685B6898472046FEF7E2FE204610BDA1
:10747000D4AA020810B50446FFF7ECFF204616F028
:10748000BFFD204610BD000038B58468054684B9AC
:107490006820FEF788FCC0E90244C0E90544C0E961
:1074A00007441A4B446003600474848480F8644089
:1074B000A860AA68164B93602E21002382F824103E
:1074C000D3601374AA682C2182F82510114A106821
:1074D000AA68C15C1A440133242B82F82610F7D124
:1074E0000D4B18680023AA68C15C1A4401331A2B9B
:1074F00082F84A10F7D1AB68084A5A6104229A61AF
:10750000074ADA6105221A6238BD00BF2C830208DF
:1075100094C402082400002020000020EC8202080D
:10752000F1820208064B10B504460360806810B172
:1075300003685B6898472046FEF77AFE204610BD38
:107540008091020810B50446FFF7ECFF204616F0C4
:1075500057FD204610BD000038B58468054694B933
:107560004FF49470FEF71FFCC0E90244C0E90544E3
:10757000C0E90744C0E90944184B4460036004743F
:1075800080F82441A860AB68154A9A6000222E2139
:10759000DA601A742C22C3E90912124A126803F144
:1075A0002C00511E233211F8014F40F8044B914238
:1075B000F9D10D4A126803F1BC00511E193211F8BD
:1075C000014F40F8044B9142F9D1084A5A61042214
:1075D0009A61074ADA6105221A6238BD3C830208C3
:1075E00094C402082400002020000020F882020831
:1075F0000C830208064B10B504460360806810B186
:1076000003685B6898472046FEF712FE204610BDCF
:10761000589C020810B50446FFF7ECFF204616F010
:10762000EFFC204610BD00000B4B10B5036090F836
:10763000643004465BB1806808B116F0E3FC606911
:1076400008B116F0DFFCE06908B116F0DBFC20465B
:10765000FEF7EEFD204610BD2C83020810B504464F
:10766000FFF7E2FF204616F0CBFC204610BD0000DD
:107670000B4B10B5036090F8243104465BB1806871
:1076800008B116F0BFFC606908B116F0BBFCE069F8
:1076900008B116F0B7FC2046FEF7CAFD204610BD23
:1076A0003C83020810B50446FFF7E2FF204616F0BF
:1076B000A7FC204610BD000038B58468054684B993
:1076C0006820FEF770FBC0E90244C0E90544C0E948
:1076D00007441A4B446003600474848480F8644057
:1076E000A860AA68164B93602E21002382F824100C
:1076F000D3601374AA682C2182F82510114A1068EF
:10770000AA68C15C1A440133242B82F82610F7D1F1
:107710000D4B18680023AA68C15C1A4401331A2B68
:1077200082F84A10F7D1AB68084A5A6104229A617C
:10773000074ADA6105221A6238BD00BF2C830208AD
:1077400094C402082400002020000020EC820208DB
:10775000F1820208064B10B504460360806810B140
:1077600003685B6898472046FEF762FD204610BD1F
:10777000F8A1020810B50446FFF7ECFF204616F00A
:107780003FFC204610BD000038B58468054694B91A
:107790004FF49470FEF707FBC0E90244C0E90544CA
:1077A000C0E90744C0E90944184B4460036004740D
:1077B00080F82441A860AB68154A9A6000222E2107
:1077C000DA601A742C22C3E90912124A126803F112
:1077D0002C00511E233211F8014F40F8044B914206
:1077E000F9D10D4A126803F1BC00511E193211F88B
:1077F000014F40F8044B9142F9D1084A5A610422E2
:107800009A61074ADA6105221A6238BD3C83020890
:1078100094C402082400002020000020F8820208FE
:107820000C830208064B10B504460360806810B153
:1078300003685B6898472046FEF7FAFC204610BDB7
:10784000F0A9020810B50446FFF7ECFF204616F039
:10785000D7FB204610BD009B03201A607047002014
:1078600070470020704704207047009B03201A6077
:107870007047009B03201A607047009B03201A602A
:107880007047F0B50546D0E90020801A65D092F91E
:1078900000401378002C03DB01322A601846F0BD4B
:1078A000C12B3BD9DF2B0FD8012856D0507800F0E0
:1078B000C004802C32D100EB8310A0F542508142ED
:1078C000EDD302322A60EAE7EF2B1AD8022844D916
:1078D000547804F0C000802820D1E02B01D19F2CE7
:1078E0001CD9907800F0C006802E17D1A40104EBBB
:1078F00003330344A3F5622080388142CFD303329F
:10790000E0E7F42B0AD8032827D9547804F0C00004
:10791000802803D1F02B04D18F2C06D84FF0FF30F4
:10792000BDE7F42B01D18F2CF8D8967806F0C00073
:107930008028F3D1D07800F0C007802FEED1240347
:1079400004EB834303EB86130344A3F17270A0F5A9
:1079500002508842A3D80432B4E76FF001009EE7DA
:10796000F0B50546D0E90020801A65D092F90040B4
:107970001378002C03DB01322A601846F0BDC12BBE
:107980003BD9DF2B0FD8012856D0507800F0C00427
:10799000802C32D100EB8310A0F542508142EDD310
:1079A00002322A60EAE7EF2B1AD8022844D9547829
:1079B00004F0C000802820D1E02B01D19F2C1CD9DD
:1079C000907800F0C006802E17D1A40104EB033399
:1079D0000344A3F5622080388142CFD30332E0E72D
:1079E000F42B0AD8032827D9547804F0C000802843
:1079F00003D1F02B04D18F2C06D84FF0FF30BDE718
:107A0000F42B01D18F2CF8D8967806F0C00080288E
:107A1000F3D1D07800F0C007802FEED1240304EB1F
:107A2000834303EB86130344A3F17270A0F5025065
:107A30008842A3D80432B4E76FF001009EE77F29A3
:107A400008D8D0E900329A4242D05A1C026019701C
:107A500001207047B1F5006F10D2D0E90032D21A80
:107A6000012A35D95A1C02608A09403A1A70036803
:107A700001F03F015A1C02608039E8E7B1F5803F10
:107A800011D2D0E90032D21A022A21D95A1C02603E
:107A90000A0B203A1A700268531C0360C1F3851365
:107AA000803B1370E3E7B1F5881F11D2D0E90032B3
:107AB000D21A032A0CD95A1C02608A0C103A1A7086
:107AC0000268531C0360C1F30533803B1370E2E787
:107AD000002070477F2910B508D8D0E900329A42BB
:107AE00047D05A1C02601970012010BDB1F5006F1B
:107AF0000FD2D0E90032D21A012A3AD98C091A469B
:107B0000403C02F8024B01F03F018039026059709D
:107B1000EAE7B1F5803F12D2D0E90032D21A022A48
:107B200027D90A0B203A1A70C1F38512803A01F066
:107B30003F015A708039DA1C02609970D4E7B1F5C0
:107B4000881F16D2D0E90032D21A032A11D98A0C22
:107B5000103A1A70C1F30532803A5A70C1F3851297
:107B6000803A01F03F019A7080391A1D0260D97085
:107B7000BAE70020B9E7B1F5803F10B5D0E900437E
:107B80000BD2A34222D0D30789B201D449BA89B219
:107B9000A31C03602180012010BD1B1B022B15D9E3
:107BA0008B0AC1F30901A3F52153A1F5105112F07D
:107BB00001029BB289B201D15BBA9BB223800AB9A0
:107BC00049BA89B2231D03606180E4E70020E3E73E
:107BD00073B51E46079B0093089B01931446A6426B
:107BE000254612D02168B1F5881F04F104040ED295
:107BF0006846FFF76FFF0028F1D10120069B009A2D
:107C00001D60099B1A6002B070BD0020F6E70220DB
:107C1000F4E7000030B585B0CDE90023099B02935D
:107C2000144D0A9B0393DDE90123009CA24215D069
:107C3000039A9A4212D029466846FFF791FE831CA8
:107C4000014609D0B0F5881F11D2012202A8FFF722
:107C500092FF0028E7D10094012000E00020089B5B
:107C6000009A1A600B9B029A1A6005B030BD022080
:107C7000F5E700BFFFFF10008B070CD5D0E90032FD
:107C8000D21A022A09D9064A1188927819809A7064
:107C9000036803330360012070470020704700BF72
:107CA000448302082DE9F0410E4604461946304649
:107CB000069D1746FFF7E0FF78B3D4E900329A42F9
:107CC0002ED01988A1F55840B0F5806F1DD2012D36
:107CD00028D0D21A022A23D95B88A3F55C42B2F5D8
:107CE000806F1FD2A3F15773A3F5773303EB812184
:107CF0004FF002088F4215D33046FFF7A0FE60B167
:107D0000236803EB48032360D7E7A1F55C43B3F591
:107D1000806F07D34FF00108ECE70120BDE8F08148
:107D20000020FBE70220F9E77FB5CDE90223099B9C
:107D300004930A9B059300230093074A04A902A811
:107D4000FFF7B0FF089B029A1A600B9B049A1A6017
:107D500007B05DF804FB00BFFFFF100070B50D46D3
:107D60000446194628461646FFF786FF70B1D4E947
:107D700000329A420CD019688E420BD32846FFF786
:107D80005EFE18B1236804332360F0E7012070BD64
:107D90000020FCE70220FAE71FB5CDE90023079B8E
:107DA0000293089B0393074A002302A96846FFF742
:107DB000D5FF069B009A1A60099B029A1A6005B0CB
:107DC0005DF804FBFFFF100038B54B0704460CD5E7
:107DD000D0E900535B1B022B07D904490322284634
:107DE00018F0F0F808B90335256038BD148402088E
:107DF00070B50C46194605461646FFF7E5FFD5E96E
:107E000000239A4212D0D4E900329A4201D10120D3
:107E100070BD31462846FFF734FD831CF7D08642FB
:107E200006D323681A1D22601860E8E70020EFE7F8
:107E30000220EDE71FB5CDE90023079B0293089BC5
:107E40000393074A002302A96846FFF7D1FF069B68
:107E5000009A1A60099B029A1A6005B05DF804FB4B
:107E6000FFFF100037B5CDE9000168469DF81810F6
:107E700014461D46FFF7A8FF002044B1A84204F1B4
:107E8000FF3404D829466846FFF7FBFCF5E7009865
:107E900003B030BD13B51446194600230093049A6D
:107EA000034B2046FFF7DEFF001B02B010BD00BFF2
:107EB000FFFF10002DE9F8430D461946044617460A
:107EC0001E46FFF781FFD4E90098C1451BD0D5E9D4
:107ED00000329A4217D039462046FFF7D2FC831C65
:107EE000014604D108980130C0B2BDE8F88387424A
:107EF0000BD332462846FFF73EFE0028E3D1C4E903
:107F000000980120F1E70020EFE70220EDE70000F4
:107F10007FB5CDE90223099B04930A9B05930023B7
:107F20000093074A012304A902A8FFF7C3FF089B97
:107F3000029A1A600B9B049A1A6007B05DF804FB62
:107F4000FFFF1000F7B5CDE900019DF8201068464D
:107F500016461C46FFF738FF00256F1CB7420ED2AD
:107F600021466846FFF78DFCA04202D9009803B075
:107F7000F0BDB0F5803F28BF3D460135EDE7F5D1B6
:107F80004FF6FF734FF6FE718C4294BF214619469F
:107F90006846FFF776FCE9E713B514461946002357
:107FA0000093049A034B2046FFF7CCFF001B02B05E
:107FB00010BD00BFFFFF100073B51D46079B009367
:107FC000089B01931446A54225D02188A1F558436A
:107FD000B3F5806F15D22B1B022B1CD96288A2F53A
:107FE0005C43B3F5806F1ED2A2F15772A2F57732CF
:107FF00002EB812102266846FFF76CFD40B90120A3
:108000000AE0A1F55C43B3F5806F0CD30126F2E7DB
:1080100004EB4604D7E70020069B009A1C60099BEE
:108020001A6002B070BD0220F6E7000037B5DDE946
:108030000745CDE900230F49DDE900329A4214D00B
:10804000A54207D10120069B009A1A60099B1C607B
:1080500003B030BD6846FFF783FC831CF2D0B0F557
:10806000881F04D244F8040BE6E70020EBE7022067
:10807000E9E700BFFFFF100037B5CDE90023069DFB
:1080800008491446002045B1B0F5881F05F1FF35B9
:1080900003D26846FFF764FCF5E70098001B03B0C5
:1080A00030BD00BFFFFF1000F7B5CDE90023089EEB
:1080B0000E4915460024671CBE420FD96846FFF7DB
:1080C0004FFCB0F5881F03D30098401B03B0F0BDF0
:1080D000B0F5803F28BF3C460134ECE7F4D14FF6C1
:1080E000FF716846FFF73CFCEEE700BFFFFF1000A2
:1080F00010B5034B03600446FEF79AF8204610BD06
:10810000F083020810B50446FFF7F2FF204615F091
:1081100077FF204610BD000010B5034B03600446F6
:10812000FEF786F8204610BD6C83020810B50446A1
:10813000FFF7F2FF204615F063FF204610BD000058
:1081400010B5034B03600446FEF772F8204610BDDD
:108150009883020810B50446FFF7F2FF204615F099
:108160004FFF204610BD000010B5034B03600446CE
:10817000FEF75EF8204610BDC483020810B5044621
:10818000FFF7F2FF204615F03BFF204610BD000030
:108190002DE9F04F89B00B6801934B68A94F02930A
:1081A0008B680393A84B3B600125019B7D600446CF
:1081B0000E46BB6000213846FFF77EFA7B68D4F894
:1081C0000480DFF818B3DFF818A32B447B609F4BC3
:1081D0001846FEF7CBF848F820709D4F9D4A7D6009
:1081E0003A60FEF747F87A68D4F80480B8602A4409
:1081F0007A609948FEF7BAF848F82070974F984A85
:10820000029B3A600022BB6011467D603846FEF753
:10821000FFFF7A68D4F804802A447A605846FEF753
:10822000A5F848F820708F4F8F4A039B3A600022D0
:10823000BB6011467D603846FEF7A6FF7A68D4F829
:1082400004802A447A605046FEF790F848F820707F
:10825000DFF89082854AD4F80490C8F800200227FD
:10826000C8F804708248FEF781F849F82080DFF8EA
:108270007882804AD4F80490C8F80020C8F80470C6
:108280007D48FEF773F849F82080DFF860827B4A6A
:10829000D4F80490C8F80020C8F804707848FEF7B5
:1082A00065F849F82080DFF84882294640460AF000
:1082B0003DF9D8F80420D4F8049072482A44C8F84C
:1082C0000420FEF753F849F82080F36804933369DB
:1082D000059373696C4E6D4A0693049BB36000214D
:1082E000756032603046FFF74FFA7268DFF804922B
:1082F000D4F804802A4472604846FEF737F848F8FC
:108300002060634E634A75603260FDF7B3FF7268A8
:10831000D4F80480B0602A4472605F48FEF726F803
:1083200048F820605D4E5E4A059B32600022B360D3
:10833000756011463046FFF72BF87268DFF8B88198
:10834000616807912A4472604046FEF70FF807996A
:10835000544A41F82060544E069B32600022B360BC
:10836000756011463046FEF7CBFF72686168079171
:108370002A4472604D4A1046FDF7F8FF079941F80C
:1083800020604B4E4B4931604B48616877600791E4
:10839000FDF7ECFF079941F82060484E48493160ED
:1083A0004848616877600791FDF7E0FF079941F859
:1083B0002060454E454931604548616877600791C6
:1083C000FDF7D4FF079941F82060424E2946304618
:1083D00010F024FC716865683F4801317160FDF759
:1083E000C5FF1A4B45F820601846E568FDF7BEFF4B
:1083F000019B45F820305846E568FDF7B7FF029B22
:1084000045F820305046E568FDF7B0FF039B45F87E
:1084100020304846E568FDF7A9FF049B45F8203069
:108420004046E568FDF7A2FF204A059B45F820304D
:108430001046E468FDF79AFF069B44F8203009B027
:10844000BDE8F08F781A0020F8A10208001C002077
:10845000F01A0020DCA10208E41B0020C01A002052
:10846000DCA20208CC1A0020A8A2020858A3020825
:10847000081C002070A30208041C00209CA3020812
:10848000EC1B0020E81B0020841A0020F0A9020841
:10849000FC1A002094A90208441C0020D81A0020CD
:1084A000D4AA0208A0AA0208E41A00206C1C00202A
:1084B000A81A002050AB0208681C0020B81A00203F
:1084C00068AB0208641C0020981A002094AB0208D4
:1084D0004C1C0020681A0020481C0020101C0020A2
:1084E0000C1C0020A01A0020B01A0020901A0020B6
:1084F000581A0020601C0020701C002001F04EBDA6
:1085000002F0F8B8F8B50B6853F80C5C0746681C25
:108510000E4615F075FE0023044601462A463046F5
:1085200001F072FC002363553C602846F8BDF8B5A5
:108530000B6853F80C5C6FF060426B1C934207466B
:1085400034BF98004FF0FF300E4615F059FE00235F
:10855000044601462A46304602F010F8002344F84B
:1085600025303C602846F8BD13B5049CCDE90034A5
:1085700013460A46C1684FF0000005F04AFD02B0FC
:1085800010BD30B58BB00D460AA901E90C00792366
:108590000693129B0593119B0493109B03930EAAC1
:1085A000044692E8030001AB83E80300099B0093B3
:1085B0002046089BAA684FF0000105F0D2FE204635
:1085C0000BB030BD30B58BB00D460AA901E90C00E7
:1085D0006D230693129B0593119B0493109B0393A9
:1085E0000EAA044692E8030001AB83E80300099B4E
:1085F00000932046089BAA684FF0000105F0B1FEE9
:1086000020460BB030BD30B58BB00D460AA901E94C
:108610000C0077230693129B0593119B0493109BE8
:1086200003930EAA044692E8030001AB83E803001B
:10863000099B00932046089BAA684FF0000105F0B3
:1086400090FE20460BB030BD30B58BB00D460AA968
:1086500001E90C0064230693129B0593119B04937C
:10866000109B03930EAA044692E8030001AB83E833
:108670000300099B00932046089BAA684FF0000165
:1086800005F06FFE20460BB030BD30B58BB00D4607
:108690000AA901E90C0074230693129B0593119B10
:1086A0000493109B03930EAA044692E8030001ABC7
:1086B00083E80300099B00932046089BAA684FF0BB
:1086C000000105F04EFE20460BB030BD81684FF032
:1086D000000005F040BEF0B591B00AAC84E80C0093
:1086E000002307930D930EAB06930DAB0593199BD7
:1086F00004939DF86030039316AA0F46054692E84E
:10870000030001AB83E803000B9B009308AE0A9BB8
:10871000BA684FF00001304606F015FA96E80300FB
:108720000D9B84E803005BB9DDE90E011B9BC3E9E7
:10873000000194E8030085E80300284611B0F0BD6D
:108740001A9A1360F5E710B588B00DF1200C0CE90A
:108750000C00002304939DF8303003930B9B02938D
:108760009DF828300193079B009313468A684FF0C9
:108770000001044606F0FEF8204608B010BD0A4687
:1087800001694FF0000005F0DEBD07B509680092F1
:1087900051F80C3C0A4601694FF0000005F0A7FDB6
:1087A00003B05DF804FB13B5049CCDE90034134617
:1087B0000A46C1684FF0000005F036FC02B010BD5B
:1087C00030B58BB00D460AA901E90C007923069358
:1087D000129B0593119B0493109B03930EAA0446CE
:1087E00092E8030001AB83E80300099B0093204655
:1087F000089BAA684FF0000105F00DFE20460BB063
:1088000030BD30B58BB00D460AA901E90C006D23CF
:108810000693129B0593119B0493109B03930EAA3E
:10882000044692E8030001AB83E80300099B009330
:108830002046089BAA684FF0000105F0ECFD204699
:108840000BB030BD30B58BB00D460AA901E90C0064
:1088500077230693129B0593119B0493109B03931C
:108860000EAA044692E8030001AB83E80300099BCB
:1088700000932046089BAA684FF0000105F0CBFD4D
:1088800020460BB030BD30B58BB00D460AA901E9CA
:108890000C0064230693129B0593119B0493109B79
:1088A00003930EAA044692E8030001AB83E8030099
:1088B000099B00932046089BAA684FF0000105F031
:1088C000AAFD20460BB030BD30B58BB00D460AA9CD
:1088D00001E90C0074230693129B0593119B0493EA
:1088E000109B03930EAA044692E8030001AB83E8B1
:1088F0000300099B00932046089BAA684FF00001E3
:1089000005F089FD20460BB030BD81684FF00000B6
:1089100005F024BDF0B591B00AAC84E80C0000234A
:1089200007930D930EAB06930DAB0593199B049320
:108930009DF86030039316AA0F46054692E803009F
:1089400001AB83E803000B9B009308AE0A9BBA6857
:108950004FF00001304606F092FA96E803000D9BB6
:1089600084E803005BB9DDE90E011B9BC3E900014C
:1089700094E8030085E80300284611B0F0BD1A9A78
:108980001360F5E710B588B00DF1200C0CE90C0070
:10899000002304930C9B03930B9B02939DF82830B8
:1089A0000193079B009313468A684FF00001044629
:1089B00006F07CF9204608B010BD0A4601694FF068
:1089C000000005F0C4BC07B50968009251F80C3CE2
:1089D0000A4601694FF0000005F09FFC03B05DF806
:1089E00004FB10B50446006843685A1E012B426020
:1089F00002D103685B689847204610BD10B5074B4D
:108A00000360036900220446DA600C30FFF7E9FFD7
:108A10002046FEF79FFE204610BD00BFF08C0208E6
:108A200010B50446FFF7EAFF204615F0E9FA2046A4
:108A300010BD000010B5084B036003690022044616
:108A4000DA609A611A629A620C30FFF7CAFF204618
:108A5000FEF722FC204610BD1C8E020810B504460D
:108A6000FFF7E8FF204615F0CBFA204610BD0000C6
:108A700010B5084B0360036900220446DA609A616E
:108A80001A629A620C30FFF7ACFF2046FEF71EFC1C
:108A9000204610BDE88D020810B50446FFF7E8FF38
:108AA000204615F0ADFA204610BD000010B5054B6C
:108AB000044640F8103BFFF794FF204609F0BEF94A
:108AC000204610BDB88C020810B50446FFF7EEFF33
:108AD000204615F095FA204610BD000010B5074B52
:108AE0000360036900220446DA600C30FFF779FF67
:108AF0002046FEF797FE204610BD00BF148D0208E9
:108B000010B50446FFF7EAFF204615F079FA204633
:108B100010BD000010B5084B036003690022044635
:108B2000DA601A629A621A630C30FFF75AFF204625
:108B3000FEF776FC204610BD848E020810B5044670
:108B4000FFF7E8FF204615F05BFA204610BD000055
:108B500010B5084B0360036900220446DA601A620C
:108B60009A621A630C30FFF73CFF2046FEF772FC56
:108B7000204610BD508E020810B50446FFF7E8FFEE
:108B8000204615F03DFA204610BD000010B5054BFB
:108B9000044640F8103BFFF724FF20460FF09EFCF0
:108BA000204610BDD48C020810B50446FFF7EEFF36
:108BB000204615F025FA204610BD000010B5054BE3
:108BC000044640F80C3BFFF70CFF204609F04EF935
:108BD000204610BD808C020810B50446FFF7EEFF5A
:108BE000204615F00DFA204610BD000010B5054BCB
:108BF000044640F8083BFFF7F4FE204609F098F8D9
:108C0000204610BD888D020810B50446FFF7EEFF20
:108C1000204615F0F5F9204610BD000010B5054BB3
:108C2000044640F8083BFFF7DCFE204609F08AF8CE
:108C3000204610BDB88D020810B50446FFF7EEFFC0
:108C4000204615F0DDF9204610BD000010B5054B9B
:108C5000044640F80C3BFFF7C4FE20460FF056FCDC
:108C6000204610BD9C8C020810B50446FFF7EEFFAD
:108C7000204615F0C5F9204610BD000010B5054B83
:108C8000044640F8083BFFF7ACFE20460FF0A0FB7F
:108C9000204610BDA08D020810B50446FFF7EEFF78
:108CA000204615F0ADF9204610BD000010B5054B6B
:108CB000044640F8083BFFF794FE20460FF092FB75
:108CC000204610BDD08D020810B50446FFF7EEFF18
:108CD000204615F095F9204610BD000010B5054B53
:108CE000044640F8083BFFF77CFE204609F05CF89C
:108CF000204610BD388D020810B50446FFF7EEFF80
:108D0000204615F07DF9204610BD000010B5054B3A
:108D1000044640F8083BFFF764FE20460FF094FB42
:108D2000204610BD608D020810B50446FFF7EEFF27
:108D3000204615F065F9204610BD836910B504463C
:108D400003B19847204610BD37B5084614460D4676
:108D500009F0B6FA84F82400284609F0B4FA002392
:108D6000A3606361E361012384F8643084F8250023
:108D7000294601A809F0AAFA01A904F10800FFF7A1
:108D8000C1FBE06001A801F009F9294601A809F03A
:108D9000A4FA01A904F11400FFF7B4FBA06101A833
:108DA00001F0FCF8294601A809F09EFA01A904F196
:108DB0001C00FFF7A7FB206201A801F0EFF803B049
:108DC00030BD37B5084614460D460FF0F1FD606220
:108DD00028460FF0F0FD0023A3606361E3610123E7
:108DE00084F82431A062294601A80FF0E7FD01A90B
:108DF00004F10800FFF786FBE06001A801F0CEF85F
:108E0000294601A80FF0E1FD01A904F11400FFF7C4
:108E10008EFBA06101A801F06DFC294601A80FF0AE
:108E2000DBFD01A904F11C00FFF781FB206201A812
:108E300001F060FC03B030BD10B4084611461A467C
:108E4000DDE9013401945DF8044B09F091BB10B4E5
:108E5000084611461A46DDE9013401945DF8044BD9
:108E60000FF0FEBE37B5084614460D4609F079F9F5
:108E70006074284609F078F9A074284609F093F93F
:108E80000023A3606361E3616362012384F84330DC
:108E9000E062294601A809F06AF901A904F1080075
:108EA000FFF730FBE06001A801F078F8294601A83F
:108EB00009F064F901A904F11400FFF723FBA06194
:108EC00001A801F06BF8294601A809F05EF901A993
:108ED00004F11C00FFF716FB206201A801F05EF808
:108EE000294601A809F058F901A904F12400FFF767
:108EF00009FBA06201A801F051F8284609F056F9D3
:108F00002063284609F057F9606303B030BD37B5D8
:108F1000084614460D4609F0F5F86074284609F035
:108F2000F4F8A074284609F00FF90023A3606361E8
:108F3000E3616362012384F84330E062294601A8BB
:108F400009F0E6F801A904F10800FFF7DBFAE06098
:108F500001A801F023F8294601A809F0E0F801A9C9
:108F600004F11400FFF7CEFAA06101A801F016F891
:108F7000294601A809F0DAF801A904F11C00FFF75D
:108F8000C1FA206201A801F009F8294601A809F0F8
:108F9000D4F801A904F12400FFF7B4FAA06201A8F3
:108FA00000F0FCFF284609F0D2F82063284609F0BB
:108FB000D3F8606303B030BD37B5084614460D469C
:108FC0000FF047FC606128460FF046FCA061284680
:108FD0000FF061FC0023A360E3616362E36201239D
:108FE00084F86C306063294601A80FF038FC01A9B1
:108FF00004F10800FFF786FAE06001A800F0CEFF58
:10900000294601A80FF032FC01A904F11C00FFF76A
:109010008EFA206201A801F06DFB294601A80FF02D
:109020002CFC01A904F12400FFF781FAA06201A839
:1090300001F060FB294601A80FF026FC01A904F10C
:109040002C00FFF774FA206301A801F053FB2846B7
:109050000FF024FCA06328460FF025FCE06303B06A
:1090600030BD37B5084614460D460FF0C3FB6061AE
:1090700028460FF0C2FBA06128460FF0DDFB00235D
:10908000A360E3616362E362012384F86C30606390
:10909000294601A80FF0B4FB01A904F10800FFF76D
:1090A00031FAE06001A800F079FF294601A80FF02D
:1090B000AEFB01A904F11C00FFF739FA206201A8F8
:1090C00001F018FB294601A80FF0A8FB01A904F143
:1090D0002400FFF72CFAA06201A801F00BFB29463F
:1090E00001A80FF0A2FB01A904F12C00FFF71FFA61
:1090F000206301A801F0FEFA28460FF0A0FBA06350
:1091000028460FF0A1FBE06303B030BD13B50C4659
:1091100001A811461A466B4601F09CF9049A01A970
:10912000204609F013FA044601A800F037FF204654
:1091300002B010BD13B50C4601A811461A466B4685
:1091400001F088F9049A01A920460FF077FD044642
:1091500001A800F023FF204602B010BD08461146CA
:1091600009F003BA084611460FF077BD084609F02A
:109170004EB908460FF0C3BC82B0F0B587B00546C3
:109180009DF850700D93742F16461398DDE9112148
:109190000FAC0DAB1ED00ED8642F2DD0CDE903102F
:1091A000029294E803008DE8030031460CCB284678
:1091B00009F084F91AE0772F2BD0CDE90310029241
:1091C00094E803008DE8030031460CCB284609F0F3
:1091D00091F90BE0CDE90310029294E803008DE8C9
:1091E000030031460CCB284609F014F9284607B095
:1091F000BDE8F04002B07047CDE90310029294E858
:1092000003008DE8030031460CCB284609F01EF917
:10921000ECE7CDE90310029294E803008DE8030027
:1092200031460CCB284609F02DF9DFE782B0F0B5C6
:1092300087B005469DF850700D93742F164613980D
:10924000DDE911210FAC0DAB1ED00ED8642F2DD04F
:10925000CDE90310029294E803008DE80300314643
:109260000CCB28460FF0A2FC1AE0772F2BD0CDE9CB
:109270000310029294E803008DE8030031460CCB02
:1092800028460FF0AFFC0BE0CDE90310029294E802
:1092900003008DE8030031460CCB28460FF032FC6A
:1092A000284607B0BDE8F04002B07047CDE9031092
:1092B000029294E803008DE8030031460CCB284667
:1092C0000FF03CFCECE7CDE90310029294E80300B8
:1092D0008DE8030031460CCB28460FF04BFCDFE74E
:1092E000F8B5AF4A0C466FF00103AE49054614F0DD
:1092F0008BFE064610B104682046F8BDAA4B9C427E
:1093000029D16820FCF74FFDA84B46600746C0E90D
:109310000266C0E90566C0E90766036006748684D4
:1093200080F864601420FCF73EFDA14B46600360AA
:10933000876031460446FEF7BFF96B68E56001338C
:109340006B609C4B236027613A4629464FF0000032
:1093500004F0E5FDD0E7984B9C4210D11020FCF7BB
:1093600022FD964B036046600446FCF783FF6B6862
:10937000C4E9020501336B60914B2360BCE7914B5C
:109380009C420AD10C20FCF70EFD6B6801336B6028
:10939000C0E901658C4B0446EFE78C4B9C420AD137
:1093A0000C20FCF700FD6B6801336B60C0E90165C0
:1093B000874B0446E1E7874B9C420AD10C20FCF71F
:1093C000F2FC6B6801336B60C0E90165824B0446B7
:1093D000D3E7824B9C422FD14420FCF7E4FC804B26
:1093E00006820746C0E90036C0E90266C0E90566A4
:1093F000C0E90766C0E90966C0E90B668674466382
:1094000080F843601420FCF7CEFC764B4660036086
:109410008760324631460446FDF7B6FE6B68E5606C
:1094200001336B60704B236027613A4629464FF049
:10943000000004F004FE5FE76C4B9C422FD14420F7
:10944000FCF7B1FC6A4B06820746C0E90036C0E96A
:109450000266C0E90566C0E90766C0E90966C0E9B9
:109460000B668674466380F843601420FCF79BFC0F
:10947000604B466003608760324631460446FDF724
:10948000C7FE6B68E56001336B605B4B236027614F
:109490003A4629464FF0000004F027FE2CE7574BD0
:1094A0009C420CD11420FCF77EFC3146044609F0A6
:1094B0003DF86B68256101336B60514B5DE7514BA3
:1094C0009C422CD14FF49470FCF76DFC00274E4B5E
:1094D00047600646C0E90277C0E90577C0E907772B
:1094E000C0E909770360077480F824711420FCF741
:1094F0005AFC464B47600360866039460446FEF7D7
:1095000043F96B68E56001336B60414B2360266172
:10951000324629464FF0000004F03FFDECE63D4B9B
:109520009C4210D11020FCF73EFC002343603A4BD4
:1095300003600446FCF79EFE6B6801336B60C4E970
:109540000205364B19E7364B9C420BD10C20FCF739
:109550002AFC0023C0E901356B6801336B600446C7
:10956000304B0AE7304B9C420BD10C20FCF71BFC24
:109570000023C0E901356B6801336B6004462B4B57
:10958000FBE62B4B9C4257D10C20FCF70CFC002334
:10959000C0E901356B6801336B600446254BECE68E
:1095A0000487020808820208001C00202C8302089D
:1095B000F8A10208F08C0208E41B0020DCA10208DC
:1095C000808C0208EC1B0020388D0208081C00204B
:1095D000888D0208041C0020B88D02080C1C002095
:1095E000B4820208A8A202081C8E0208101C0020E7
:1095F000C4820208DCA20208E88D0208E81B0020F1
:10960000B88C0208601C00203C830208F0A9020804
:10961000148D0208441C002094A902089C8C0208A6
:109620004C1C0020608D0208681C0020A08D0208E0
:10963000641C0020D08D02083E4B9C4231D170202A
:10964000FCF7B1FB00273C4B47600646C0E90277B8
:10965000C0E90577C0E90777C0E90977C0E90B776A
:10966000C0E90D7703600774C76380F86C7014203D
:10967000FCF799FB314B4760036086603A463946F8
:109680000446FDF73DFE6B68E56001336B602C4BD3
:1096900023602661324629464FF0000004F07BFD2E
:1096A0002AE6284B9C4231D17020FCF77CFB002736
:1096B000254B47600646C0E90277C0E90577C0E957
:1096C0000777C0E90977C0E90B77C0E90D77036038
:1096D0000774C76380F86C701420FCF764FB1B4BA5
:1096E0004760036086603A4639460446FDF750FEFF
:1096F0006B68E56001336B60154B23602661324671
:1097000029464FF0000004F09CFDF5E5114B9C420A
:109710000CD11420FCF747FB002104460FF07EFA21
:109720006B68256101336B600B4B26E60B4808F034
:1097300049F800BF6C1C0020D4820208A0AA0208CD
:10974000848E0208701C0020E4820208D4AA020859
:10975000508E0208481C0020D48C0208A086020803
:109760008B6913B5044613B9054808F02BF8D1E905
:10977000001201AB00F06EFE204602B010BD00BF2B
:10978000CD86020810B58AB0044600930020134627
:10979000C968099003AA05F0C5F903A92046FFF797
:1097A000DFFF03A8FFF7C9FA20460AB010BD30B5A5
:1097B0008DB0044600200B901198006850F80C5CA6
:1097C000CDE902051098CDE900301346096905AAD4
:1097D0004FF0000005F030FA05A92046FFF7C0FF62
:1097E00005A8FFF7AAFA20460DB030BD82B02DE9DA
:1097F000F04786B0044614999DF84480DDF84890FF
:109800009DF84CA00F9315460FAEB1B105AF384689
:10981000FFF7A6FFCDE902A7CDE90089204696E82B
:109820000C00294608F020FD384600F0B7FB204622
:1098300006B0BDE8F04702B07047CDE9019ACDF817
:10984000008096E80C00294608F0F8FCEFE7F0B538
:1098500097B00AAC84E80C000FAE0023CDE90636C1
:1098600015930D930DAB05931F9B04939DF87830D2
:1098700003931CAA8C46054692E8030001AB83E8DB
:1098800003000B9B009308AF0A9BDCF808204FF005
:109890000001384605F057F997E803000D9B84E86E
:1098A0000300A3B931460EA8FFF75AFF21980EA96D
:1098B00000F0C6FA0EA800F071FB94E8030085E8FA
:1098C00003003046FFF739FA284617B0F0BD209A5A
:1098D0001360F2E738B5836904460D4603B1984733
:1098E0002946204600F098FD2B6853F80C3C636035
:1098F000014BA361204638BDFD8400080000000034
:1099000070B590B009AD0E4606A981E80C0004467A
:109910001799002328460F93FFF7DCFF9DF8583076
:109920000393159B02939DF850300193079BB268F7
:1099300000939FED070B069B04954FF00001204616
:1099400005F018F82846FFF7F8F9204610B070BD6A
:10995000000000000000000013B5144601A81A46DC
:10996000049B08F00CFE01A92046FFF7B3FF01A8F5
:1099700000F014FB02B010BDF0B587B004AC0E4689
:1099800015461F46DDE90E1203AB204600F062FDCE
:109990000D9B00933A460C9B0194314605A808F0B4
:1099A000D8FD05A92846FFF795FF05A800F0F6FAAF
:1099B000204600F0F3FA07B0F0BD000082B02DE9B8
:1099C000F0438BB005461A9813931646DDE9181834
:1099D0009DF85C2015AB13AC98B1CDE90480CDE9BE
:1099E000022193E803008DE80300314694E80C005F
:1099F000284608F0E5FB28460BB0BDE8F04302B06E
:109A0000704709AFCDE90487CDE9022110480990DC
:109A100093E803008DE803000DF1180994E80C00A9
:109A20003146484608F0EBFB99E80300D8F80030CF
:109A300084E803001BB91B983946FFF74BFF94E8F5
:109A4000030085E80300384600F0A8FAD3E700BF1A
:109A5000141B00208B6913B5044613B9054807F0A1
:109A6000B1FED1E9001201AB01F078F8204602B056
:109A700010BD00BFCD86020810B58AB00446009321
:109A800000201346C968099003AA05F0E7F903A965
:109A90002046FFF7DFFF03A8FFF74FF920460AB083
:109AA00010BD30B58DB0044600200B9011980068B1
:109AB00050F80C5CCDE902051098CDE90030134652
:109AC000096905AA4FF0000005F052FA05A92046E1
:109AD000FFF7C0FF05A8FFF730F920460DB030BDF5
:109AE00082B02DE9F04786B0DDE9129A14999DF80D
:109AF00044800F93044615460FAEB1B105AF38460A
:109B0000FFF7A8FFCDE902A7CDE90089204696E836
:109B10000C0029460EF01FFF384600F0EBFD2046F2
:109B200006B0BDE8F04702B07047CDE9019ACDF824
:109B3000008096E80C0029460EF0F8FEEFE7F0B53D
:109B400097B00AAC84E80C000FAE0023CDE90636CE
:109B500015930D930DAB05931F9B04939DF87830DF
:109B600003931CAA8C46054692E8030001AB83E8E8
:109B700003000B9B009308AF0A9BDCF808204FF012
:109B80000001384605F07BF997E803000D9B84E857
:109B90000300A3B931460EA8FFF75CFF21980EA978
:109BA00000F00AFD0EA800F0A5FD94E8030085E88A
:109BB00003003046FFF7C1F8284617B0F0BD209AE1
:109BC0001360F2E738B5836904460D4603B1984740
:109BD0002946204600F0A4FF2B6853F80C3C636034
:109BE000014BA361204638BD01850008000000003C
:109BF00070B590B009AD0E4606A981E80C00044688
:109C00001799002328460F93FFF7DCFF169B039359
:109C1000159B02939DF850300193079BB268009307
:109C20009FED070B069B04954FF00001204605F0C1
:109C30003DF82846FFF781F8204610B070BD00BF00
:109C4000000000000000000013B5144601A81A46E9
:109C5000049B0FF00CF801A92046FFF7B3FF01A801
:109C600000F048FD02B010BDF0B587B004AC0E4660
:109C700015461F46DDE90E1203AB204600F06EFFCD
:109C80000D9B00933A460C9B0194314605A80EF0BB
:109C9000D8FF05A92846FFF795FF05A800F02AFD83
:109CA000204600F027FD07B0F0BD000082B02DE98E
:109CB000F0438BB005461A9813931646DDE9181841
:109CC0009DF85C2015AB13AC98B1CDE90480CDE9CB
:109CD000022193E803008DE80300314694E80C006C
:109CE00028460EF0E5FD28460BB0BDE8F04302B073
:109CF000704709AFCDE90487CDE9022110480990EA
:109D000093E803008DE803000DF1180994E80C00B6
:109D1000314648460EF0EBFD99E80300D8F80030D4
:109D200084E803001BB91B983946FFF74BFF94E802
:109D3000030085E80300384600F0DCFCD3E700BFF1
:109D4000241B002013460A4611B11978F6F740BAD1
:109D50000846704708B5034608461B6853F80C3C94
:109D60008342114603D20246014807F031FD08BD87
:109D7000B08E0208006801F1804150F80C0C0439E3
:109D8000091A914208B502D2184607F01EFD08BD17
:109D90000068884207D850F80C3C1844814294BFB0
:109DA00000200120704701207047012A30B403D100
:109DB0000B78037030BC7047002AFBD030BC16F023
:109DC00011B9012A30B403D10B78037030BC70474D
:109DD000002AFBD030BC16F013B90B46012B10B48F
:109DE0001146044603D122705DF8044B7047002BE6
:109DF000FAD05DF8044B1A4616F01CB908B5521A91
:109E0000FFF7D3FF08BD00002DE9F041044690465E
:109E10000F460A4A19461E46FFF79CFF216851F873
:109E20000C5CAC1B444528BF444624B12246314457
:109E30003846FFF7BAFF2046BDE8F081E78E0208FA
:109E4000036853F8042C002AB8BF002210B5B8BF2D
:109E500043F8042C0A6852F8044C002CBCBF0024C0
:109E600042F8044C02600B6010BD10B5036853F853
:109E70000C0C824204D29C5C8C4203D10132F8E784
:109E80004FF0FF32104610BD044B984204D000231F
:109E90008360016008440373704700BF081B002003
:109EA000154B984210B5044602D9144807F08DFCB2
:109EB000884203D94B00984238BF1C4604F11D0369
:109EC000B3F5805F04F10D000CD98C420AD90A4821
:109ED00004F58054C3F30B03E41A844228BF0446FC
:109EE00004F10D00002801DA07F066FCFBF75BFFC8
:109EF00000224460826010BDFCFFFF3FFA8E020822
:109F0000F8B50F46044680B10021FFF7C9FF00F104
:109F10000C060546214630463A46FFF75EFF2146CD
:109F20002846FFF7B1FF3046F8BD014EFBE700BF02
:109F3000141B002010B50446084611461A46FFF7C8
:109F4000DFFF2060204610BD2DE9F041A1EB0008A5
:109F500005460E4640460021FFF7A2FF00F10C0720
:109F60000446324629463846FFF748FF2046414618
:109F7000FFF78AFF3846BDE8F08114F041B80000D1
:109F8000054A904210B506D08268541E002A8460AB
:109F900001DCFFF7F2FF10BD081B002013B50446DB
:109FA000006801A90C38FFF7EBFF204602B010BD96
:109FB000036813B50446A3F10C0053F8043C002BCE
:109FC00006DD01A9FFF7DCFF034B236002B010BDE3
:109FD0000021FFF759FFF9E7141B00202DE9F74F87
:109FE0000546006850F80C7C02EB01090C46A3EB17
:109FF000020850F8081CB84488451E46A7EB09071C
:10A0000003D850F8043C002B1EDD01AA4046FFF7A0
:10A0100047FF824600F10C0B24B1296822465846BE
:10A02000FFF7C3FE47B1296804F10C0030443A46FB
:10A0300049445044FFF7B9FE286801A90C38FFF7DE
:10A040009FFFC5F800B000E03FB9286841460C38D2
:10A05000FFF71AFF03B0BDE8F08F9642F5D0344405
:10A0600000EB09013A462044FFF7ABFEEDE70000A4
:10A0700003680A4A934210B504460DD053F8043CD5
:10A08000002B04DD00231A461946FFF7A7FF2368BB
:10A090004FF0FF3243F8042C10BD00BF141B00200A
:10A0A00008B5036853F8043C002B01DBFFF7E0FF21
:10A0B00008BD10B50446FFF7F3FF206810BD00008F
:10A0C00070B504461546094A0E46FFF743FE23685D
:10A0D00053F80C2C921BAA4201464FF00003204675
:10A0E00028BF2A46FFF77AFF204670BD128F02086C
:10A0F000F8B51C4617460B4B05460E462246394618
:10A10000FFF738FE23463A4631462846FFF766FFFA
:10A1100034B128689DF8182021463044FFF75DFED1
:10A120002846F8BD268F020837B504680092054618
:10A130000C1B012300222146FFF7DAFF28684FF0AD
:10A14000FF3340F8043C204403B030BDF8B5069F0F
:10A150001E463B4604460D46FFF740FF2FB12068E0
:10A160003A4631462844FFF720FE2046F8BD00005D
:10A170002DE9F34107681A4B57F80C8C04460E463C
:10A1800041461546FFF7F6FD31462046FFF700FE33
:10A1900018B957F8043C002B0BDD204600953346D8
:10A1A00042460021FFF7D2FF0446204602B0BDE838
:10A1B000F081F31B9D420AD82A4631463846FFF704
:10A1C000F4FD206829460C38FFF75EFEEDE7002B12
:10A1D000F7D02A4631463846FFF7F3FDF1E700BFD6
:10A1E000438F0208034B98421EBF8368013383608C
:10A1F0000C307047081B002070B5044610462368D9
:10A200000A4618446168FFF74BFE2268054600F1D4
:10A210000C0622B104F10C013046FFF7C6FD2846BA
:10A220002168FFF731FE304670BD37B5044600683F
:10A2300050F8082C914203D150F8042C002A11DD6B
:10A2400050F80C2D91422CBFC2EB0102C2EB02026E
:10A2500001A9FFF7D1FF0546206801A90C38FFF7D7
:10A260008FFE256003B030BDF8B50B6853F80C7C49
:10A2700004460E46E7B1036853F80C5C53F8082C0B
:10A280003D44954203D853F8043C002B03DD294696
:10A290002046FFF7CAFF2368316853F80C0C3A4692
:10A2A0001844FFF782FD206829460C38FFF7ECFDC3
:10A2B0002046F8BD2DE9F04104460D4690462AB3EC
:10A2C000184B0021FFF756FD276857F80C6C57F81C
:10A2D000083C46449E4203D857F8043C002B08DD56
:10A2E00029462046FFF754FD98B131462046FFF736
:10A2F0009CFF236853F80C0C294618444246FFF78C
:10A3000054FD206831460C38FFF7BEFD2046BDE8FD
:10A31000F08131462046FFF788FF2168ED1B0D4490
:10A32000E7E700BF588F0208F8B5044617460D4608
:10A3300009B30A46114B0021FFF71CFD236853F8AF
:10A340000C6C53F8082C2E44964203D853F8043C66
:10A35000002B03DD31462046FFF767FF236853F8E3
:10A360000C0C294618443A46FFF737FD2068314661
:10A370000C38FFF789FD2046F8BD00BF588F020852
:10A38000F8B5036853F80C6C0B4B0C4617460A469D
:10A3900031460546FFF7EEFCA64205D23A46A11B20
:10A3A0002846FFF7C1FFF8BDFDD94FF0FF32214627
:10A3B0002846FFF785FEF6E76D8F020808B50022F4
:10A3C000FFF7DEFF08BD37B5026852F80C3C0D46BA
:10A3D000591C52F8083C9942044603D852F8043CF0
:10A3E000002B04DD20460191FFF71FFF0199236830
:10A3F00053F80C2C9D5420680C38FFF745FD03B032
:10A4000030BD08B58368002B02DBFFF7EBFE08BD0B
:10A410000022FFF7F1FEFAE713B50446086801AA27
:10A4200069460C38FFF7EDFF2060204602B010BDF2
:10A43000884208B507D018B1BDE80840FFF784BDD1
:10A44000024807F0BFF9024808BD00BF828F02082A
:10A45000141B002010B504460846114601441A4654
:10A460004FF00003FFF7E4FF2060204610BD10B559
:10A470000446084611461A464FF00003FFF7D8FF7E
:10A480002060204610BD37B505460C4671B1084620
:10A490000192F5F7F7FE019A21184FF000032046CC
:10A4A000FFF7C6FF2860284603B030BD4FF0FF31EC
:10A4B000F3E713460A4611B1196819F001BE0846C0
:10A4C0007047000008B5034608461B6853F80C3C6B
:10A4D0008342114603D20246014807F079F908BDCC
:10A4E000B08E0208006801F1805150F80C0C02395E
:10A4F000091A914208B502D2184607F066F908BD5C
:10A500000068884208D850F80C3C00EB8300814278
:10A5100094BF00200120704701207047012A30B409
:10A5200003D10B68036030BC7047002AFBD030BCFD
:10A5300019F0D5BD012A30B403D10B68036030BCDB
:10A540007047002AFBD030BC19F0CCBD0B46012B64
:10A5500010B41146044603D122605DF8044B7047E5
:10A56000002BFAD05DF8044B1A4619F0BEBD08B5B1
:10A57000521A9210FFF7D2FF08BD00002DE9F041FA
:10A58000044690460F460B4A19461E46FFF79AFFAF
:10A59000216851F80C5CAC1B444528BF44462CB1E3
:10A5A000224601EB86013846FFF7B8FF2046BDE89A
:10A5B000F08100BFE78E0208036853F8042C002ADC
:10A5C000B8BF002210B5B8BF43F8042C0A6852F88F
:10A5D000044C002CBCBF002442F8044C02600B6009
:10A5E00010BD0000044B984205D000238360016039
:10A5F00000EB8100C3607047181B00206FF07043B0
:10A60000984210B5044602D3114807F0DEF888429C
:10A6100003D94B00984238BF1C46201D800000F132
:10A620001003B3F5805F0DD98C420BD9C3F30B0334
:10A630000848C3F5805304EB9304844228BF0446C2
:10A64000201D8000FBF7AFFB00224460826010BD3C
:10A65000FA8E0208FEFFFF0FF8B50F46044680B1E0
:10A660000021FFF7CBFF00F10C06054621463046DE
:10A670003A46FFF76BFF21462846FFF7B3FF304607
:10A68000F8BD014EFBE700BF241B002010B50446B7
:10A69000084611461A46FFF7DFFF2060204610BD2E
:10A6A0002DE9F0410D1AAD1006460F46284600214F
:10A6B000FFF7A4FF00F10C0804463A463146404635
:10A6C000FFF755FF20462946FFF78CFF4046BDE8BF
:10A6D000F08113F095BC0000054A904210B506D0F9
:10A6E0008268541E002A846001DCFFF7F2FF10BD6F
:10A6F000181B002013B50446006801A90C38FFF7A9
:10A70000EBFF204602B010BD2DE9F74F054600686B
:10A7100050F80C6C02EB010A0F46A3EB020950F84B
:10A72000081CB14489451C46A6EB0A0603D850F81C
:10A73000043C002B1FDD01AA4846FFF75FFF80465F
:10A7400000F10C0B27B129683A465846FFF7E6FEA0
:10A750004EB129683C4408EB8400324601EB8A0183
:10A760000C30FFF7DBFE286801A90C38FFF7B4FFB7
:10A77000C5F800B000E03EB9286849460C38FFF73C
:10A7800031FF03B0BDE8F08F9442F5D03C4400EBBC
:10A790008A01324600EB8400FFF7CCFEECE70000B4
:10A7A00003680A4A934210B504460DD053F8043C9E
:10A7B000002B04DD00231A461946FFF7A5FF236886
:10A7C0004FF0FF3243F8042C10BD00BF241B0020C3
:10A7D00008B5036853F8043C002B01DBFFF7E0FFEA
:10A7E00008BD000070B504461546094A0E46FFF73D
:10A7F00069FE236853F80C2C921BAA4201464FF0C5
:10A800000003204628BF2A46FFF77EFF204670BD82
:10A81000128F0208F8B51C4617460B4B05460E462C
:10A8200022463946FFF75EFE23463A463146284621
:10A83000FFF76AFF34B12868069A214600EB8600CC
:10A84000FFF784FE2846F8BD268F0208F8B5069F5C
:10A850001E463B4604460D46FFF756FF37B12068BB
:10A860003A46314600EB8500FFF758FE2046F8BD1A
:10A870002DE9F34107681B4B57F80C8C04460E4634
:10A8800041461546FFF72EFE31462046FFF738FEBB
:10A8900018B957F8043C002B0BDD204600953346D1
:10A8A00042460021FFF7D2FF0446204602B0BDE831
:10A8B000F081F31BB5EBA30F4FEAA3020AD82A4697
:10A8C00031463846FFF72AFE206829460C38FFF744
:10A8D00089FEEAE7002AF7D02A4631463846FFF7D4
:10A8E00029FEF1E7438F0208034B98421EBF83689D
:10A8F000013383600C307047181B002070B504468C
:10A90000104623680A4618446168FFF777FE2268FC
:10A91000054600F10C0622B104F10C013046FFF7A8
:10A92000FDFD28462168FFF75DFE304670BD37B556
:10A930000446006850F8082C914203D150F8042CCA
:10A94000002A11DD50F80C2D91422CBFC2EB010200
:10A95000C2EB020201A9FFF7D1FF0546206801A959
:10A960000C38FFF7B9FE256003B030BDF8B50B68B1
:10A9700053F80C7C04460E46EFB1036853F80C5CA8
:10A9800053F8082C3D44954203D853F8043C002B5F
:10A9900003DD29462046FFF7CAFF2368316853F8D4
:10A9A0000C0C3A4603EB8000FFF7B8FD20682946FF
:10A9B0000C38FFF717FE2046F8BD00002DE9F041E6
:10A9C00004460D46904632B3184B0021FFF78AFD2E
:10A9D000276857F80C6C57F8083C46449E4203D849
:10A9E00057F8043C002B08DD29462046FFF788FD78
:10A9F000A0B131462046FFF79AFF236853F80C0CAC
:10AA0000294603EB80004246FFF788FD2068314667
:10AA10000C38FFF7E7FD2046BDE8F08131462046BF
:10AA2000FFF785FF2168ED1B0D44E6E7588F02080C
:10AA3000F8B5044617460D4611B30A46114B0021DE
:10AA4000FFF750FD236853F80C6C53F8082C2E4484
:10AA5000964203D853F8043C002B03DD31462046D0
:10AA6000FFF765FF236853F80C0C294603EB8000C1
:10AA70003A46FFF76BFD206831460C38FFF7B2FD10
:10AA80002046F8BD588F0208F8B5036853F80C6CDF
:10AA90000B4B0C4617460A4631460546FFF722FD8A
:10AAA000A64205D23A46A11B2846FFF7C1FFF8BDD2
:10AAB000FDD94FF0FF3221462846FFF793FEF6E717
:10AAC0006D8F020808B50022FFF7DEFF08BD37B51D
:10AAD000026852F80C3C0D46591C52F8083C994249
:10AAE000044603D852F8043C002B04DD20460191B3
:10AAF000FFF71DFF0199206850F80C3C40F82350E7
:10AB00000C38FFF76FFD03B030BD08B58368002B2C
:10AB100002DBFFF7E9FE08BD0022FFF7EFFEFAE7D0
:10AB200013B50446086801AA69460C38FFF7EDFF23
:10AB30002060204602B010BD884208B507D018B189
:10AB4000BDE80840FFF7ACBD024806F03BFE0248F6
:10AB500008BD00BF828F0208241B002010B50446E8
:10AB60000846114600EB81011A464FF00003FFF73B
:10AB7000E3FF2060204610BD10B50446084611468C
:10AB80001A464FF00003FFF7D7FF2060204610BDA4
:10AB900037B505460C4679B10846019219F016F909
:10ABA000019A04EB80014FF000032046FFF7C4FF39
:10ABB0002860284603B030BD6FF00301F3E7084674
:10ABC000704708467047000010B5084B044640F82F
:10ABD000083B13F05BFE237B1BB1A06908B113F0A7
:10ABE00011FA2046FBF724FB204610BD1090020806
:10ABF00010B50446FFF7E8FF204613F001FA20469F
:10AC000010BD8A4210B5144603D00298521A15F0AE
:10AC1000E9F9204610BD8A4238B51846144602D0DC
:10AC2000521A15F0DFF9204638BD000010B5064B6A
:10AC3000044640F8083B13F029FE044B23602046ED
:10AC4000FBF7F6FA204610BD40900208B0A90208B2
:10AC500010B50446FFF7EAFF204613F0D1F920466D
:10AC600010BD2DE9F041C0B06B46044600251F46DB
:10AC700003F8015B0135B5F5807FF9D1264640AA7E
:10AC800056F81D3B3946D3F81C8020463346C04752
:10AC9000012323772A463146384615F093F908B147
:10ACA0000223237740B0BDE8F0810000003918BFCF
:10ACB0000121074B10B5416003600446FBF7DAFA47
:10ACC0000023A0602373204600F088F9204610BDC1
:10ACD0004090020838B5003B18BF012343600F4B7A
:10ACE00003600F4B00250029044604BF2A4619467D
:10ACF000C0E90455027381614FF4807229461D300A
:10AD000015F098F925774FF48072294604F21D104A
:10AD100015F090F984F81D52204638BD10900208B5
:10AD20003BB8020883695B5C9B0744BF2039C9B20A
:10AD30000846704770B506460C461546AC4207D229
:10AD4000336821789B683046984704F8010BF5E793
:10AD5000284670BD83695B5CDB0744BF2031C9B204
:10AD60000846704770B506460C461546AC4207D2F9
:10AD7000336821781B693046984704F8010BF5E7E2
:10AD8000284670BD172911D8B1B14B1E162B13D808
:10AD9000DFE803F01C1E20221212261712121212D4
:10ADA000121212241212121212122800442906D072
:10ADB00097291CD0202907D011F0440F14D00D483A
:10ADC00000E00D4819F074B90C48FBE70C48F9E7AE
:10ADD0000C48F7E70C48F5E70C48F3E70C48F1E7B7
:10ADE0000C48EFE70C48EDE711F0970001D00B4855
:10ADF000E8E770479C900208CCBA02087E900208EF
:10AE0000849002088A900208909002089D9002089F
:10AE100096900208A3900208A99002087890020870
:10AE2000084617F0FFBE38B50C461546AC4205D2B1
:10AE3000206817F0F7FE44F8040BF7E7284638BD02
:10AE4000084617F0E3BE38B50C461546AC4205D2AD
:10AE5000206817F0DBFE44F8040BF7E7284638BDFE
:10AE60002DE9F0418846154600F5926700F5946695
:10AE700000F5936417F8013B13EA080F05D1A742C8
:10AE800006F10406F6D1002006E03168284614F0E9
:10AE90001FFF0028F3D00120BDE8F0812DE9F84F15
:10AEA00005460C4616461F4600F5986BB44217D26D
:10AEB00005F5946905F5926A4FF0000859F8041BEE
:10AEC000206814F005FF18B19AF8003048EA03082A
:10AED000D9450AF1010AF1D107F8018B0434E5E7FD
:10AEE0003046BDE8F88F2DE9F041054688461E46FC
:10AEF0001446B442274608D22B683A689B684146FC
:10AF00002846043498470028F3D03846BDE8F0813D
:10AF10002DE9F041054688461E461446B4422746B0
:10AF200008D22B683A689B68414628460434984703
:10AF30000028F3D13846BDE8F081243150F82100D3
:10AF4000704710B58A420C4607D924782434013161
:10AF500050F8244043F8044BF4E7104610BD7F2915
:10AF600010B503461446084605D81A7B1AB159187D
:10AF70004C7B204610BD18F0BFFF431C18BFC4B265
:10AF8000F7E72DE9F0411D46037B069E80460C46FF
:10AF9000174693B1A7421ED954F8040B7F2804D852
:10AFA0004044437B33700136F4E718F0A5FF421CA0
:10AFB00014BFC1B229463170F5E7A74223460AD92A
:10AFC000186818F099FF431C14BFC1B2294606F84F
:10AFD000011B0434F1E73846BDE8F0812DE9F0416A
:10AFE000044600F10D060025284618F085FF431C95
:10AFF00028D00135802D06F8010BF5D101232373EC
:10B0000004F190060025284614F08AF90135B5F5BB
:10B01000807F46F8040BF6D104F5926704F5946638
:10B0200000254FF0010808FA05F1C9B207F8011B25
:10B030002046FFF7A7FE0135082D46F8040BF2D194
:10B04000BDE8F0810023DAE78368587C70478368A5
:10B05000987C70478368D86A704783681B6B0020B0
:10B06000DAB262F30700C3F3072262F30F20C3F3DF
:10B07000074262F317401B0E82B063F31F6002B0F9
:10B08000704783685B6B0020DAB262F30700C3F39A
:10B09000072262F30F20C3F3074262F317401B0E2F
:10B0A00082B063F31F6002B070478368587C7047BA
:10B0B0008368987C70478368D86A704783681B6B85
:10B0C0000020DAB262F30700C3F3072262F30F2015
:10B0D000C3F3074262F317401B0E82B063F31F6095
:10B0E00002B0704783685B6B0020DAB262F307003E
:10B0F000C3F3072262F30F20C3F3074262F3174042
:10B100001B0E82B063F31F6002B07047836893F830
:10B1100024007047836893F825007047002070472B
:10B120000020704770470020914204D211F8013B83
:10B1300003EB7060F8E7704713B58B6801AA996854
:10B1400004460DF04BF8204602B010BD13B58B68D5
:10B1500001AA596904460DF041F8204602B010BD1D
:10B1600013B58B6801AAD96904460DF037F820465B
:10B1700002B010BD13B58B6801AA596A04460DF0E0
:10B180002DF8204602B010BD13B58B6801AA99684E
:10B1900004460DF023F8204602B010BD13B58B68AD
:10B1A00001AA596904460DF019F8204602B010BDF5
:10B1B00013B58B6801AAD96904460DF00FF8204633
:10B1C00002B010BD13B58B6801AA596A04460DF090
:10B1D00005F8204602B010BD13B58B6801AA996826
:10B1E00004460CF0FBFF204602B010BD13B58B687F
:10B1F00001AA596904460CF0F1FF204602B010BDC7
:10B2000013B58B6801AAD96904460CF0E7FF204604
:10B2100002B010BD10B5034B03600446FBF708F8FD
:10B22000204610BD2892020810B50446FFF7F2FF31
:10B23000204612F0E5FE204610BD000010B5034B7D
:10B2400003600446FAF7F4FF204610BD409202085E
:10B2500010B50446FFF7F2FF204612F0D1FE20465B
:10B2600010BD000010B5034B03600446FAF7E0FF81
:10B27000204610BD5892020810B50446FFF7F2FFB1
:10B28000204612F0BDFE204610BD000010B5054B53
:10B29000044640F8083B13F0F9FA2046FAF7C8FFD5
:10B2A000204610BD0C92020810B50446FFF7EEFFD1
:10B2B000204612F0A5FE204610BD000010B5054B3B
:10B2C000044640F8083B13F0E1FA2046FAF7B0FFD5
:10B2D000204610BD6491020810B50446FFF7EEFF4A
:10B2E000204612F08DFE204610BDD0E902218A4290
:10B2F00002D201328260704703689B6A184707B523
:10B3000000920B46002241680CF05CFD03B05DF832
:10B3100004FB00002DE9F04107461648FBF726F82C
:10B320003B68D3F80C8058F820500646EDB944200D
:10B33000FAF739FD104B05820446C0E90035C0E933
:10B340000255C0E90555C0E90755C0E90955C0E9EE
:10B350000B558574456380F84350394607F0F8FA79
:10B36000386832462146FBF7C7F858F82600BDE892
:10B37000F08100BF6C1B0020C482020838B543680E
:10B380009942054604D90A460A480B4906F020FAB4
:10B39000B2F1FF3F04D10368696000225A5438BDFE
:10B3A000002AFCD05B1A9A4228BF1A46BDE83840F2
:10B3B0000CF079BCB08E0208128F020810B504465A
:10B3C0000068FFF792FF4FF0FF33636010BD00008D
:10B3D0002DE9F04107461648FAF7C8FF3B68D3F855
:10B3E0000C8058F820500646EDB94420FAF7DBFCF3
:10B3F000104B05820446C0E90035C0E90255C0E99A
:10B400000555C0E90755C0E90955C0E90B558574D4
:10B41000456380F84350394607F0CAF93868324628
:10B420002146FBF769F858F82600BDE8F08100BF17
:10B43000681B0020B482020837B54568A94205D9C7
:10B440000A46064806492B4606F0C2F90093134601
:10B4500000220CF0B7FC03B030BD00BFB08E020874
:10B46000AF90020808B4FFB50E460420002117462D
:10B4700014F0ECFC16490546F4F7FAFE044680B1D8
:10B480002846F4F7FFFE421C1046019212F0B8FE67
:10B490002946019A044614F0A5FD0D49042014F034
:10B4A000D5FC0AAB099A03933946304617F0C4FE1F
:10B4B000054634B12146042014F0C8FC204612F0A1
:10B4C000A1FD284604B0BDE8F04001B0704700BFC0
:10B4D000C490020803689B68184770B5037F044650
:10B4E0000D4643B9FFF7BDFB2368294620469B69FB
:10B4F000BDE8704018474118487F70BDF7B5144645
:10B50000027F012A05460E4608D1A14203D0621AE5
:10B51000184614F067FD204603B0F0BD1AB9019338
:10B52000FFF79FFB019B2A68D769314622462846D0
:10B53000BC4603B0BDE8F040604770B544181646FD
:10B5400094F81D313BB903681B6A9847864203464D
:10B5500018BF84F81D01184670BD03689B68184722
:10B560000368DB68184710B50B6804461B699847E9
:10B57000204610BD10B50B6804465B69984720460D
:10B5800010BD10B50B6804469B699847204610BD56
:10B5900010B50B680446DB699847204610BD036868
:10B5A0001B6A184703685B6A82B002B018470368D9
:10B5B0009B6A82B002B0184703689B68184703680B
:10B5C000DB68184710B50B6804461B69984720468E
:10B5D00010BD10B50B6804465B699847204610BD46
:10B5E00010B50B6804469B699847204610BD10B5FE
:10B5F0000B680446DB699847204610BD03681B6A48
:10B60000184703685B6A82B002B0184703689B6AF8
:10B6100082B002B01847F0B589B006AE86E80C00DB
:10B62000139A0B680592129A0492119A03929DF84C
:10B63000402002920EAA04460D4692E803008DE8CF
:10B64000030020469F68294696E80C00B84720462C
:10B6500009B0F0BDF0B589B006AE86E80C00139ACB
:10B660000B680592129A0492119A03929DF8402059
:10B6700002920EAA04460D4692E803008DE80300EC
:10B680002046DF68294696E80C00B847204609B0F6
:10B69000F0BD70B586B004AC84E80C009DF8302095
:10B6A00002920B9A01920B689DF8282000929E68E6
:10B6B00094E80C000546B047284606B070BD70B54A
:10B6C00086B004AC84E80C000D9A03929DF83020FB
:10B6D00002920B9A01920B689DF828200092DE6876
:10B6E00094E80C000546B047284606B070BD0368D4
:10B6F0009B6818470368DB68184710B50B68044659
:10B700001B699847204610BD10B50B6804465B695D
:10B710009847204610BD10B50B6804469B699847B2
:10B72000204610BD03689B681847F0B589B006AE87
:10B7300086E80C00129A0B680492119A0392109AF0
:10B7400002920EAA04460D4692E803008DE803001B
:10B750002046DF68294696E80C00B847204609B025
:10B76000F0BDF0B589B006AE86E80C00129A0B6801
:10B770000492119A0392109A02920EAA04460D4660
:10B7800092E803008DE8030020461F69294696E8E9
:10B790000C00B847204609B0F0BDF0B589B006AE40
:10B7A00086E80C00129A0B680492119A0392109A80
:10B7B00002920EAA04460D4692E803008DE80300AB
:10B7C00020465F69294696E80C00B847204609B034
:10B7D000F0BDF0B589B006AE86E80C00129A0B6891
:10B7E0000492119A0392109A02920EAA04460D46F0
:10B7F00092E803008DE8030020469F69294696E8F9
:10B800000C00B847204609B0F0BDF0B589B006AECF
:10B8100086E80C00129A0B680492119A0392109A0F
:10B8200002920EAA04460D4692E803008DE803003A
:10B830002046DF69294696E80C00B847204609B043
:10B84000F0BD0000003910B5054B036018BF0121A1
:10B8500041600446FAF70EFDA060204610BD00BF0F
:10B860000C92020803689B68184773B5079E0196FF
:10B870000D68069E0096ED680446A847204602B073
:10B8800070BD03681B69184710B40468A468A44617
:10B890005DF8044B604738B50D680446ED68A8476D
:10B8A000204638BDF7B56D4685E806009DF8046072
:10B8B000089F0446194636B900983A460CF003F939
:10B8C000874218BF01268DF8046095E8030084E8DC
:10B8D0000300204603B0F0BD2DE9F04F99B006A952
:10B8E000DDF88880059008F16C04204681E80C00A2
:10B8F000249F9DF88C9006F049FE06462046FFF7EF
:10B9000067FD3D6890F838302A789A4204467A6894
:10B910007DD0036B0993D0F820A0C36903932A4418
:10B920002B469A421F4606D93878B169095C490707
:10B9300003F10103F5D47F1B00F0BA800EAB4FF08A
:10B94000000B79000CA80C93CDF834B08DF838B00A
:10B950000CF0E6F9E36AFE1A5E451DDDE1680D9A1A
:10B960005B45B8BF3E4600295CD073005946CDF810
:10B9700000B00CA80CF026FAAB19A17C0C98CDE90C
:10B980000053D4E9022307F00DF90C994FF0FF3270
:10B99000411A0CA8FFF7F2FCE36A002B0ADD617C78
:10B9A0000CA80CF0EFF9002E42DBE26AA9190CA8F2
:10B9B0000CF014FBD8F80C5005F0B003049315F408
:10B9C00000750D9B18BFA5690AEB0302154414AB63
:10B9D0000026690012A8129313968DF850600CF09F
:10B9E0009FF9049BD8F80870102B03D1BD422CBFDF
:10B9F000002601264FF0000B7D1B09AB13F80B301E
:10BA0000042B27D8DFE803F0786F1D606900436BD3
:10BA10000993436AD0F828A00393002A3FF47FAF2C
:10BA200001357CE700962B460CA80CF037FAB3E7FB
:10BA300094F8392071420CA8FFF761FC3A46294678
:10BA4000B5E7D8F80C309B0504D5D4E9051212A847
:10BA50000CF0C4FA0BF1010BBBF1040FCDD1BAF11C
:10BA6000010F06D903990AF1FF32013112A80CF037
:10BA7000B5FA13998F4249D9049B202BA7EB0101FA
:10BA80003DD14A4612A8FFF73AFC0AACDDE906129E
:10BA9000129B00972046FFF705FF94E803000690ED
:10BAA00012A88DF81C100CF047F80CA80CF044F804
:10BAB000DDE906010023C8F80830059B83E8030090
:10BAC000184619B0BDE8F08FBAF1000FC2D0039B41
:10BAD000197812A80CF056F9BCE7DDE90C1212A88F
:10BAE0000CF05AFAB6E72EB14A46294612A8FFF7DB
:10BAF00006FCAFE74946ECE7002EABD0F4E70A4678
:10BB00004B46002112A8FFF797FCBEE70F46BCE7A3
:10BB10002DE9F04F99B006A9DDF88880059008F16D
:10BB20006C04204681E80C00249F9DF88C9006F060
:10BB30002DFD06462046FFF7EDFB3D6890F83830B6
:10BB40002A789A4204467A687DD0036B0993D0F82C
:10BB500020A0C36903932A442B469A421F4606D964
:10BB60003878B169095C490703F10103F5D47F1BFB
:10BB700000F0BA800EAB4FF0000B79000CA80C93CC
:10BB8000CDF834B08DF838B00CF0CAF8E36AFE1A7C
:10BB90005E451DDDE1680D9A5B45B8BF3E46002954
:10BBA0005CD073005946CDF800B00CA80CF00AF92F
:10BBB000AB19A17C0C98CDE90053D4E9022306F01F
:10BBC000F1FF0C994FF0FF32411A0CA8FFF7D6FB9A
:10BBD000E36A002B0ADD617C0CA80CF0D3F8002E80
:10BBE00042DBE26AA9190CA80CF0F8F9D8F80C505D
:10BBF00005F0B003049315F400750D9B18BFA569FB
:10BC00000AEB0302154414AB0026690012A8129334
:10BC100013968DF850600CF083F8049BD8F80870E8
:10BC2000102B03D1BD422CBF002601264FF0000B84
:10BC30007D1B09AB13F80B30042B27D8DFE803F08A
:10BC4000786F1D606900436B0993436AD0F828A0A0
:10BC50000393002A3FF47FAF01357CE700962B4623
:10BC60000CA80CF01BF9B3E794F8392071420CA82A
:10BC7000FFF745FB3A462946B5E7D8F80C309B0557
:10BC800004D5D4E9051212A80CF0A8F90BF1010BA8
:10BC9000BBF1040FCDD1BAF1010F06D903990AF116
:10BCA000FF32013112A80CF099F913998F4249D94A
:10BCB000049B202BA7EB01013DD14A4612A8FFF7B8
:10BCC0001EFB0AACDDE90612129B00972046FFF727
:10BCD000E9FD94E80300069012A88DF81C100BF003
:10BCE0002BFF0CA80BF028FFDDE906010023C8F8A4
:10BCF0000830059B83E80300184619B0BDE8F08FB3
:10BD0000BAF1000FC2D0039B197812A80CF03AF8D0
:10BD1000BCE7DDE90C1212A80CF03EF9B6E72EB133
:10BD20004A46294612A8FFF7EAFAAFE74946ECE788
:10BD3000002EABD0F4E70A464B46002112A8FFF7CD
:10BD40007BFBBEE70F46BCE72DE9F04F2DED028BE4
:10BD5000B0EE408AF0EE608A91B004AF07F10804BB
:10BD600084E80C0097F860307B607B6E97F868A0E1
:10BD70000546884607F1140003F16C01FAF762FAF0
:10BD800007F1140006F002FC90B08146FAF772FA4F
:10BD900004AE4FF0000BB86131468DED028B2E4B97
:10BDA000CDF800B0402207F11800FFF75BFB3F28F9
:10BDB000014616DD083121F00701ADEB010D421CF3
:10BDC0003A60FAF757FA04AEB86131468DED028B4E
:10BDD000214B3A68CDF800B007F11800FFF742FB9D
:10BDE000014607F12003002207F11800BB6139600A
:10BDF0000BF0F9FE3968BB69721848463146FFF707
:10BE00007DFB7B68D3B107F11803CDE901A37B6EFD
:10BE10000093414694E80C002846FFF75DFD07F1CA
:10BE200018000BF089FE07F11400FAF779FA28469A
:10BE30003437BD46BDEC028BBDE8F08F07F1180327
:10BE4000CDE901A37B6E0093414694E80C0028469F
:10BE5000FFF75EFEE3E700BFC6900208F0B587B0CB
:10BE600004AC84E80C000F9E9DF838200D9B9DF8D3
:10BE700030700093CDE90126054694E80C0027B107
:10BE8000FFF72AFD284607B0F0BDFFF741FEF9E7AE
:10BE900010B50446D0E9003043B1421C06D1184623
:10BEA0000BF0F7FD431C04BF0023236010BD38B521
:10BEB0000D46FFF7EDFF04462846FFF7E9FF431C58
:10BEC000584204F10102584154425441011B484276
:10BED000484138BD08B5FFF7EAFF80F00100C0B265
:10BEE00008BD2DE9F74F0546DDE9120602A96C30C1
:10BEF000DDF8449001E90C0006F048FBB9F1020FAF
:10BF000082462FD0B9F1040F0CBF4FF47A77012786
:10BF10000024A0464FF00A0B0CA96846FFF7DAFF91
:10BF200010B3C84522D06846FFF7B2FF2A22C1B23B
:10BF30005046FFF702FB3038C2B2092A21D8109BC5
:10BF40000BFB040404FB07F29A421ADC0F9B3A44F1
:10BF50009A4216DDB7FBFBF76846FFF72FFA08F1A8
:10BF60000108D9E70A27D3E7C8450AD10E9B1C6010
:10BF700002AB13E9030085E80300284603B0BDE8DF
:10BF8000F08FB9F1040F04D1B8F1020F01D1643C74
:10BF9000ECE7336843F004033360E9E72DE9F04F41
:10BFA00085B000AF07F108047860F86CD7F84490CA
:10BFB0006C3084E80C0006F0E9FABB6C9B00073398
:10BFC00023F007038246ADEB030D07F1380120464D
:10BFD0006E46FFF77FFF002843D02046FFF758FF4B
:10BFE0004FF000085FFA80FB4546BB6C984510D0C7
:10BFF00059F828100978594505D146F825800135AA
:10C0000008F10108F1E75046FFF764FA5845F7D107
:10C01000F3E74FF0000A012D4ED9B04658F8043B23
:10C0200059F82300F4F72EF906EB8501834658F8FA
:10C03000040B396059F82000F4F724F93968834576
:10C0400028BF83464145F2D120460AF1010AFFF795
:10C05000B5F9DA4505D207F138012046FFF73AFF76
:10C0600078B93B6D3A6D1B6843F00403136094E8A4
:10C0700003007B68143783E803001846BD46BDE81B
:10C08000F08F4FF0000B56F82B2059F82220204655
:10C0900012F80A203A60FFF7FBFE3A68C0B282420B
:10C0A00017BF05F1FF350BF1010B56F8252046F8B7
:10C0B0002B205D45E7D8AEE7D3D12046FFF77EF9C8
:10C0C000366859F826904846F4F7DCF80AF1010A78
:10C0D0000546AA4514D207F138012046FFF7FAFEBB
:10C0E0000028BED0204619F80AB0FFF7D1FEC0B232
:10C0F0008345B6D12046FFF761F90AF1010AE8E766
:10C10000AFD13B6C1E60B2E72DE9F04F87B000AFB6
:10C110008146786DD7E913AB07F110046C3084E8E1
:10C120000C0006F033FA6B46A3EBCB0306469D46A4
:10C1300007F140012046E846FFF7CCFEC0B3204699
:10C14000FFF7A6FE4FEA4B03FB600023C2B21D4679
:10C15000F968994213D05AF823100978914204D112
:10C1600048F8253001350133F2E73046C7E90123AD
:10C17000FFF7B0F97A68BB689042F4D1F0E7BDB13F
:10C180002046FFF71BF9AB00073323F00703ADEBA5
:10C19000030D6E46002458F824305AF82300F4F7B3
:10C1A00071F846F824000134A542F4D1012502E0DB
:10C1B00000242546264607F1400107F11000FFF74D
:10C1C00089FE60B307F11000FFF762FE0023C0B2E2
:10C1D00019469C421BD956F82320AA424FEA830EE7
:10C1E00006EB830C02D801310133F2E758F8232023
:10C1F0005AF82220525D8242F6D0013C58F82420A1
:10C2000048F80E2056F82420CCF80020E1E78C42B4
:10C2100005D007F11000FFF7D1F80135CBE7012C6D
:10C2200015D13368AB4219D1D8F80030BA6C5B45F0
:10C23000A8BFA3EB0B03136007F1180313E9030076
:10C240001C3789E803004846BD46BDE8F08F022C44
:10C2500004D13368AB42E7D07368E3E7BB6DBA6DD6
:10C260001B6843F00403E6E72DE9F04F9FB00C464E
:10C27000DDF8A8A00B900AF16C050EA9284681E80C
:10C280000C00DDF8B09006F015FC8346284606F059
:10C290007DF905462D98F3F7F5FF00260A901096D4
:10C2A0000EAF28A93846FFF715FEDDF840800028BC
:10C2B00066D00A9B9E4263D2B8F1000F64D12D9BD9
:10C2C0004246995D2846FFF738F9252840F0AA82B2
:10C2D000731C0993711C2D9B4246595C2846FFF73D
:10C2E0002CF94528CDF8448001D04F2808D1B31C43
:10C2F000099309992D9B0022595C2846FFF71DF9E7
:10C3000041380EAE382800F28882DFE810F06A006B
:10C310009500D801EE008602860286020E013201E7
:10C3200086028602860260018602860286028602F4
:10C3300094019901C801860286028602D301D801C0
:10C340000202860286028602860286028602440075
:10C3500070009B00A100C500860286027000860264
:10C360008602860286023C018501860286028602DA
:10C3700086028602BE01860286028602CC01D801B0
:10C38000B8F1000F00F060822B9B2B9A1B6843F0E2
:10C39000040313605CE212AE3146584605F0E2FF3A
:10C3A00010ABCDE905A30723CDE9036311AB0293DD
:10C3B00028AB93E803008DE803000CAF0EAE96E8BF
:10C3C0000C0021463846FFF7E9FD97E80300109B73
:10C3D00086E8030013B9119BC9F81830099E01368D
:10C3E0005EE712AE3146584605F0ACFFD8E712AE14
:10C3F0003146584605F0E5FF10ABCDE905A30C2307
:10C40000CDE9036311AB029328AB93E803008DE8F9
:10C4100003000CAF0EAE96E80C0021463846FFF73D
:10C42000BDFD97E80300109B86E80300002BD5D1E3
:10C43000119BC9F81030D1E712AE3146584605F0CD
:10C44000A1FFD9E7DBF808309B690CAF059356E0F4
:10C4500010ABCDE906A34FF0020C1F23CDE9043C3D
:10C460000123039311AB029328AB93E803008DE8FB
:10C4700003000CAF0EAE96E80C0021463846FFF7DD
:10C4800030FD97E80300109B86E80300002BA5D140
:10C49000119BC9F80C30A1E73046FFF7F9FCAB69F6
:10C4A000C0B21B5C1F0716D50E98FEF71EFF4FF09B
:10C4B000FF330F9310ABCDE906A309220123CDE989
:10C4C00004230CAF039311AB029328AB93E8030052
:10C4D0008DE80300CFE710ABCDE906A302201F23B0
:10C4E000CDE904300CAF0A23ECE712AEC04A334664
:10C4F000A2F109012846FFF701F80CAF059610AB31
:10C50000CDE902A3CDF8109028AB93E803008DE8A5
:10C5100003000EAE2146384696E80C00FFF7A4FE55
:10C5200097E8030086E8030058E710ABCDE906A3BF
:10C5300002211723CDE904310CAF0023039311AB83
:10C54000029328AB93E803008DE803000EAE96E853
:10C550000C0021463846FFF7C4FC97E80300109B07
:10C5600086E80300002B7FF439AF119BC9F808302F
:10C5700034E710ABCDE906A302220C23CDE9043247
:10C580000CAF0123DAE710ABCDE906A34FF00208A8
:10C590000C23CDE904380123039311AB029328AB9C
:10C5A00093E803008DE803000CAF0EAE96E80C0094
:10C5B00021463846FFF795FC97E80300109B86E874
:10C5C0000300002B7FF40AAF119B013B31E710AB56
:10C5D000CDE906A34FF0020E3B23CDE9043E002334
:10C5E000039311AB029328AB93E803008DE803009B
:10C5F0000CAF0EAE96E80C0021463846FFF771FCF2
:10C6000097E80300109B86E80300002B7FF4E6AE5A
:10C61000119BC9F80430E1E63046FFF739FC0022EF
:10C62000C1B22846FEF789FF0A2840F0F68030465E
:10C63000FEF7C4FED2E66F4A12AE3346911F59E7A9
:10C6400010ABCDE906A34FF0020C3D23CDE9043C2D
:10C650000023039311AB029328AB93E803008DE80A
:10C6600003000CAF0EAE96E80C0021463846FFF7EB
:10C6700038FC97E80300109B86E80300002B7FF44A
:10C68000ADAE119BC9F80030A8E63046FFF700FCBC
:10C690000022C1B22846FEF750FF0928C5E712AEB6
:10C6A000554A334624E712A9584605F039FE129B35
:10C6B0000CAFCBE612A9584605F038FEF7E710ABF1
:10C6C000CDE906A3042642F20F73CDE90436002318
:10C6D000039311AB029328AB93E803008DE80300AA
:10C6E0000CAF0EAE96E80C0021463846FFF7F9FB7A
:10C6F00097E80300109B86E80300002B7FF46EAEE2
:10C70000119B002BB4BF6433A3F26C73C9F81430CF
:10C7100064E63046FFF7BCFBAB69C0B21B5CD807D0
:10C720007BD510ABCDE905A30E230493334B0393C4
:10C7300012AB029328AB93E803008DE803000CAF23
:10C740002146384696E80C00FFF728FC97E80300DE
:10C7500086E8030028A93046FFF7BCFB00283FF419
:10C760003DAE109A129B13437FF438AE3046FFF76C
:10C770008FFB2D2107462846FEF7AFFEFFB2B842D9
:10C780003ED110AF17230222CDE90432CDE906A72E
:10C790000023039312AB029328AB93E803008DE8C8
:10C7A00003000CAE0DF1380898E80C002146304625
:10C7B000FFF797FB96E803003B2388E8030002217C
:10C7C000CDE90431CDE906A70023039312AB029310
:10C7D00028AB93E803008DE803002146304698E833
:10C7E0000C00FFF77EFB96E8030088E80300F5E500
:10C7F000D5900208DB900208E49002082C0000208B
:10C800003046FFF745FB2B2106462846FEF765FE1E
:10C81000F6B2B0427FF4E2ADB3E7109B43F00403FD
:10C820001093DBE52D9B384613F80680FFF730FBAD
:10C83000C0B2804503D13846FEF7C0FDCFE5109B5E
:10C8400043F004031093CAE50A9B9E427FF49CAD1B
:10C8500097E803000B9B83E8030018461FB0BDE870
:10C86000F08F00BFF0B58FB00AAC84E80C000DAAC1
:10C870000792169A06928C4642F20F720421CDE975
:10C880000421002303930D930CAB029314AB0546D4
:10C8900093E803008DE8030008AF94E80C006146BC
:10C8A0003846179EFFF71DFB97E803000D9B84E8B1
:10C8B0000300BBB90C9B189A002BB4BF6433A3F2DE
:10C8C0006C73536114A92046FFF7F1FA18B133686D
:10C8D00043F00203336094E8030085E80300284630
:10C8E0000FB0F0BD336843F004033360EAE72DE98D
:10C8F000F0479CB0DDE926960AAC054609F16C00CC
:10C9000084E80C00884606F0D5F80DF1380A074691
:10C91000514605F027FD384615A905F013FD002303
:10C920000D930DABCDE905930723CDE903A30CAB24
:10C93000029324AB93E803008DE8030008AF94E86A
:10C940000C0041463846FFF7DFFB97E803000D9BDC
:10C9500084E803009BB9289B0C9A9A6124A920467D
:10C96000FFF7A5FA18B1336843F00203336094E887
:10C97000030085E8030028461CB0BDE8F087336853
:10C9800043F004033360E9E72DE9F047A6B0DDE9A1
:10C9900030960AAC054609F16C0084E80C00884624
:10C9A00006F088F80DF1380A0746514605F009FDF2
:10C9B00038461AA905F0E6FC00230D930DABCDE92E
:10C9C00005930C23CDE903A30CAB02932EAB93E8A4
:10C9D00003008DE8030008AF94E80C004146384698
:10C9E000FFF792FB97E803000D9B84E803009BB9D7
:10C9F000329B0C9A1A612EA92046FFF758FA18B1FB
:10CA0000336843F00203336094E8030085E80300D1
:10CA1000284626B0BDE8F087336843F0040333604E
:10CA2000E9E72DE9F0438DB0DDE9169608AC05463F
:10CA300009F16C0084E80C00884606F03BF80AA96E
:10CA400005F074FC0A9B0593189BCDF80890CDE97E
:10CA5000036314AB93E803008DE8030006AF41467F
:10CA6000384694E80C00FFF7FFFB97E8030084E8E2
:10CA7000030014A92046FFF71AFA18B1336843F0EF
:10CA80000203336094E8030085E8030028460DB0F4
:10CA9000BDE8F0832DE9F0438DB0DDE9169608ACD2
:10CAA000054609F16C0084E80C00884606F002F89F
:10CAB0000AA905F035FC0A9B0593189BCDF8089050
:10CAC000CDE9036314AB93E803008DE8030006AFE0
:10CAD0004146384694E80C00FFF7C6FB97E8030090
:10CAE00084E8030014A92046FFF7E1F918B1336880
:10CAF00043F00203336094E8030085E8030028460E
:10CB00000DB0BDE8F0832DE9F04F8DB0DDE918964A
:10CB1000054608AC09F16C004FF0000A84E80C00EF
:10CB200088469DF86CB09DF8707005F02FFDC6F832
:10CB300000A02521FEF7D1FC8DF82C005FBB8DF8FD
:10CB40002DB08DF82E700BAB05931A9BCDF8089085
:10CB5000CDE9036316AB93E803008DE8030006AF4D
:10CB60004146384694E80C00FFF77EFB97E8030047
:10CB700084E8030016A92046FFF799F918B1336835
:10CB800043F00203336094E8030085E8030028467D
:10CB90000DB0BDE8F08F8DF82D708DF82EB08DF8AA
:10CBA0002FA0D0E72DE9F04F2DED028B99B008A909
:10CBB00081E80C00DDE9263803F16C04069020467C
:10CBC00005F0E4FC04902046FEF702FC00F1380377
:10CBD0000793036A04461BB1836A003B18BF012315
:10CBE00002930EAB0C9300230D938DF83830237C09
:10CBF0001BB120210CA80BF093F8002514AB2021C9
:10CC000012A8129313958DF850500BF089F804F187
:10CC1000390308EE103A636B0B932F462E460395AB
:10CC2000A94601950BAB5B5D042B40D8DFE813F000
:10CC300058012B012B00A200DE00BAF1000FF1D148
:10CC4000D8F8003043F00403C8F8003008AC24A939
:10CC50002046FFF72CF928B1D8F8003043F0020342
:10CC6000C8F8003094E80300069B83E8030012A88C
:10CC70000AF062FF0CA80AF05FFF069819B0BDEC3D
:10CC8000028BBDE8F08F269BDB6898051ED4B9F1B6
:10CC9000010F1BD8D5B1012D0CD1029BB3B99DF862
:10CCA0002C30032B12D09DF82E30012B0ED04FF0DC
:10CCB000010A2CE0022DFAD19DF82F30042B05D06B
:10CCC000029A002AF3D0032B40F00D81A36905934B
:10CCD0004FF0000B24A908A8FFF7FCF8059B82463B
:10CCE00000283ED09B4512D008A8FFF7D1F8636911
:10CCF00013F80B30C0B2834236D0BBF1000F40F0C6
:10CD0000F580269BDB6883F40073C3F3402A01356A
:10CD1000042D92D1B9F1010F40F22D81BAF1000F2B
:10CD20008ED0019B002B00F0E480656A4FF0010B70
:10CD300024A908A8FFF7CEF8002800F0DC80D94528
:10CD400000F0DC8008A8FFF7A3F815F80B30C0B29C
:10CD500083427FF475AF08A8FEF730FB0BF1010B9F
:10CD6000E6E79B45C9D1A2E708A8FEF727FB0BF130
:10CD7000010BAFE7236ABBB9A36A53B324A908A880
:10CD8000FFF7A8F8824620B308A8FFF781F8626A87
:10CD90001278C0B282421CD108A8D4F82890FEF7BD
:10CDA0000DFBCDF804A0B2E724A908A8FFF792F87C
:10CDB00082460028E0D008A8FFF76AF8E2691278F6
:10CDC000C0B28242D8D108A8D4F82090FEF7F6FA73
:10CDD0009DE7236A1BB9029B83F0010A97E7A36AC8
:10CDE000002BF8D1012301939A4690E724A908A8C3
:10CDF000FFF770F88246002842D008A8FFF748F8ED
:10CE00000DF12B025FFA80FB0A2118EE100A8DF853
:10CE10002BB0FCF797FF80B1079BC01A594B1B68DA
:10CE2000195C12A80AF0AEFF06F1010B039E08A8D8
:10CE3000FEF7C4FA03965E46D8E7627C5A4506D1EF
:10CE40002FB9E26A002A11DD57468346EFE7227CBC
:10CE500062B1A37C5B4508D177B97EB1F1B20CA871
:10CE60000AF090FFBB46039EE1E79246139A002A20
:10CE700008BF4FF0000A4AE7BA46F7E7B246F5E7BF
:10CE80004FF0010AF2E724A908A8FFF723F8824629
:10CE9000C8B94FF0000A032D3FF439AF24A908A800
:10CEA000FFF718F800283FF432AF08A8FEF7F0FFAC
:10CEB000049BC0B29A69125C12077FF528AF08A8DC
:10CEC000FEF77CFAEAE708A8FEF7E2FF049BC0B28F
:10CED0009A69125C1107DCD508A8FEF76FFADAE749
:10CEE0004FF0010AD7E7DDF808A010E74FF0000A7D
:10CEF0000DE7E5691AE7D9457FF4A2AE139B012B34
:10CF000011D90022302112A80BF002F9024650B1CB
:10CF1000431C08BF13984FF0000108BF00F1FF3217
:10CF200012A8FEF72BFA019B3BB112990B78302B1C
:10CF300003D02D2212A80AF0A3FF0D9B8BB1F7B1ED
:10CF40009DF80C100CA80AF01DFFD4E902010CAAF0
:10CF500011F0C7FE28B9D8F8003043F00403C8F830
:10CF600000301FB1E36AB3427FF46AAE289812A979
:10CF70000BF060F86AE6BAF1000FBFD160E6F1B2DB
:10CF8000E0E700BF280000202DE9F04F2DED028BD7
:10CF900099B008A981E80C00DDE9263803F16C049A
:10CFA0000690204605F0F2FA04902046FEF7B2F90A
:10CFB00000F138030793036A04461BB1836A003B00
:10CFC00018BF012302930EAB0C9300230D938DF831
:10CFD0003830237C1BB120210CA80AF0A1FE0025CB
:10CFE00014AB202112A8129313958DF850500AF01B
:10CFF00097FE04F1390308EE103A636B0B932F464A
:10D000002E460395A94601950BAB5B5D042B40D8DA
:10D01000DFE813F058012B012B00A200DE00BAF16B
:10D02000000FF1D1D8F8003043F00403C8F8003005
:10D0300008AC24A92046FEF73AFF28B1D8F8003002
:10D0400043F00203C8F8003094E80300069B83E82D
:10D05000030012A80AF070FD0CA80AF06DFD0698F6
:10D0600019B0BDEC028BBDE8F08F269BDB689805FC
:10D070001ED4B9F1010F1BD8D5B1012D0CD1029BE3
:10D08000B3B99DF82C30032B12D09DF82E30012B14
:10D090000ED04FF0010A2CE0022DFAD19DF82F306E
:10D0A000042B05D0029A002AF3D0032B40F00D8107
:10D0B000A36905934FF0000B24A908A8FEF70AFF07
:10D0C000059B824600283ED09B4512D008A8FEF75B
:10D0D000DFFE636913F80B30C0B2834236D0BBF178
:10D0E000000F40F0F580269BDB6883F40073C3F3E8
:10D0F000402A0135042D92D1B9F1010F40F22D8162
:10D10000BAF1000F8ED0019B002B00F0E480656A1D
:10D110004FF0010B24A908A8FEF7DCFE002800F060
:10D12000DC80D94500F0DC8008A8FEF7B1FE15F8D8
:10D130000B30C0B283427FF475AF08A8FEF73EF90A
:10D140000BF1010BE6E79B45C9D1A2E708A8FEF762
:10D1500035F90BF1010BAFE7236ABBB9A36A53B3EF
:10D1600024A908A8FEF7B6FE824620B308A8FEF759
:10D170008FFE626A1278C0B282421CD108A8D4F82D
:10D180002890FEF71BF9CDF804A0B2E724A908A85F
:10D19000FEF7A0FE82460028E0D008A8FEF778FE41
:10D1A000E2691278C0B28242D8D108A8D4F820909F
:10D1B000FEF704F99DE7236A1BB9029B83F0010A7D
:10D1C00097E7A36A002BF8D1012301939A4690E7D1
:10D1D00024A908A8FEF77EFE8246002842D008A8AF
:10D1E000FEF756FE0DF12B025FFA80FB0A2118EEC6
:10D1F000100A8DF82BB0FCF7A5FD80B1079BC01A73
:10D20000594B1B68195C12A80AF0BCFD06F1010B12
:10D21000039E08A8FEF7D2F803965E46D8E7627C24
:10D220005A4506D12FB9E26A002A11DD57468346D6
:10D23000EFE7227C62B1A37C5B4508D177B97EB170
:10D24000F1B20CA80AF09EFDBB46039EE1E79246B0
:10D25000139A002A08BF4FF0000A4AE7BA46F7E7D8
:10D26000B246F5E74FF0010AF2E724A908A8FEF755
:10D2700031FE8246C8B94FF0000A032D3FF439AFA2
:10D2800024A908A8FEF726FE00283FF432AF08A81C
:10D29000FEF7FEFD049BC0B29A69125C12077FF58F
:10D2A00028AF08A8FEF78AF8EAE708A8FEF7F0FD1D
:10D2B000049BC0B29A69125C1107DCD508A8FEF77E
:10D2C0007DF8DAE74FF0010AD7E7DDF808A010E7AC
:10D2D0004FF0000A0DE7E5691AE7D9457FF4A2AEE1
:10D2E000139B012B11D90022302112A80AF010FF44
:10D2F000024650B1431C08BF13984FF0000108BF0D
:10D3000000F1FF3212A8FEF739F8019B3BB11299E8
:10D310000B78302B03D02D2212A80AF0B1FD0D9B03
:10D320008BB1F7B19DF80C100CA80AF02BFDD4E9D5
:10D3300002010CAA11F0D5FC28B9D8F8003043F04E
:10D340000403C8F800301FB1E36AB3427FF46AAE49
:10D35000289812A90AF06EFE6AE6BAF1000FBFD152
:10D3600060E6F1B2E0E700BF280000202DE9F041BF
:10D3700092B008AC84E80C00DDE91B380EAA8C469C
:10D380009DF868100C920CAF00220293CDE9038740
:10D3900006460D928DF8382006AD18AB11B393E810
:10D3A00003008DE80300614694E80C002846FFF76F
:10D3B000F9FB95E803000C9D84E80300F8F75AFF99
:10D3C0001D990B900BAB4246284611F0F7F994E8F3
:10D3D000030086E8030038460AF0AEFB304612B080
:10D3E000BDE8F08193E803008DE80300614694E80E
:10D3F0000C002846FFF7C8FDDBE72DE9F04F91B0A0
:10D4000008ACDDF874B09DF870A006460BF16C0016
:10D4100084E80C00884605F0B9F81E9BCDE902B3FC
:10D420000AAF04971AAB814693E803008DE8030026
:10D430000CAA0A9206AD00220B928DF830204146CC
:10D4400094E80C002846BAF1000F1DD0FFF7AAFBA4
:10D4500095E803000B9D84E8030055B11F98294609
:10D460000AF009FD0A991F9B4A191B684846FEF7F6
:10D4700045F894E8030086E8030038460AF05CFBB0
:10D48000304611B0BDE8F08FFFF77EFDE0E7000009
:10D4900073B5044616460D4619B912B10D4804F08D
:10D4A00091F9731B0F2B019307D9002201A9204684
:10D4B0000AF020FB019B2060A360324629462068C9
:10D4C0000AF0B0FB019B226863600021D15402B0D6
:10D4D00070BD00BFE49002082DE9F0438DB01C46FA
:10D4E000804602AB68460093FFF7D2FF08AB149A60
:10D4F0000693214606A8FFF7CBFFDDE90097DDE99B
:10D5000006564F442E442A464946404611F001FB38
:10D51000044670B94846F2F7B5FE81442846F2F752
:10D52000B1FE4F4505EB00040DD1341B18BF4FF081
:10D53000FF3406A80AF000FB68460AF0FDFA204610
:10D540000DB0BDE8F083A64203D009F10109651CC6
:10D55000D9E70124EDE72DE9F0431C4600F108036B
:10D5600087B015460360002343600372224602AB76
:10D5700006468846684629460093FFF789FF621BE6
:10D58000DDE900735400204607EB030910F038FE74
:10D59000054623463A462946404611F0C5FA8442DC
:10D5A0000DD8441C284610F02DFD204610F028FE12
:10D5B0002346054601463A46404611F0B5FA024672
:10D5C000294630460AF00AFD3846F2F75BFE384439
:10D5D000814505D0471C002130460AF0D3FBD8E72F
:10D5E000284610F00FFD68460AF0A6FA304607B04C
:10D5F000BDE8F083184B1A68D1075CBF01221A609E
:10D60000164B1A68D2075CBF01221A60144B1A68C5
:10D61000D0075CBF01221A60124B1A68D1075CBFA9
:10D6200001221A60104B1A68D2075CBF01221A60EF
:10D630000E4B1A68D0075CBF01221A600C4B1A68A7
:10D64000D1075CBF01221A600A4B1A68D2075CBF7F
:10D6500001221A60704700BF4C1B0020481B0020AD
:10D66000441B0020401B00203C1B0020381B0020D6
:10D67000341B0020301B00200AF05EBA10F0EAB91B
:10D68000F8B54D680746681C0E4610F0B9FD00233A
:10D69000044601462A4630460AF0B0FC0023635592
:10D6A0003C602846F8BDF8B54D686FF060426B1CD1
:10D6B0009342074634BF98004FF0FF300E4610F0FB
:10D6C0009FFD0023044601462A46304610F00EFC1A
:10D6D000002344F825303C602846F8BD13B5049C6F
:10D6E000CDE9003413460A46C1684FF00000FBF74D
:10D6F000A3FB02B010BD30B58BB00D460AA901E9FD
:10D700000C0079230693129B0593119B0493109BA5
:10D7100003930EAA044692E8030001AB83E80300DA
:10D72000099B00932046089BAA684FF00001FBF775
:10D7300023FD20460BB030BD30B58BB00D460AA995
:10D7400001E90C006D230693129B0593119B049332
:10D75000109B03930EAA044692E8030001AB83E8F2
:10D760000300099B00932046089BAA684FF0000124
:10D77000FBF702FD20460BB030BD30B58BB00D4637
:10D780000AA901E90C0077230693129B0593119BCC
:10D790000493109B03930EAA044692E8030001AB86
:10D7A00083E80300099B00932046089BAA684FF07A
:10D7B0000001FBF7E1FC20460BB030BD30B58BB06B
:10D7C0000D460AA901E90C0064230693129B0593F8
:10D7D000119B0493109B03930EAA044692E8030046
:10D7E00001AB83E80300099B00932046089BAA68CD
:10D7F0004FF00001FBF7C0FC20460BB030BD30B548
:10D800008BB00D460AA901E90C0074230693129B04
:10D810000593119B0493109B03930EAA044692E870
:10D82000030001AB83E80300099B00932046089B9B
:10D83000AA684FF00001FBF79FFC20460BB030BDFB
:10D8400081684FF00000FBF791BCF0B591B00AACD5
:10D8500084E80C00002307930D930EAB06930DABE9
:10D860000593199B04939DF86030039316AA0F4605
:10D87000054692E8030001AB83E803000B9B00938D
:10D8800008AE0A9BBA684FF000013046FCF796F8E4
:10D8900096E803000D9B84E803005BB9DDE90E0107
:10D8A0001B9BC3E9000194E8030085E803002846B8
:10D8B00011B0F0BD1A9A1360F5E710B588B00DF1FC
:10D8C000200C0CE90C00002304939DF830300393E6
:10D8D0000B9B02939DF828300193079B00931346FE
:10D8E0008A684FF000010446FBF780FF204608B02D
:10D8F00010BD0A4601694FF00000FBF72FBC07B5C9
:10D900000092D1E9002301694FF00000FBF7FEFB14
:10D9100003B05DF804FB13B5049CCDE90034134655
:10D920000A46C1684FF00000FBF791FA02B010BD43
:10D9300030B58BB00D460AA901E90C007923069396
:10D94000129B0593119B0493109B03930EAA04460C
:10D9500092E8030001AB83E80300099B0093204693
:10D96000089BAA684FF00001FBF760FC20460BB053
:10D9700030BD30B58BB00D460AA901E90C006D230E
:10D980000693129B0593119B0493109B03930EAA7D
:10D99000044692E8030001AB83E80300099B00936F
:10D9A0002046089BAA684FF00001FBF73FFC204689
:10D9B0000BB030BD30B58BB00D460AA901E90C00A3
:10D9C00077230693129B0593119B0493109B03935B
:10D9D0000EAA044692E8030001AB83E80300099B0A
:10D9E00000932046089BAA684FF00001FBF71EFC3D
:10D9F00020460BB030BD30B58BB00D460AA901E909
:10DA00000C0064230693129B0593119B0493109BB7
:10DA100003930EAA044692E8030001AB83E80300D7
:10DA2000099B00932046089BAA684FF00001FBF772
:10DA3000FDFB20460BB030BD30B58BB00D460AA9BA
:10DA400001E90C0074230693129B0593119B049328
:10DA5000109B03930EAA044692E8030001AB83E8EF
:10DA60000300099B00932046089BAA684FF0000121
:10DA7000FBF7DCFB20460BB030BD81684FF00000A7
:10DA8000FBF777BBF0B591B00AAC84E80C0000233B
:10DA900007930D930EAB06930DAB0593199B04935F
:10DAA0009DF86030039316AA0F46054692E80300DE
:10DAB00001AB83E803000B9B009308AE0A9BBA6896
:10DAC0004FF000013046FCF7F1F896E803000D9B9B
:10DAD00084E803005BB9DDE90E011B9BC3E900018B
:10DAE00094E8030085E80300284611B0F0BD1A9AB7
:10DAF0001360F5E710B588B00DF1200C0CE90C00AF
:10DB0000002304930C9B03930B9B02939DF82830F6
:10DB10000193079B009313468A684FF00001044667
:10DB2000FBF7DEFF204608B010BD0A4601694FF042
:10DB30000000FBF717BB07B50092D1E9002301698C
:10DB40004FF00000FBF7F6FA03B05DF804FB0000AD
:10DB500073B5044616460D4619B912B10D4803F0C7
:10DB600031FE731B9A100C2B019207D9002201A9D8
:10DB700020460FF04BFF019B2060A36020683246D7
:10DB800029460FF0DEFF019920460FF039FF02B061
:10DB900070BD00BFE490020873B5044616460D46FA
:10DBA00019B912B10D4803F00DFE731B0F2B019331
:10DBB00007D9002201A9204609F09CFF019B2060A3
:10DBC000A3603246294620680AF02CF8019B22689F
:10DBD00063600021D15402B070BD00BFE490020820
:10DBE00010B5074B0360036900220446DA600C306D
:10DBF000FAF7F7FE2046F9F795FC204610BD00BF66
:10DC00006C9A020810B50446FFF7EAFF204610F0B0
:10DC1000F7F9204610BD000010B5084B03600369FA
:10DC200000220446DA609A611A629A620C30FAF7AE
:10DC3000D8FE2046F9F710F9204610BDA09B020837
:10DC400010B50446FFF7E8FF204610F0D9F920464A
:10DC500010BD000010B5084B0360036900220446A4
:10DC6000DA609A611A629A620C30FAF7BAFE2046BC
:10DC7000F9F70CF9204610BD6C9B020810B504465C
:10DC8000FFF7E8FF204610F0BBF9204610BD00006A
:10DC900010B5054B044640F8103BFAF7A2FE2046AB
:10DCA000FDF7F4FA204610BD349A020810B5044678
:10DCB000FFF7EEFF204610F0A3F9204610BD00004C
:10DCC00010B5074B0360036900220446DA600C308C
:10DCD000FAF787FE2046F9F78DFC204610BD00BFFD
:10DCE000909A020810B50446FFF7EAFF204610F0AC
:10DCF00087F9204610BD000010B5084B036003698A
:10DD000000220446DA601A629A621A630C30FAF74B
:10DD100068FE2046F9F764F9204610BD089C020809
:10DD200010B50446FFF7E8FF204610F069F92046D9
:10DD300010BD000010B5084B0360036900220446C3
:10DD4000DA601A629A621A630C30FAF74AFE2046C9
:10DD5000F9F760F9204610BDD49B020810B50446BF
:10DD6000FFF7E8FF204610F04BF9204610BD0000F9
:10DD700010B5054B044640F8103BFAF732FE20463A
:10DD800001F03AFA204610BD509A020810B5044638
:10DD9000FFF7EEFF204610F033F9204610BD0000DB
:10DDA00010B5054B044640F80C3BFAF71AFE204626
:10DDB000FDF784FA204610BDFC99020810B5044610
:10DDC000FFF7EEFF204610F01BF9204610BD0000C3
:10DDD00010B5054B044640F8083BFAF702FE204612
:10DDE000FDF718FA204610BD0C9B020810B504463A
:10DDF000FFF7EEFF204610F003F9204610BD0000AB
:10DE000010B5054B044640F8083BFAF7EAFD2046FA
:10DE1000FDF714FA204610BD3C9B020810B50446DD
:10DE2000FFF7EEFF204610F0EBF8204610BD000093
:10DE300010B5054B044640F80C3BFAF7D2FD2046DE
:10DE400001F0F2F9204610BD189A020810B50446F8
:10DE5000FFF7EEFF204610F0D3F8204610BD00007B
:10DE600010B5054B044640F8083BFAF7BAFD2046CA
:10DE700001F086F9204610BD249B020810B5044627
:10DE8000FFF7EEFF204610F0BBF8204610BD000063
:10DE900010B5054B044640F8083BFAF7A2FD2046B2
:10DEA00001F082F9204610BD549B020810B50446CB
:10DEB000FFF7EEFF204610F0A3F8204610BD00004B
:10DEC00010B5054B044640F8083BFAF78AFD20469A
:10DED000FDF7C8F9204610BDB49A020810B50446F3
:10DEE000FFF7EEFF204610F08BF8204610BD000033
:10DEF00010B5054B044640F8083BFAF772FD204682
:10DF000001F066F9204610BDE09A020810B50446FB
:10DF1000FFF7EEFF204610F073F8204610BD30B535
:10DF2000084687B014460D46FDF7E1FB84F824004F
:10DF30002846FDF7DFFB0023A3606361E361012353
:10DF400084F8643084F8250029466846FDF7D5FB3F
:10DF5000694604F10800FFF793FBE060684609F0AA
:10DF6000EBFD29466846FDF7CFFB694604F1140036
:10DF7000FFF786FBA061684609F0DEFD294668468A
:10DF8000FDF7C9FB694604F11C00FFF779FB20622D
:10DF9000684609F0D1FD07B030BD30B5084687B0FE
:10DFA00014460D4601F0DCFA6062284601F0DBFA07
:10DFB0000023A3606361E361012384F82431A0623C
:10DFC0002946684601F0D2FA694604F10800FFF7D5
:10DFD00057FBE060684609F0AFFD2946684601F04E
:10DFE000CCFA694604F11400FFF75DFBA0616846B6
:10DFF0000FF030FD2946684601F0C6FA694604F183
:10E000001C00FFF750FB206268460FF023FD07B0AD
:10E0100030BD10B4084611461A46DDE901340194BA
:10E020005DF8044BFDF730BC10B4084611461A46A3
:10E03000DDE9013401945DF8044B01F05DBB30B5BE
:10E04000084687B014460D46FDF7B6FA60742846B8
:10E05000FDF7B5FAA0742846FDF7D0FA0023A360B7
:10E060006361E3616362012384F84330E06229461F
:10E070006846FDF7A7FA694604F10800FFF700FBC0
:10E08000E060684609F058FD29466846FDF7A1FAA8
:10E09000694604F11400FFF7F3FAA061684609F03D
:10E0A0004BFD29466846FDF79BFA694604F11C00C2
:10E0B000FFF7E6FA2062684609F03EFD2946684609
:10E0C000FDF795FA694604F12400FFF7D9FAA0623A
:10E0D000684609F031FD2846FDF793FA206328468B
:10E0E000FDF794FA606307B030BD30B5084687B0DD
:10E0F00014460D46FDF731FA60742846FDF730FAF4
:10E10000A0742846FDF74BFA0023A3606361E36126
:10E110006362012384F84330E06229466846FDF7D4
:10E1200022FA694604F10800FFF7AAFAE06068469F
:10E1300009F002FD29466846FDF71CFA694604F11C
:10E140001400FFF79DFAA061684609F0F5FC294626
:10E150006846FDF716FA694604F11C00FFF790FACD
:10E160002062684609F0E8FC29466846FDF710FA87
:10E17000694604F12400FFF783FAA062684609F0BB
:10E18000DBFC2846FDF70EFA20632846FDF70FFA60
:10E19000606307B030BD30B5084687B014460D4601
:10E1A00001F045F96061284601F044F9A061284674
:10E1B00001F05FF90023A360E3616362E36201237E
:10E1C00084F86C3060632946684601F036F9694688
:10E1D00004F10800FFF754FAE060684609F0ACFC6F
:10E1E0002946684601F030F9694604F11C00FFF742
:10E1F0005AFA206268460FF02DFC2946684601F065
:10E200002AF9694604F12400FFF74DFAA062684636
:10E210000FF020FC2946684601F024F9694604F114
:10E220002C00FFF740FA206368460FF013FC2846E5
:10E2300001F022F9A063284601F023F9E06307B05A
:10E2400030BD30B5084687B014460D4601F0C0F821
:10E250006061284601F0BFF8A061284601F0DAF8B5
:10E260000023A360E3616362E362012384F86C30FE
:10E2700060632946684601F0B1F8694604F1080078
:10E28000FFF7FEF9E060684609F056FC294668464B
:10E2900001F0ABF8694604F11C00FFF704FA2062B4
:10E2A00068460FF0D7FB2946684601F0A5F8694695
:10E2B00004F12400FFF7F7F9A06268460FF0CAFBEB
:10E2C0002946684601F09FF8694604F12C00FFF7E3
:10E2D000EAF9206368460FF0BDFB284601F09DF87F
:10E2E000A063284601F09EF8E06307B030BD10B58A
:10E2F00086B00C46114602AA00926846CA18FFF77B
:10E300004BFC089A69462046FDF7ACFA044668467D
:10E3100009F012FC204606B010BD10B586B00C46C0
:10E32000114602AA00926846CA18FFF735FC089AFF
:10E330006946204601F0CEF90446684609F0FCFB28
:10E34000204606B010BD08461146FDF79ABA0846A9
:10E35000114601F0CEB90846FDF7E4B9084601F0D0
:10E360001AB982B0F0B587B005469DF850700D938C
:10E37000742F16461398DDE911210FAC0DAB1ED09A
:10E380000ED8642F2DD0CDE90310029294E803003B
:10E390008DE8030031460CCB2846FDF71AFA1AE047
:10E3A000772F2BD0CDE90310029294E803008DE87B
:10E3B000030031460CCB2846FDF727FA0BE0CDE9E8
:10E3C0000310029294E803008DE8030031460CCB61
:10E3D0002846FDF7AAF9284607B0BDE8F04002B08C
:10E3E0007047CDE90310029294E803008DE8030022
:10E3F00031460CCB2846FDF7B4F9ECE7CDE9031024
:10E40000029294E803008DE8030031460CCB2846C5
:10E41000FDF7C3F9DFE782B0F0B587B005469DF898
:10E4200050700D93742F16461398DDE911210FAC2F
:10E430000DAB1ED00ED8642F2DD0CDE90310029263
:10E4400094E803008DE8030031460CCB284601F028
:10E45000F9F81AE0772F2BD0CDE90310029294E857
:10E4600003008DE8030031460CCB284601F006F985
:10E470000BE0CDE90310029294E803008DE803005D
:10E4800031460CCB284601F089F8284607B0BDE894
:10E49000F04002B07047CDE90310029294E8030007
:10E4A0008DE8030031460CCB284601F093F8ECE7E9
:10E4B000CDE90310029294E803008DE80300314691
:10E4C0000CCB284601F0A2F8DFE70000F8B5AF4A10
:10E4D0000C466FF00103AE4905460FF095FD064668
:10E4E00010B104682046F8BDAA4B9C4229D168208F
:10E4F000F7F759FCA84B46600746C0E90266C0E939
:10E500000566C0E9076603600674868480F8646067
:10E510001420F7F748FCA14B466003608760314642
:10E520000446F8F7B1FF6B68E56001336B609C4B04
:10E53000236027613A4629464FF00000FAF704FCB1
:10E54000D0E7984B9C4210D11020F7F72CFC964B4B
:10E55000036046600446F7F78DFE6B68C4E9020568
:10E5600001336B60914B2360BCE7914B9C420AD115
:10E570000C20F7F718FC6B6801336B60C0E901658C
:10E580008C4B0446EFE78C4B9C420AD10C20F7F7EA
:10E590000AFC6B6801336B60C0E90165874B044678
:10E5A000E1E7874B9C420AD10C20F7F7FCFB6B6834
:10E5B00001336B60C0E90165824B0446D3E7824BAF
:10E5C0009C422FD14420F7F7EEFB804B0682074692
:10E5D000C0E90036C0E90266C0E90566C0E9076621
:10E5E000C0E90966C0E90B668674466380F843603B
:10E5F0001420F7F7D8FB764B4660036087603246FD
:10E6000031460446F8F7A0FB6B68E56001336B60A8
:10E61000704B236027613A4629464FF00000FAF715
:10E6200021FC5FE76C4B9C422FD14420F7F7BBFBEA
:10E630006A4B06820746C0E90036C0E90266C0E9B7
:10E640000566C0E90766C0E90966C0E90B6686741D
:10E65000466380F843601420F7F7A5FB604B4660E3
:10E6600003608760324631460446F8F7B1FB6B68B9
:10E67000E56001336B605B4B236027613A462946B6
:10E680004FF00000FAF743FC2CE7574B9C420CD1AB
:10E690001420F7F788FB31460446FDF7D3F86B6882
:10E6A000256101336B60514B5DE7514B9C422CD18E
:10E6B0004FF49470F7F777FB00274E4B4760064600
:10E6C000C0E90277C0E90577C0E90777C0E90977B3
:10E6D0000360077480F824711420F7F764FB464B3D
:10E6E00047600360866039460446F8F735FF6B687B
:10E6F000E56001336B60414B236026613246294659
:10E700004FF00000FAF75DFBECE63D4B9C4210D168
:10E710001020F7F748FB002343603A4B03600446A0
:10E72000F7F7A8FD6B6801336B60C4E90205364B4F
:10E7300019E7364B9C420BD10C20F7F734FB002332
:10E74000C0E901356B6801336B600446304B0AE762
:10E75000304B9C420BD10C20F7F725FB0023C0E97E
:10E7600001356B6801336B6004462B4BFBE62B4B8A
:10E770009C4257D10C20F7F716FB0023C0E9013566
:10E780006B6801336B600446254BECE60487020896
:10E79000088202085C1B00202C830208809102087A
:10E7A0006C9A0208501B002064910208FC99020830
:10E7B000581B0020B49A0208641B00200C9B02081E
:10E7C000601B00203C9B0208681B0020B4820208EA
:10E7D000A4910208A09B02086C1B0020C4820208BE
:10E7E000D89102086C9B0208541B0020349A02083E
:10E7F0009C1B00203C830208589C0208909A020847
:10E80000901B00203C9C0208189A0208981B0020CC
:10E81000E09A0208A41B0020249B0208A01B0020F1
:10E82000549B02083E4B9C4231D17020F7F7BBFA53
:10E8300000273C4B47600646C0E90277C0E90577F0
:10E84000C0E90777C0E90977C0E90B77C0E90D7720
:10E8500003600774C76380F86C701420F7F7A3FA9D
:10E86000314B4760036086603A4639460446F8F704
:10E8700027FB6B68E56001336B602C4B23602661DE
:10E88000324629464FF00000FAF796FB2AE6284B5D
:10E890009C4231D17020F7F786FA0027254B47605C
:10E8A0000646C0E90277C0E90577C0E90777C0E905
:10E8B0000977C0E90B77C0E90D7703600774C76378
:10E8C00080F86C701420F7F76EFA1B4B47600360FA
:10E8D00086603A4639460446F8F73AFB6B68E560CD
:10E8E00001336B60154B23602661324629464FF099
:10E8F0000000FAF7B6FBF5E5114B9C420CD1142051
:10E90000F7F751FA0021044600F0D4FE6B68256148
:10E9100001336B600B4B26E60B4802F053FF00BF40
:10E92000A81B0020D48202087C9C0208089C0208D4
:10E93000AC1B0020E4820208B09C0208D49B0208B1
:10E94000941B0020509A0208A08602088B6910B51B
:10E95000044613B9064802F035FFD1E9003200F150
:10E96000080101601A441946FFF716F9204610BD48
:10E97000CD86020882B02DE9F0478AB00446189986
:10E980009DF85480DDF858909DF85CA013931546CF
:10E9900013AEB1B104AF3846FFF7D8FFCDE902A7F7
:10E9A000CDE90089204696E80C002946FCF787FE51
:10E9B000384609F0C1F820460AB0BDE8F04702B079
:10E9C0007047CDE9019ACDF8008096E80C00294601
:10E9D000FCF75FFEEFE710B58AB004460093002015
:10E9E0001346C968099003AAFAF7B6FF03A920469F
:10E9F000FFF7ACFF03A8FAF7A0F920460AB010BD54
:10EA0000F0B59BB00AAC84E80C0013AE0023CDE94E
:10EA1000063619930C930CAB0593239B04939DF836
:10EA20008830039320AA8C46054692E8030001AB88
:10EA300083E803000B9B009308AF0A9BDCF80820D7
:10EA40004FF000013846FAF7B9FF97E803000C9B36
:10EA500084E80300A3B931460DA8FFF777FF259896
:10EA60000DA909F035F90DA809F066F894E803003E
:10EA700085E803003046FAF760F928461BB0F0BD80
:10EA8000249A1360F2E730B58DB004461198002542
:10EA90000B9545680395006802901098CDE9003009
:10EAA0001346096905AA4FF00000FAF765FF05A9AA
:10EAB0002046FFF74BFF05A8FAF73FF920460DB0B7
:10EAC00030BD0000836973B504460D4603B1984715
:10EAD00004F108032360D5E90063F5181EB915B1E8
:10EAE0000E4802F06FFE0F2B019307D9002201A9F7
:10EAF000204608F0FFFF019B2060A36020682A46A3
:10EB0000314609F08AF8019B226863600021D154E4
:10EB1000034BA361204602B070BD00BFE490020821
:10EB200079D6000810B586B0144668461A46089B88
:10EB3000FCF7B1FE69462046FFF7C4FF684608F0BF
:10EB4000FBFF06B010BD82B02DE9F0438FB0164632
:10EB50001E9A179305469DF86C10DDE91C0819AB49
:10EB600017AC9AB1CDE90482CDE9021093E8030015
:10EB70008DE80300314694E80C002846FCF74BFD75
:10EB800028460FB0BDE8F04302B0704708AFCDE9AA
:10EB90000487CDE9021093E803008DE803000DF12E
:10EBA000280C0DF11809CDE908C28DF8282031464E
:10EBB00094E80C004846FCF74DFD99E80300D8F8AE
:10EBC000003084E803001BB91F983946FFF77AFF2D
:10EBD00094E8030085E80300384608F0ADFFCFE76E
:10EBE00070B590B009AD0E4606A981E80C00044648
:10EBF0001799002328460F93FFF764FF9DF85830BC
:10EC00000393159B02939DF850300193079BB268C4
:10EC100000939FED070B069B04954FF000012046E3
:10EC2000FAF7E4FD2846FAF788F8204610B070BDE0
:10EC30000000000000000000F0B58FB00E46154641
:10EC40001699179A02AC1F460A4404AB2046029359
:10EC5000FEF7A2FF159B00933A46149B01943146A0
:10EC600008A8FCF702FE08A92846FFF72BFF08A812
:10EC700008F062FF204608F05FFF0FB0F0BD000013
:10EC80008B6910B5044613B9074802F09BFDD1E922
:10EC9000003200F10801016003EB82021946FEF721
:10ECA00057FF204610BD00BFCD86020882B02DE977
:10ECB000F0478AB0DDE9169A18999DF854801393AD
:10ECC0000446154613AEB1B104AF3846FFF7D8FF7E
:10ECD000CDE902A7CDE90089204696E80C00294637
:10ECE00000F027FC38460EF0B5FE20460AB0BDE81D
:10ECF000F04702B07047CDE9019ACDF8008096E860
:10ED00000C00294600F000FCEFE710B58AB004467D
:10ED1000009300201346C968099003AAFAF794FFEC
:10ED200003A92046FFF7ACFF03A8FAF706F8204630
:10ED30000AB010BDF0B59BB00AAC84E80C0013AE6D
:10ED40000023CDE9063619930C930CAB0593239B56
:10ED500004939DF88830039320AA8C46054692E8D8
:10ED6000030001AB83E803000B9B009308AF0A9BF1
:10ED7000DCF808204FF000013846FAF797FF97E8D3
:10ED800003000C9B84E80300A3B931460DA8FFF7EC
:10ED900077FF25980DA90EF017FF0DA80EF05AFE6B
:10EDA00094E8030085E803003046F9F7C6FF2846DB
:10EDB0001BB0F0BD249A1360F2E730B58DB0044665
:10EDC000119800250B9545680395006802901098EE
:10EDD000CDE900301346096905AA4FF00000FAF7A3
:10EDE00043FF05A92046FFF74BFF05A8F9F7A5FF4C
:10EDF00020460DB030BD0000836973B504460D4652
:10EE000003B1984704F108032360D5E90065AB001E
:10EE100006EB85051EB915B10E4802F0D3FC9A1019
:10EE20000C2B019207D9002201A920460EF0EEFD1D
:10EE3000019B2060A36020682A4631460EF07BFECD
:10EE4000204601990EF0DCFD034BA361204602B081
:10EE500070BD00BFE49002087DD6000810B586B0F2
:10EE6000144668461A46089B00F04DFC6946204649
:10EE7000FFF7C2FF68460EF0EDFD06B010BD82B090
:10EE80002DE9F0438FB016461E9A179305469DF85C
:10EE90006C10DDE91C0819AB17AC9AB1CDE90482FE
:10EEA000CDE9021093E803008DE80300314694E8B1
:10EEB0000C00284600F0EAFA28460FB0BDE8F043FF
:10EEC00002B0704708AFCDE90487CDE9021093E89E
:10EED00003008DE803000DF1280C0DF11809CDE9B0
:10EEE00008C20A92314694E80C00484600F0EDFA58
:10EEF00099E80300D8F8003084E803001BB91F9894
:10EF00003946FFF779FF94E8030085E803003846A7
:10EF10000EF0A0FDD0E7000070B590B009AD0E4630
:10EF200006A981E80C0004461799002328460F9390
:10EF3000FFF762FF169B0393159B02939DF85030D9
:10EF40000193079BB26800939FED070B069B049506
:10EF50004FF000012046FAF7C3FD2846F9F7EDFE11
:10EF6000204610B070BD00BF00000000000000008F
:10EF7000F0B58FB00E4615461699179A02AC1F468B
:10EF800001EB820204AB20460293FEF7E1FD159BE4
:10EF900000933A46149B0194314608A800F09DFB6B
:10EFA00008A92846FFF728FF08A80EF053FD2046C1
:10EFB0000EF050FD0FB0F0BD83685869704783684C
:10EFC000986970478368586B704783689B6B002013
:10EFD000DAB262F30700C3F3072262F30F20C3F330
:10EFE000074262F317401B0E82B063F31F6002B04A
:10EFF00070478368DB6B0020DAB262F30700C3F36B
:10F00000072262F30F20C3F3074262F317401B0E7F
:10F0100082B063F31F6002B070478368586970471D
:10F020008368986970478368586B704783689B6BE7
:10F030000020DAB262F30700C3F3072262F30F2065
:10F04000C3F3074262F317401B0E82B063F31F60E5
:10F0500002B070478368DB6B0020DAB262F307000E
:10F06000C3F3072262F30F20C3F3074262F3174092
:10F070001B0E82B063F31F6002B070478368586A4A
:10F0800070478368986A7047002070470020704777
:10F0900070470020914204D251F8043B03EB7060AA
:10F0A000F8E7704713B58B6801AA9968044609F020
:10F0B00095F8204602B010BD13B58B6801AA996877
:10F0C000044609F08BF8204602B010BD13B58B68DA
:10F0D00001AA9968044609F081F8204602B010BDE3
:10F0E00013B58B6801AAD96904460EF073FF204658
:10F0F00002B010BD13B58B6801AA596A04460EF020
:10F1000069FF204602B010BD13B58B6801AAD96A09
:10F1100004460EF05FFF204602B010BD13B58B68A9
:10F1200001AAD96904460EF055FF204602B010BD71
:10F1300013B58B6801AA596A04460EF04BFF2046AE
:10F1400002B010BD13B58B6801AAD96A04460EF04F
:10F1500041FF204602B010BD13B58B6801AA596962
:10F1600004460EF037FF204602B010BD13B58B6881
:10F1700001AAD96904460EF02DFF204602B010BD49
:10F1800010B5034B03600446F7F752F8204610BD54
:10F19000009D020810B50446FFF7F2FF20460EF06E
:10F1A0002FFF204610BD000010B5034B036004463E
:10F1B000F7F73EF8204610BD189D020810B504462A
:10F1C000FFF7F2FF20460EF01BFF204610BD0000A7
:10F1D00010B5034B03600446F7F72AF8204610BD2C
:10F1E000309D020810B50446FFF7F2FF20460EF0EE
:10F1F00007FF204610BD000010B5054B044640F83F
:10F20000083B0FF043FB2046F7F712F8204610BDED
:10F21000E49C020810B50446FFF7EEFF20460EF00E
:10F22000EFFE204610BD000010B5054B044640F827
:10F23000083B0FF02BFB2046F6F7FAFF204610BDE7
:10F240003C9C020810B50446FFF7EEFF20460EF086
:10F25000D7FE204610BDD0E902218A4202D20432F4
:10F260008260704703689B6A184707B500920B4697
:10F27000002241680EF022FD03B05DF804FB00009F
:10F280002DE9F04107461648F7F770F83B68D3F8C8
:10F290000C8058F820500646F5B97020F6F783FD2B
:10F2A000104B45600446C0E90255C0E90555C0E968
:10F2B0000755C0E90955C0E90B55C0E90D55036074
:10F2C0000574C56380F86C50394609F011FF386841
:10F2D00032462146F7F710F958F82600BDE8F081CC
:10F2E000AC1B0020E482020838B543689942054609
:10F2F00004D90A460A480B4902F06AFAB2F1FF3F04
:10F3000004D10368696000225A5438BD002AFCD039
:10F310005B1A9A4228BF1A46BDE8384008F0C3BCC1
:10F32000B08E0208128F020810B504460068FFF77D
:10F3300092FF4FF0FF33636010BD00002DE9F041F4
:10F3400007461648F7F712F83B68D3F80C8058F8D0
:10F3500020500646F5B97020F6F725FD104B4560A4
:10F360000446C0E90255C0E90555C0E90755C0E9A2
:10F370000955C0E90B55C0E90D5503600574C56317
:10F3800080F86C50394609F07BFF386832462146D8
:10F39000F7F7B2F858F82600BDE8F081A81B002066
:10F3A000D482020837B54568A94205D90A460648FD
:10F3B00006492B4602F00CFA0093134600220EF089
:10F3C0007DFC03B030BD00BFB08E0208AF900208D4
:10F3D00003689B6818470368DB68184710B50B681B
:10F3E00004461B699847204610BD10B50B680446BB
:10F3F0005B699847204610BD10B50B6804469B69B1
:10F400009847204610BD10B50B680446DB69984745
:10F41000204610BD03681B6A184703685B6A82B008
:10F4200002B0184703689B6A82B002B018470368AD
:10F430009B6818470368DB68184710B50B680446DB
:10F440001B699847204610BD10B50B6804465B69E0
:10F450009847204610BD10B50B6804469B69984735
:10F46000204610BD10B50B680446DB69984720465E
:10F4700010BD03681B6A184703685B6A82B002B05C
:10F48000184703689B6A82B002B01847F0B589B08C
:10F4900006AE86E80C00139A0B680592129A049245
:10F4A000119A03929DF8402002920EAA04460D463E
:10F4B00092E803008DE8030020469F68294696E8FD
:10F4C0000C00B847204609B0F0BDF0B589B006AED3
:10F4D00086E80C00139A0B680592129A0492119A0E
:10F4E00003929DF8402002920EAA04460D4692E82F
:10F4F00003008DE803002046DF68294696E80C00EB
:10F50000B847204609B0F0BD70B586B004AC84E8B9
:10F510000C000C9A02920B9A01920B689DF828201D
:10F5200000929E6894E80C000546B047284606B055
:10F5300070BD70B586B004AC84E80C000D9A0392DF
:10F540000C9A02920B9A01920B689DF82820009267
:10F55000DE6894E80C000546B047284606B070BD4A
:10F5600003689B6818470368DB68184710B50B6889
:10F5700004461B699847204610BD10B50B68044629
:10F580005B699847204610BD10B50B6804469B691F
:10F590009847204610BD03689B681847F0B589B0AE
:10F5A00006AE86E80C00129A0B680492119A039238
:10F5B000109A02920EAA04460D4692E803008DE8C6
:10F5C00003002046DF68294696E80C00B84720462D
:10F5D00009B0F0BDF0B589B006AE86E80C00129A0D
:10F5E0000B680492119A0392109A02920EAA044692
:10F5F0000D4692E803008DE8030020461F69294666
:10F6000096E80C00B847204609B0F0BDF0B589B0C7
:10F6100006AE86E80C00129A0B680492119A0392C7
:10F62000109A02920EAA04460D4692E803008DE855
:10F63000030020465F69294696E80C00B84720463B
:10F6400009B0F0BDF0B589B006AE86E80C00129A9C
:10F650000B680492119A0392109A02920EAA044621
:10F660000D4692E803008DE8030020469F69294675
:10F6700096E80C00B847204609B0F0BDF0B589B057
:10F6800006AE86E80C00129A0B680492119A039257
:10F69000109A02920EAA04460D4692E803008DE8E5
:10F6A00003002046DF69294696E80C00B84720464B
:10F6B00009B0F0BD003910B5054B036018BF01213A
:10F6C00041600446F6F7D6FDA060204610BD00BF9D
:10F6D000E49C020803689B68184773B5079E01966F
:10F6E0000D68069E0096ED680446A847204602B0C5
:10F6F00070BD03681B69184710B40468A468A44669
:10F700005DF8044B604738B50D680446ED68A847BE
:10F71000204638BD10B40468E46AA4465DF8044B82
:10F72000604703689B681847F7B56D4685E8060093
:10F730009DF80460089F0446194636B900983A4679
:10F7400008F0D0F9874218BF01268DF8046095E8CB
:10F75000030084E80300204603B0F0BD2DE9F04F1C
:10F7600099B0DDE9228908F16C0406A905902046CC
:10F7700081E80C00249F09F081FA06462046FFF735
:10F78000DDFD3D68036C2A689A4204467B6843D0DD
:10F79000826B0992D0F828A0426A03923268304600
:10F7A000576905EB83032A460421B847401B86109E
:10F7B00000F0C0800EAB4FF0000B71000CA80C9352
:10F7C000CDE90DBB0EF027FA636BF71A5F4531DD0B
:10F7D000E1680D9A5B45B8BF3746002965D07B00CC
:10F7E0005946CDF800B00CA80EF068FA05EB870377
:10F7F000CDE900530C98A169D4E9022309F06AFB12
:10F800000C9BC01A0D9BB3EBA00F4FEAA0020DD2C8
:10F810006049614801F0DCFFC26B0992C26AD0F80E
:10F8200030A00392002BB9D00435B7E711460CA8DD
:10F830000EF0E6F8636B002B0BDD61690CA80EF08F
:10F840001CFA002F37DB626B05EB87010CA80EF06A
:10F850003DFBD8F80C5005F0B003049315F4007587
:10F860000D9B18BF256A0AEB0302154414AB002652
:10F87000690012A81293CDE913660EF0CCF9049B2F
:10F88000D8F80870102B03D1BD422CBF00260126EA
:10F890004FF0000B7D1B09AB13F80B30042B1BD86A
:10F8A000DFE803F06C6311545D0000972B460CA851
:10F8B0000EF060FABEE7626C79420CA8FFF7D5FC47
:10F8C00032462946C2E7D8F80C309B0504D5D4E966
:10F8D000071212A80EF0FAFA0BF1010BBBF1040F9C
:10F8E000D9D1BAF1010F06D903990AF1FF320431D7
:10F8F00012A80EF0EBFA13998F4249D9049B202BE2
:10F90000A7EB01013DD14A4612A8FFF7AEFC0AACB5
:10F91000DDE90612129B00972046FFF705FF94E8E9
:10F920000300069012A88DF81C100EF093F80CA896
:10F930000EF090F8DDE906010023C8F80830059BB9
:10F9400083E80300184619B0BDE8F08FBAF1000F44
:10F95000C2D0039B196812A80EF08FF9BCE7DDE94D
:10F960000C1212A80EF08EFAB6E72EB14A462946BE
:10F9700012A8FFF77AFCAFE74946ECE7002EABD0C0
:10F98000F4E70A464B46002112A8FFF70BFDBEE73D
:10F990000F46BCE7128F0208B08E02082DE9F04F27
:10F9A00099B0DDE9228908F16C0406A9059020468A
:10F9B00081E80C00249F09F061F906462046FFF714
:10F9C0005FFC3D68036C2A689A4204467B6843D01A
:10F9D000826B0992D0F828A0426A039232683046BE
:10F9E000576905EB83032A460421B847401B86105C
:10F9F00000F0C0800EAB4FF0000B71000CA80C9310
:10FA0000CDE90DBB0EF007F9636BF71A5F4531DDE9
:10FA1000E1680D9A5B45B8BF3746002965D07B0089
:10FA20005946CDF800B00CA80EF048F905EB870355
:10FA3000CDE900530C98A169D4E9022309F04AFAF0
:10FA40000C9BC01A0D9BB3EBA00F4FEAA0020DD286
:10FA50006049614801F0BCFEC26B0992C26AD0F8ED
:10FA600030A00392002BB9D00435B7E711460CA89B
:10FA70000DF0C6FF636B002B0BDD61690CA80EF067
:10FA8000FCF8002F37DB626B05EB87010CA80EF04A
:10FA90001DFAD8F80C5005F0B003049315F4007566
:10FAA0000D9B18BF256A0AEB0302154414AB002610
:10FAB000690012A81293CDE913660EF0ACF8049B0E
:10FAC000D8F80870102B03D1BD422CBF00260126A8
:10FAD0004FF0000B7D1B09AB13F80B30042B1BD828
:10FAE000DFE803F06C6311545D0000972B460CA80F
:10FAF0000EF040F9BEE7626C79420CA8FFF7B5FB47
:10FB000032462946C2E7D8F80C309B0504D5D4E923
:10FB1000071212A80EF0DAF90BF1010BBBF1040F7A
:10FB2000D9D1BAF1010F06D903990AF1FF32043194
:10FB300012A80EF0CBF913998F4249D9049B202BC0
:10FB4000A7EB01013DD14A4612A8FFF78EFB0AAC94
:10FB5000DDE90612129B00972046FFF7E5FD94E8C9
:10FB60000300069012A88DF81C100DF073FF0CA86E
:10FB70000DF070FFDDE906010023C8F80830059B91
:10FB800083E80300184619B0BDE8F08FBAF1000F02
:10FB9000C2D0039B196812A80EF06FF8BCE7DDE92C
:10FBA0000C1212A80EF06EF9B6E72EB14A4629469D
:10FBB00012A8FFF75AFBAFE74946ECE7002EABD09F
:10FBC000F4E70A464B46002112A8FFF7EBFBBEE71D
:10FBD0000F46BCE7128F0208B08E02082DE9F04FE5
:10FBE0002DED028BB0EE408AF0EE608A91B004AF4A
:10FBF00007F1080484E80C007B6E97F860B00546B6
:10FC0000884607F1140003F16C01F6F71BFB07F1BE
:10FC1000140009F033F890B08146F6F72BFB04AEE0
:10FC20004FF0000AB86131468DED028B294BCDF8BB
:10FC300000A0402207F11800FBF714FC3F28014602
:10FC400016DD083121F00701ADEB010D421C7A6091
:10FC5000F6F710FB04AEB86131468DED028B1D4BFB
:10FC60007A68CDF800A007F11800FBF7FBFB01460E
:10FC700007F12003002207F11800BB6179600DF045
:10FC800041FF7968BB69721848463146FFF742FD6B
:10FC900007F118030293BB6E01937B6E00934146FC
:10FCA00094E80C002846BBF1000F10D0FFF756FD7A
:10FCB00007F118000DF0CEFE07F11400F6F730FB47
:10FCC00028463437BD46BDEC028BBDE8F08FFFF708
:10FCD00065FEEDE7C6900208F0B587B004AC84E895
:10FCE0000C00DDE90D320F9E9DF830700093CDE9D8
:10FCF0000126054694E80C0027B1FFF72FFD2846A2
:10FD000007B0F0BDFFF74AFEF9E703681B6B184721
:10FD100003689B69184703689B6A184710B5044637
:10FD2000D0E9003043B1421C06D1184607F0D1FE9D
:10FD3000431C04BF0023236010BD38B50D46FFF7F8
:10FD4000EDFF04462846FFF7E9FF431C584204F143
:10FD50000102584154425441011B4842484138BDB8
:10FD600008B5FFF7EAFF80F00100C0B208BD2DE939
:10FD7000F74F0546DDE9120602A96C30DDF8449024
:10FD800001E90C0008F07AFFB9F1020F82462FD08A
:10FD9000B9F1040F0CBF4FF47A7701270024A04675
:10FDA0004FF00A0B0CA96846FFF7DAFF10B3C845FD
:10FDB00022D06846FFF7B2FF2A2201465046FFF7DD
:10FDC000A4FF3038C2B2092A21D8109B0BFB0404CF
:10FDD00004FB07F29A421ADC0F9B3A449A4216DD62
:10FDE000B7FBFBF76846FFF79FFA08F10108D9E770
:10FDF0000A27D3E7C8450AD10E9B1C6002AB13E962
:10FE0000030085E80300284603B0BDE8F08FB9F190
:10FE1000040F04D1B8F1020F01D1643CECE7336860
:10FE200043F004033360E9E72DE9F04F85B000AFFC
:10FE30008046F86CD7F8449007F108046C3084E8E9
:10FE40000C0008F01BFFBB6C9B00073323F007037B
:10FE50008246ADEB030D07F1380120466E46FFF7F1
:10FE60007FFF00287FD02046FFF758FF4FF0000BA0
:10FE700002465D46BB6C9B4512D059F82B100968B1
:10FE8000914205D146F825B001350BF1010BF1E7A0
:10FE900050467A60FFF73CFF7A689042F5D1F1E76F
:10FEA0004FF0000A012D40D9336859F8230013F0B0
:10FEB0008DFF0122834656F822107A6059F82100FE
:10FEC00013F084FF7A68834502F1010228BF83465C
:10FED0009542F0D120460AF1010AFFF725FADA45EA
:10FEE00041D207F138012046FFF73AFF00283AD007
:10FEF0004FEA8A024FF0000B56F82B1059F82110E8
:10FF000089582046C7E90021FFF708FF79683A6859
:10FF1000814217BF05F1FF350BF1010B56F8251093
:10FF200046F82B105D45E7D8BCE71CD12046FFF70B
:10FF3000FBF9366859F82690484613F047FF0AF156
:10FF4000010A0546AA451DD207F138012046FFF7F0
:10FF500007FF40B159F82A307B602046FFF7DEFEEC
:10FF60007B68834212D03B6D3A6D1B6843F00403FB
:10FF7000136094E80300143788E803004046BD4648
:10FF8000BDE8F08FEFD13B6C1E60F2E72046FFF733
:10FF9000CBF90AF1010AD5E72DE9F04F85B000AFA2
:10FFA0008046F86CD7F844A007F108096C3089E85E
:10FFB0000C0008F063FEBB6C6A46A2EBC3038346E9
:10FFC0009D4607F1380148466C46FFF7C9FEB0B3BD
:10FFD0004846FFF7A3FEBA6C00260346520035469A
:10FFE000B24213D05AF826100968994204D144F855
:10FFF000256001350136F3E75846C7E90032FFF7BF
:020000040801F1
:1000000087FE3B687A689842F4D1F0E7BDB1484674
:10001000FFF78AF9AB00073323F00703ADEB030DBD
:10002000E946002654F826305AF8230013F0CEFE95
:1000300049F826000136B542F4D1012502E0002638
:100040003546B14607F1380107F10800FFF788FE91
:1000500070B307F10800FFF761FE002383464FEA03
:10006000850E19469E421BD959F82320AA424FEA11
:10007000830C09EB830002D801310133F2E754F815
:1000800023205AF8222052F80E205A45F5D0013E7E
:1000900054F8262044F80C2059F826200260E1E7A5
:1000A0008E4205D007F10800FFF73EF90135C9E798
:1000B000012E15D1D9F80030AB421AD1BA6C2368A1
:1000C0009342A8BF9B1A3A6C136007F1100313E91F
:1000D0000300143788E803004046BD46BDE8F08FB2
:1000E000022E06D1D9F80030AB42E7D0D9F804305F
:1000F000E2E73B6D3A6D1B6843F00403E4E7000060
:100100002DE9F04F9FB00C46DDF8A8A00B900AF146
:100110006C050EA9284681E80C00DDF8B08008F0D7
:1001200061FE8346284608F0A9FD05462D9813F088
:100130004DFE00260A90109628A90EA8FFF710FE83
:10014000DDF84090002865D00A9B9E4262D2B9F14A
:10015000000F63D12D9B4A4653F82610284603EB27
:100160008607FFF7D2FD252840F0A582731C796829
:1001700009934A462846FFF7C8FD4528CDF8449024
:1001800001D04F2806D1B31CB96809930022284634
:10019000FFF7BBFD41380EAE382800F28782DFE85A
:1001A00010F06A009500D801EE00850285028502F4
:1001B000F400180185028502850247018502850247
:1001C000850285027B019A01C801850285028502AC
:1001D000D301D801020285028502850285028502CB
:1001E0008502440070009B00A100C40085028502C6
:1001F0007000850285028502850223016C0185025B
:100200008502850285028502BE018502850285027E
:10021000CC01D801B9F1000F00F05E822B9B2B9A24
:100220001B6843F0040313605AE212AE314658468D
:1002300008F010FC10ABCDE905A30723CDE903635B
:1002400011AB029328AB93E803008DE803000CAFD9
:100250000EAE96E80C0021463846FFF7E5FD97E81C
:100260000300109B86E8030013B9119BC8F81830EF
:10027000099E013660E712AE3146584608F0DAFBB7
:10028000D8E712AE3146584608F013FC10ABCDE962
:1002900005A30C23CDE9036311AB029328AB93E8CC
:1002A00003008DE803000CAF0EAE96E80C0021466B
:1002B0003846FFF7B9FD97E80300109B86E8030076
:1002C000002BD5D1119BC8F81030D1E712AE3146C2
:1002D000584608F0CFFBD9E7DBF808309B690CAF34
:1002E0000593E2E010ABCDE906A302201F23CDE980
:1002F00004300123039311AB029328AB93E803006E
:100300008DE803000CAF0EAE96E80C00214638468F
:10031000FFF72DFD97E80300109B86E80300002BF4
:10032000A6D1119BC8F80C30A2E73046FFF7F6FCC7
:10033000082102462846FFF7F4F9B0B10E98FEF7FF
:100340008AFF4FF0FF330F9310ABCDE906A30922CC
:100350000123CDE904230CAF039311AB029328AB27
:1003600093E803008DE80300CEE710ABCDE906A3C8
:1003700002211F23CDE904310CAF0A23ECE712AEB2
:10038000C04A3346A2F109018AE010ABCDE906A3C9
:1003900002221723CDE904320CAF0023039311ABE3
:1003A000029328AB93E803008DE803000EAE96E8B5
:1003B0000C0021463846FFF7DAFC97E80300109B53
:1003C00086E80300002B7FF453AF119BC8F8083078
:1003D0004EE710ABCDE906A34FF002090C23CDE99F
:1003E00004390CAF0123D9E710ABCDE906A34FF0D8
:1003F000020E0C23CDE9043E0123039311AB0293BB
:1004000028AB93E803008DE803000CAF0EAE96E82E
:100410000C0021463846FFF7AAFC97E80300109B22
:1004200086E80300002B7FF423AF119B013B4AE7D2
:1004300010ABCDE906A34FF0020C3B23CDE9043C01
:100440000023039311AB029328AB93E803008DE8DC
:1004500003000CAF0EAE96E80C0021463846FFF7BD
:1004600086FC97E80300109B86E80300002B7FF4CE
:10047000FFAE119BC8F80430FAE63046FFF74EFC99
:10048000002201462846FFF740FC0A2840F00E8172
:100490003046FEF749FFEBE67B4A12AE3346911F2A
:1004A0002846FFF737F90CAF059610ABCDE902A34C
:1004B000CDF8108028AB93E803008DE803000EAE62
:1004C0002146384696E80C00FFF71AFE97E803002D
:1004D00086E80300CCE610ABCDE906A302263D2357
:1004E000CDE904360023039311AB029328AB93E8C4
:1004F00003008DE803000CAF0EAE96E80C00214619
:100500003846FFF734FC97E80300109B86E80300A9
:10051000002B7FF4ADAE119BC8F80030A8E6304642
:10052000FFF7FCFB002201462846FFF7EEFB0928F7
:10053000ACE712AE554A334624E712A9584608F0F4
:1005400067FA129B0CAFCBE612A9584608F066FA80
:10055000F7E710ABCDE906A3042042F20F73CDE913
:1005600004300023039311AB029328AB93E80300FC
:100570008DE803000CAF0EAE96E80C00214638461D
:10058000FFF7F5FB97E80300109B86E80300002BBC
:100590007FF46EAE119B002BB4BF6433A3F26C7377
:1005A000C8F8143064E63046FFF7B8FB0121024674
:1005B0002846FFF7B6F8002878D010ABCDE905A3A0
:1005C0000E230493324B039312AB029328AB93E8B0
:1005D00003008DE803000CAF2146384696E80C0076
:1005E000FFF722FC97E8030086E8030028A93046BD
:1005F000FFF7B6FB00283FF43BAE109A129B134363
:100600007FF436AE3046FFF789FB2D21074628469A
:10061000FFF781FBB8423DD110AF17230222CDE98D
:100620000432CDE906A70023039312AB029328AB53
:1006300093E803008DE803000DF130090EAE96E853
:100640000C0021464846FFF792FB99E803003B2344
:1006500086E803000221CDE90431CDE906A7002395
:10066000039312AB029328AB93E803008DE80300D9
:100670002146484696E80C00FFF779FB99E803000D
:1006800026E700BFD5900208DB900208E49002083C
:10069000640000203046FFF741FB2B210646284628
:1006A000FFF739FBB0427FF4E3ADB5E7109B43F0B1
:1006B00004031093DCE52D9B0EA853F82670FFF77A
:1006C0002DFB874203D10EA8FEF72EFED1E5109B2D
:1006D00043F004031093CCE50A9B9E427FF49EAD49
:1006E0000EAB93E803000B9B83E8030018461FB092
:1006F000BDE8F08FF0B58FB00AAC84E80C000DAA0D
:100700000792169A06928C4642F20F720421CDE9A6
:100710000421002303930D930CAB029314AB054605
:1007200093E803008DE8030008AF94E80C006146ED
:100730003846179EFFF71BFB97E803000D9B84E8E4
:100740000300BBB90C9B189A002BB4BF6433A3F20F
:100750006C73536114A92046FFF7EFFA18B13368A0
:1007600043F00203336094E8030085E80300284661
:100770000FB0F0BD336843F004033360EAE72DE9BE
:10078000F0479CB0DDE926960AAC054609F16C00FD
:1007900084E80C00884608F025FB0DF1380A07466E
:1007A000514608F057F9384615A908F043F90023D7
:1007B0000D930DABCDE905930723CDE903A30CAB56
:1007C000029324AB93E803008DE8030008AF94E89C
:1007D0000C0041463846FFF7DFFB97E803000D9B0E
:1007E00084E803009BB9289B0C9A9A6124A92046AF
:1007F000FFF7A3FA18B1336843F00203336094E8BB
:10080000030085E8030028461CB0BDE8F087336884
:1008100043F004033360E9E72DE9F047A6B0DDE9D2
:1008200030960AAC054609F16C0084E80C00884655
:1008300008F0D8FA0DF1380A0746514608F039F9A0
:1008400038461AA908F016F900230D930DABCDE92F
:1008500005930C23CDE903A30CAB02932EAB93E8D5
:1008600003008DE8030008AF94E80C0041463846C9
:10087000FFF792FB97E803000D9B84E803009BB908
:10088000329B0C9A1A612EA92046FFF756FA18B12E
:10089000336843F00203336094E8030085E8030003
:1008A000284626B0BDE8F087336843F00403336080
:1008B000E9E72DE9F0438DB0DDE9169608AC054671
:1008C00009F16C0084E80C00884608F08BFA0AA94C
:1008D00008F0A4F80A9B0593189BCDF80890CDE981
:1008E000036314AB93E803008DE8030006AF4146B1
:1008F000384694E80C00FFF703FC97E8030084E80F
:10090000030014A92046FFF718FA18B1336843F022
:100910000203336094E8030085E8030028460DB025
:10092000BDE8F0832DE9F0438DB0DDE9169608AC03
:10093000054609F16C0084E80C00884608F052FA7C
:100940000AA908F065F80A9B0593189BCDF8089052
:10095000CDE9036314AB93E803008DE8030006AF11
:100960004146384694E80C00FFF7CAFB97E80300BD
:1009700084E8030014A92046FFF7DFF918B13368B3
:1009800043F00203336094E8030085E8030028463F
:100990000DB0BDE8F0832DE9F04F8FB0DDE91A9678
:1009A000054608AC09F16C004FF0000A84E80C0021
:1009B00088469DF874B09DF8787008F05FF9C6F825
:1009C00000A02521FFF7A7F90A904FBBCDE90BB78F
:1009D0000AAB05931C9BCDF80890CDE9036318ABD7
:1009E00093E803008DE8030006AF4146384694E8DB
:1009F0000C00FFF785FB97E8030084E8030018A9C3
:100A00002046FFF79AF918B1336843F002033360C8
:100A100094E8030085E8030028460FB0BDE8F08F96
:100A2000CDE90B7BCDF834A0D2E700002DE9F04FE3
:100A30002DED028B97B006A981E80C00DDE9243882
:100A400003F16C040490204608F018F908EE100A2F
:100A50002046FEF773FC00F140030593836A0446C9
:100A60001BB1036B003B18BF012301930CAB0A932E
:100A700000230B938DF83030237C1BB120210AA872
:100A800007F04EF9002512AB202110A81093119504
:100A90008DF8485007F044F904F1440308EE903A09
:100AA000E36B08932F462E460295A946009508ABA6
:100AB0005B5D042B40D8DFE813F0590128012B00BF
:100AC000A000DA00BBF1000FF1D1D8F8003043F0FC
:100AD0000403C8F8003006AC22A92046FFF72DF920
:100AE00028B1D8F8003043F00203C8F8003094E889
:100AF0000300049B83E8030010A807F01DF80AA870
:100B000007F01AF8049817B0BDEC028BBDE8F08F1F
:100B1000249BDB689A051ED4B9F1010F1BD8D5B10F
:100B2000012D0CD1019BB3B99DF82030032B12D0BD
:100B30009DF82230012B0ED04FF0010B2BE0022D3F
:100B4000FAD19DF82330042B05D0019A002AF3D066
:100B5000032B40F00E81236A03934FF0000A22A971
:100B600006A8FFF7FDF8039B834600283CD09A4572
:100B700011D006A8FFF7D2F8E36953F82A30834270
:100B800035D0BAF1000F40F0F780249BDB6883F486
:100B90000073C3F3402B0135042D93D1B9F1010F3C
:100BA00040F22F81BBF1000F8FD0009B002B00F093
:100BB000E680E56A4FF0010B22A906A8FFF7D0F8FE
:100BC000002800F0DE80D94500F0DE8006A8FFF79F
:100BD000A5F855F82B3083427FF477AF06A8FEF7CF
:100BE000A3FB0BF1010BE7E79A45CAD1A4E706A8DE
:100BF000FEF79AFB0AF1010AB1E7A36AB3B9236BC6
:100C000043B322A906A8FFF7ABF8834610B306A8A2
:100C1000FFF784F8E26A126882421BD106A8D4F872
:100C20003090FEF781FBCDF800B0B4E722A906A80A
:100C3000FFF796F883460028E1D006A8FFF76EF884
:100C4000626A12688242DAD106A8D4F82890FEF7C8
:100C50006BFBA0E7A36A1BB9019B83F0010B9AE72A
:100C6000236B002BF8D1012300939B4693E722A925
:100C700006A8FFF775F88346002843D006A8FFF7BB
:100C80004DF809AA09900A2118EE900AF9F711FC0B
:100C9000A0B1059BA0EB030B5D4B4FEAAB0B1B68B0
:100CA00010A813F80B1007F06DF806F1010B029E67
:100CB00006A8FEF739FB02965E46D8E709996269F5
:100CC0008A4206D12FB9626B002A11DD5F46834646
:100CD000EEE7227C62B1A369994208D177B97EB16F
:100CE000F1B20AA807F04EF8BB46029EE0E7934631
:100CF000119A002A08BF4FF0000B4CE7BB46F7E7FC
:100D0000B346F5E74FF0010BF2E722A906A8FFF77B
:100D100027F8D8B94FF0000B032D3FF43CAF22A9C0
:100D200006A8FFF71DF800283FF435AF06A8FEF728
:100D3000F5FF0821024618EE100AFEF7F2FC002823
:100D40003FF429AF06A8FEF7EFFAE8E706A8FEF79A
:100D5000E5FF0821024618EE100AFEF7E2FC834682
:100D60000028D7D006A8FEF7DFFAD5E74FF0010B31
:100D7000D2E7DDF804B00EE74FF0000B0BE7656A31
:100D800018E7D9457FF4A1AE119B012B11D90022A0
:100D9000302110A807F0BCF9024650B1431C08BF2F
:100DA00011984FF0000108BF00F1FF3210A8FEF7C4
:100DB0009BFA009B3BB110990B78302B03D02D226E
:100DC00010A807F05DF80B9B8BB1F7B19DF80810E8
:100DD0000AA806F0D7FFD4E902010AAA0DF081FFA4
:100DE00028B9D8F8003043F00403C8F800301FB128
:100DF000636BB3427FF469AE269810A907F01AF925
:100E000069E6BBF1000FBFD15FE6F1B2E0E700BFDA
:100E1000280000202DE9F04F2DED028B97B006A998
:100E200081E80C00DDE9243803F16C0404902046CD
:100E300007F024FF08EE100A2046FEF721FA00F121
:100E400040030593836A04461BB1036B003B18BF44
:100E5000012301930CAB0A9300230B938DF83030E0
:100E6000237C1BB120210AA806F05AFF002512ABF3
:100E7000202110A8109311958DF8485006F050FFCE
:100E800004F1440308EE903AE36B08932F462E4694
:100E90000295A946009508AB5B5D042B40D8DFE8BE
:100EA00013F0590128012B00A000DA00BBF1000F5C
:100EB000F1D1D8F8003043F00403C8F8003006AC94
:100EC00022A92046FEF739FF28B1D8F8003043F0B8
:100ED0000203C8F8003094E80300049B83E8030091
:100EE00010A806F029FE0AA806F026FE049817B0FE
:100EF000BDEC028BBDE8F08F249BDB689A051ED405
:100F0000B9F1010F1BD8D5B1012D0CD1019BB3B99B
:100F10009DF82030032B12D09DF82230012B0ED0EB
:100F20004FF0010B2BE0022DFAD19DF82330042B5A
:100F300005D0019A002AF3D0032B40F00E81236ADA
:100F400003934FF0000A22A906A8FEF709FF039BAE
:100F5000834600283CD09A4511D006A8FEF7DEFE55
:100F6000E36953F82A30834235D0BAF1000F40F0DC
:100F7000F780249BDB6883F40073C3F3402B0135B7
:100F8000042D93D1B9F1010F40F22F81BBF1000F75
:100F90008FD0009B002B00F0E680E56A4FF0010B3C
:100FA00022A906A8FEF7DCFE002800F0DE80D94565
:100FB00000F0DE8006A8FEF7B1FE55F82B30834224
:100FC0007FF477AF06A8FEF7AFF90BF1010BE7E767
:100FD0009A45CAD1A4E706A8FEF7A6F90AF1010AC4
:100FE000B1E7A36AB3B9236B43B322A906A8FEF7FE
:100FF000B7FE834610B306A8FEF790FEE26A1268B9
:1010000082421BD106A8D4F83090FEF78DF9CDF8B6
:1010100000B0B4E722A906A8FEF7A2FE8346002886
:10102000E1D006A8FEF77AFE626A12688242DAD13F
:1010300006A8D4F82890FEF777F9A0E7A36A1BB9B1
:10104000019B83F0010B9AE7236B002BF8D101235E
:1010500000939B4693E722A906A8FEF781FE8346EC
:10106000002843D006A8FEF759FE09AA09900A21D4
:1010700018EE900AF9F71DFAA0B1059BA0EB030B3F
:101080005D4B4FEAAB0B1B6810A813F80B1006F072
:1010900079FE06F1010B029E06A8FEF745F90296BD
:1010A0005E46D8E7099962698A4206D12FB9626B18
:1010B000002A11DD5F468346EEE7227C62B1A36918
:1010C000994208D177B97EB1F1B20AA806F05AFE6A
:1010D000BB46029EE0E79346119A002A08BF4FF0F4
:1010E000000B4CE7BB46F7E7B346F5E74FF0010BC3
:1010F000F2E722A906A8FEF733FED8B94FF0000B9D
:10110000032D3FF43CAF22A906A8FEF729FE0028D4
:101110003FF435AF06A8FEF701FE0821024618EE9F
:10112000100AFEF7FEFA00283FF429AF06A8FEF7E2
:10113000FBF8E8E706A8FEF7F1FD0821024618EEE5
:10114000100AFEF7EEFA83460028D7D006A8FEF76D
:10115000EBF8D5E74FF0010BD2E7DDF804B00EE76E
:101160004FF0000B0BE7656A18E7D9457FF4A1AE95
:10117000119B012B11D90022302110A806F0C8FFC5
:10118000024650B1431C08BF11984FF0000108BF40
:1011900000F1FF3210A8FEF7A7F8009B3BB11099B1
:1011A0000B78302B03D02D2210A806F069FE0B9B84
:1011B0008BB1F7B19DF808100AA806F0E3FDD4E959
:1011C00002010AAA0DF08DFD28B9D8F8003043F0CD
:1011D0000403C8F800301FB1636BB3427FF469AEFB
:1011E000269810A906F026FF69E6BBF1000FBFD1D3
:1011F0005FE6F1B2E0E700BF280000202DE9F041F2
:1012000092B008AC84E80C00DDE91B380EAA8C46CD
:101210009DF868100C920CAF00220293CDE9038771
:1012200006460D928DF8382006AD18AB11B393E841
:1012300003008DE80300614694E80C002846FFF7A0
:10124000F5FB95E803000C9D84E80300F5F712F820
:101250001D990B900BAB424628460DF0AFFA94E86F
:10126000030086E80300384606F066FC304612B0FC
:10127000BDE8F08193E803008DE80300614694E83F
:101280000C002846FFF7C6FDDBE72DE9F04F91B0D3
:1012900008ACDDF874B09DF870A006460BF16C0048
:1012A00084E80C00884607F0E9FC1E9BCDE902B3F8
:1012B0000AAF04971AAB814693E803008DE8030058
:1012C0000CAA0A9206AD00220B928DF830204146FE
:1012D00094E80C002846BAF1000F1DD0FFF7A6FBDA
:1012E00095E803000B9D84E8030055B11F9829463B
:1012F0000CF03AFD0A991F9B4A191B684846FEF7F5
:1013000009FA94E8030086E80300384606F014FC66
:10131000304611B0BDE8F08FFFF77CFDE0E700003C
:1013200073B5044616460D4619B912B10D4800F0C2
:1013300049FA731B9A100C2B019207D9002201A9BC
:1013400020460CF063FB019B2060A36020683246BE
:1013500029460CF0F6FB019920460CF051FB02B037
:1013600070BD00BFE49002082DE9F0438DB01C462B
:10137000804602AB68460093FFF7D2FF08AB149A91
:101380000693214606A8FFF7CBFFDDE90097DDE9CC
:10139000065609EB870705EB86062A46494640466E
:1013A0000DF0C7FB044678B9484612F00FFD09EB73
:1013B0008009284612F00AFD4F4505EB80040DD147
:1013C000341B18BF4FF0FF3406A80CF043FB6846EF
:1013D0000CF040FB20460DB0BDE8F083A64203D0E0
:1013E00009F10409251DD8E70124EDE72DE9F047AF
:1013F0001C4600F1080386B0164603600023C0E9CE
:101400000133224602AB05468846684631460093C2
:10141000FFF786FFDDE9007307EB8309214BA21B71
:101420009A424FEA620694BFB0004FF0FF300CF0D2
:10143000E7FE6FF0604A044633463A46214640468E
:101440000DF082FB864211D8461C20460CF0DAFDD6
:10145000564534BFB0004FF0FF300CF0D1FE33469C
:10146000044601463A4640460DF06EFB02462146D0
:1014700028460CF02BFD384612F0A8FC07EB800044
:10148000814505D0071D002128460CF0F6FBD3E767
:1014900020460CF0B7FD68460CF0DCFA284606B092
:1014A000BDE8F087FCFFFF3F184B1A68D1075CBF0F
:1014B00001221A60164B1A68D2075CBF01221A601B
:1014C000144B1A68D0075CBF01221A60124B1A68CD
:1014D000D1075CBF01221A60104B1A68D2075CBFAB
:1014E00001221A600E4B1A68D0075CBF01221A60F5
:1014F0000C4B1A68D1075CBF01221A600A4B1A68AC
:10150000D2075CBF01221A60704700BF8C1B00200D
:10151000881B0020841B0020801B00207C1B0020D7
:10152000781B0020741B0020701B002082B037B590
:1015300006AD85E80C000A9A0B6801920022009221
:101540001D69DDE906230446A847204603B0BDE82F
:10155000304002B0704782B037B506AD85E80C0068
:101560000A9A0B680192002200921D69DDE90623A8
:101570000446A847204603B0BDE8304002B070479B
:1015800010B50446006A0EF039FB216ABDE8104030
:1015900011F0BABD006A0DF0E3BF006A0DF0E0BFC4
:1015A000F8B5069B0D464FF0FF3611464FF0FF375A
:1015B0000022C0E90067C0E9022204467BB1012B8A
:1015C0000CBF01220222286A0EF034F928B9286AD9
:1015D0000EF0EEF9C317C4E900032046F8BD1A4621
:1015E000F1E7F8B5069B0D464FF0FF3611464FF078
:1015F000FF370022C0E90067C0E9022204467BB140
:10160000012B0CBF01220222286A0EF013F928B91F
:10161000286A0EF0CDF9C317C4E900032046F8BDCF
:101620001A46F1E710B50446006A0EF02BFB606223
:1016300010BD034608461B6A01210EF0D1BA38B529
:101640000C46036A0546012120460EF0E5F8002805
:10165000CABF24184FF0FF3314F8013C6B6238BD49
:1016600008B50B465A1C016A04D01846BDE808406C
:101670000FF07ABA08460DF073FF003818BF01204A
:10168000404208BD08B50B465A1C016A04D01846F2
:10169000BDE808400FF0E6BA08460DF061FF0038DB
:1016A00018BF0120404208BDF8B505460E46174652
:1016B0000024BC4208D0296A56F824000FF0D2FA60
:1016C000013001D00134F4E72046F8BD10B5044BD9
:1016D000044640F81C3BF4F723FE204610BD00BF33
:1016E000C0A8020810B50446FFF7F0FF20460CF032
:1016F00087FC204610BD000010B5044B044640F89E
:101700001C3BF4F70DFE204610BD00BF80A8020868
:1017100010B50446FFF7F0FF20460CF071FC2046A0
:1017200010BD10B50446006A0EF068FA606210BD84
:101730004A1C10B50446084602D1606A431C02D018
:10174000216A11F025FD4FF0FF33636210BD10B523
:101750000446006A0EF096FA216ABDE8104011F0C6
:1017600017BDF8B505460E4617460024BC4208D002
:10177000286A0EF087FA431C03D046F8240001348F
:10178000F4E73CB104F18043013B56F823306B622F
:101790002046F8BD4FF0FF33F9E74A1C10B5044668
:1017A000084602D1606A431C02D0216A11F0ACFCE9
:1017B0004FF0FF33636210BD08B50DF0A9FD08B509
:1017C0000DF0A6FD08B50DF0A3FD08B50DF0A0FDC8
:1017D0000FB480B584B000AF07F1180454F8042B9F
:1017E0007A601046EEF74EFD00F2072323F0070360
:1017F000ADEB030D00F500717A68FC602346684686
:1018000005F0C2FF0DF084FD08B50DF081FD00006C
:1018100010B5034B0360044600F01AF9204610BDD2
:1018200080A0020810B5034B0360044600F010F9D5
:10183000204610BD90A0020810B50446FFF7E8FF4F
:1018400020460CF0DDFB204610BD10B50446FFF726
:10185000E9FF20460CF0D4FB204610BD08B5836F8D
:101860000BB941F0010103694161194202D00248FC
:101870000DF096FC08BD00BF64A0020808B54369DE
:101880001943FFF7EBFF08BD70B5C46F0D460CB9E7
:10189000FFF795FF237F4BB92046F9F7E2F923685C
:1018A000294620469B69BDE8704018476118487F6B
:1018B00070BD90F8753010B504463BB92021FFF794
:1018C000E3FF012384F8740084F8753094F8740001
:1018D00010BD38B5044608460D4601F009F910B1AF
:1018E000284600F053FEE067284601F01FF910B1CA
:1018F000284600F003FFC4F88000284601F034F9C0
:1019000010B1284600F018FFC4F8840038BD38B57F
:1019100004460D460DF03DF904F16C012046FFF739
:10192000D8FFA567B5FA85F500236D092367A4F8EC
:1019300074302361656138BD08B5C36F0BB941F0E0
:10194000010103694161194202D002480DF028FCEF
:1019500008BD00BF64A0020808B543691943FFF73A
:10196000EBFF08BD38B5044608460D4607F058FAA7
:1019700010B1284607F082F9C4F88000284607F025
:101980006DFA10B1284607F0B5F9C4F8840028466E
:1019900007F082FA10B1284607F0CAF9C4F88800A7
:1019A00038BD38B504460D460DF0F3F804F16C016E
:1019B0002046FFF7D7FFE567B5FA85F500236D09E7
:1019C000636784F8783023672361656138BD000060
:1019D0000F4B10B500F1240103600023C0E901336F
:1019E000C0E90333C0E90533C0E9073304460A46BA
:1019F0006430C2E9003308329042FAD10823C4E9C6
:101A0000193104F16C00F5F785F9204610BD00BFCF
:101A100010A1020870B5846905460E4634B1D4E9B8
:101A200001322946304698472468F7E770BD38B53B
:101A30000446806940B1C3685A1EC26023B9056874
:101A40000CF0DEFA2846F5E70023A36138BD00005C
:101A50000C4B10B5002104460360FFF7DBFF204666
:101A6000FFF7E5FFA06E04F12403984204D008B10B
:101A70000CF0C8FA0023A36604F16C00F4F750FCE4
:101A8000204610BD10A1020810B50446FFF7E0FF84
:101A900020460CF0B5FA204610BD000010B5064BEC
:101AA0000360143383600023044643600830FFF76B
:101AB000AFFE204610BD00BF2CA10208D0F800C028
:101AC000ACF10C0CDCF800C06044E7E710B5064B45
:101AD0000360143383600023044643600830FFF73B
:101AE000A1FE204610BD00BF5CA10208D0F800C0D6
:101AF000ACF10C0CDCF800C06044E7E710B504461C
:101B0000FFF7CCFF20460CF07BFA204610BDD0F842
:101B100000C0ACF10C0CDCF800C06044EEE710B57E
:101B20000446FFF7D3FF20460CF06AFA204610BDAA
:101B3000D0F800C0ACF10C0CDCF800C06044EEE75B
:101B40000A68026052F80C2C4968815000224260F9
:101B500070470A68026052F80C2C496881500022D4
:101B6000426070478368587C70478368987C7047F0
:101B70008368D86A704783681B6B0020DAB262F30F
:101B80000700C3F3072262F30F20C3F3074262F397
:101B900017401B0E82B063F31F6002B0704783686A
:101BA0005B6B0020DAB262F30700C3F3072262F333
:101BB0000F20C3F3074262F317401B0E82B063F39A
:101BC0001F6002B070478368587C70478368987CB8
:101BD00070478368D86A704783681B6B0020DAB24D
:101BE00062F30700C3F3072262F30F20C3F3074237
:101BF00062F317401B0E82B063F31F6002B07047A0
:101C000083685B6B0020DAB262F30700C3F307223C
